 javaaccessbridge

 Timestamp is ffffffff (Sun Feb  7 06:28:15 2106)

 Preferred load address is 10000000

 Start         Length     Name                   Class
 0001:00000000 0000d143H .text$mn                CODE
 0002:00000000 00000120H .idata$5                DATA
 0002:00000120 00000004H .00cfg                  DATA
 0002:00000124 00000004H .CRT$XCA                DATA
 0002:00000128 00000004H .CRT$XCZ                DATA
 0002:0000012c 00000004H .CRT$XIA                DATA
 0002:00000130 00000004H .CRT$XIZ                DATA
 0002:00000134 00000004H .CRT$XPA                DATA
 0002:00000138 00000004H .CRT$XPZ                DATA
 0002:0000013c 00000004H .CRT$XTA                DATA
 0002:00000140 00000010H .CRT$XTZ                DATA
 0002:00000144 00000000H .gfids$y                DATA
 0002:00000150 0000f3c0H .rdata                  DATA
 0002:0000f510 00000130H .rdata$r                DATA
 0002:0000f640 00000004H .rdata$sxdata           DATA
 0002:0000f644 000002b4H .rdata$zzzdbg           DATA
 0002:0000f8f8 00000004H .rtc$IAA                DATA
 0002:0000f8fc 00000004H .rtc$IZZ                DATA
 0002:0000f900 00000004H .rtc$TAA                DATA
 0002:0000f904 00000004H .rtc$TZZ                DATA
 0002:0000f908 00000118H .xdata$x                DATA
 0002:0000fa20 00000a78H .edata                  DATA
 0002:00010498 000000b4H .idata$2                DATA
 0002:0001054c 00000014H .idata$3                DATA
 0002:00010560 00000120H .idata$4                DATA
 0002:00010680 0000057eH .idata$6                DATA
 0003:00000000 00000018H .data                   DATA
 0003:00000018 00000078H .data$r                 DATA
 0003:00000090 000003a4H .bss                    DATA
 0004:00000000 00000120H .rsrc$01                DATA
 0004:00000120 00000620H .rsrc$02                DATA

  Address         Publics by Value              Rva+Base       Lib:Object

 0000:00000000       ___guard_fids_table        00000000     <absolute>
 0000:00000000       ___guard_iat_count         00000000     <absolute>
 0000:00000000       ___enclave_config          00000000     <absolute>
 0000:00000000       ___hybrid_auxiliary_iat    00000000     <absolute>
 0000:00000000       ___dynamic_value_reloc_table 00000000     <absolute>
 0000:00000000       ___hybrid_code_map         00000000     <absolute>
 0000:00000000       ___hybrid_code_map_count   00000000     <absolute>
 0000:00000000       ___guard_iat_table         00000000     <absolute>
 0000:00000000       ___guard_longjmp_table     00000000     <absolute>
 0000:00000000       ___volatile_metadata       00000000     <absolute>
 0000:00000000       ___guard_longjmp_count     00000000     <absolute>
 0000:00000000       ___guard_fids_count        00000000     <absolute>
 0000:00000001       ___safe_se_handler_count   00000001     <absolute>
 0000:00000100       ___guard_flags             00000100     <absolute>
 0000:00000000       ___ImageBase               10000000     <linker-defined>
 0001:00000000       ??0AccessBridgeATInstance@@QAE@PAUHWND__@@0PADPAV0@@Z 10001000 f   AccessBridgeATInstance.obj
 0001:0000003b       ??1AccessBridgeATInstance@@QAE@XZ 1000103b f   AccessBridgeATInstance.obj
 0001:00000198       ?findABATInstanceFromATHWND@AccessBridgeATInstance@@QAEPAV1@PAUHWND__@@@Z 10001198 f   AccessBridgeATInstance.obj
 0001:000001b7       ?initiateIPC@AccessBridgeATInstance@@QAEJXZ 100011b7 f   AccessBridgeATInstance.obj
 0001:0000027b       ?sendAccessibilityEventPackage@AccessBridgeATInstance@@QAEJPADHJ@Z 1000127b f   AccessBridgeATInstance.obj
 0001:000002b7       ?sendJavaEventPackage@AccessBridgeATInstance@@QAEJPADHJ@Z 100012b7 f   AccessBridgeATInstance.obj
 0001:000002ff       _PrintDebugString          100012ff f   AccessBridgeDebug.obj
 0001:00000349       ___local_stdio_printf_options 10001349 f i AccessBridgeDebug.obj
 0001:0000034f       __vfprintf_l               1000134f f i AccessBridgeDebug.obj
 0001:00000373       __vfwprintf_l              10001373 f i AccessBridgeDebug.obj
 0001:00000397       _finalizeFileLogger        10001397 f   AccessBridgeDebug.obj
 0001:000003b0       _fprintf                   100013b0 f i AccessBridgeDebug.obj
 0001:000003c8       _getTimeStamp              100013c8 f   AccessBridgeDebug.obj
 0001:000003f6       _initializeFileLogger      100013f6 f   AccessBridgeDebug.obj
 0001:000004b8       _printf                    100014b8 f i AccessBridgeDebug.obj
 0001:000004d6       _wPrintJavaDebugString     100014d6 f   AccessBridgeDebug.obj
 0001:000004d6       _wPrintDebugString         100014d6 f   AccessBridgeDebug.obj
 0001:00000520       ??0AccessBridgeJavaEntryPoints@@QAE@PAUJNIEnv_@@PAV_jobject@@@Z 10001520 f   AccessBridgeJavaEntryPoints.obj
 0001:00000545       ?BuildJavaEntryPoints@AccessBridgeJavaEntryPoints@@QAEHXZ 10001545 f   AccessBridgeJavaEntryPoints.obj
 0001:00001ae6       ?CallBooleanMethod@JNIEnv_@@QAAEPAV_jobject@@PAU_jmethodID@@ZZ 10002ae6 f i AccessBridgeJavaEntryPoints.obj
 0001:00001b01       ?CallCharMethod@JNIEnv_@@QAAGPAV_jobject@@PAU_jmethodID@@ZZ 10002b01 f i AccessBridgeJavaEntryPoints.obj
 0001:00001b1c       ?CallFloatMethod@JNIEnv_@@QAAMPAV_jobject@@PAU_jmethodID@@ZZ 10002b1c f i AccessBridgeJavaEntryPoints.obj
 0001:00001b37       ?CallIntMethod@JNIEnv_@@QAAJPAV_jobject@@PAU_jmethodID@@ZZ 10002b37 f i AccessBridgeJavaEntryPoints.obj
 0001:00001b52       ?CallObjectMethod@JNIEnv_@@QAAPAV_jobject@@PAV2@PAU_jmethodID@@ZZ 10002b52 f i AccessBridgeJavaEntryPoints.obj
 0001:00001b6d       ?CallVoidMethod@JNIEnv_@@QAAXPAV_jobject@@PAU_jmethodID@@ZZ 10002b6d f i AccessBridgeJavaEntryPoints.obj
 0001:00001b88       ?activateAccessibleHyperlink@AccessBridgeJavaEntryPoints@@QAEHPAV_jobject@@0@Z 10002b88 f   AccessBridgeJavaEntryPoints.obj
 0001:00001c0c       ?addAccessibilityEventNotification@AccessBridgeJavaEntryPoints@@QAEH_J@Z 10002c0c f   AccessBridgeJavaEntryPoints.obj
 0001:00001ca8       ?addAccessibleSelectionFromContext@AccessBridgeJavaEntryPoints@@QAEXPAV_jobject@@H@Z 10002ca8 f   AccessBridgeJavaEntryPoints.obj
 0001:00001d20       ?addJavaEventNotification@AccessBridgeJavaEntryPoints@@QAEH_J@Z 10002d20 f   AccessBridgeJavaEntryPoints.obj
 0001:00001da0       ?clearAccessibleSelectionFromContext@AccessBridgeJavaEntryPoints@@QAEXPAV_jobject@@@Z 10002da0 f   AccessBridgeJavaEntryPoints.obj
 0001:00001e14       ?doAccessibleActions@AccessBridgeJavaEntryPoints@@QAEHPAV_jobject@@PAUAccessibleActionsToDoTag@@PAJ@Z 10002e14 f   AccessBridgeJavaEntryPoints.obj
 0001:00001f40       ?getAccessibleActions@AccessBridgeJavaEntryPoints@@QAEHPAV_jobject@@PAUAccessibleActionsTag@@@Z 10002f40 f   AccessBridgeJavaEntryPoints.obj
 0001:00002156       ?getAccessibleChildFromContext@AccessBridgeJavaEntryPoints@@QAEPAV_jobject@@PAV2@J@Z 10003156 f   AccessBridgeJavaEntryPoints.obj
 0001:0000222a       ?getAccessibleContextAt@AccessBridgeJavaEntryPoints@@QAEPAV_jobject@@JJPAV2@@Z 1000322a f   AccessBridgeJavaEntryPoints.obj
 0001:000022e6       ?getAccessibleContextFromHWND@AccessBridgeJavaEntryPoints@@QAEPAV_jobject@@J@Z 100032e6 f   AccessBridgeJavaEntryPoints.obj
 0001:00002375       ?getAccessibleContextInfo@AccessBridgeJavaEntryPoints@@QAEHPAV_jobject@@PAUAccessibleContextInfoTag@@@Z 10003375 f   AccessBridgeJavaEntryPoints.obj
 0001:00003199       ?getAccessibleContextWithFocus@AccessBridgeJavaEntryPoints@@QAEPAV_jobject@@XZ 10004199 f   AccessBridgeJavaEntryPoints.obj
 0001:00003237       ?getAccessibleHyperlink@AccessBridgeJavaEntryPoints@@QAEHQAV_jobject@@JPAUAccessibleHyperlinkInfoTag@@@Z 10004237 f   AccessBridgeJavaEntryPoints.obj
 0001:000034a4       ?getAccessibleHyperlinkCount@AccessBridgeJavaEntryPoints@@QAEJQAV_jobject@@@Z 100044a4 f   AccessBridgeJavaEntryPoints.obj
 0001:00003524       ?getAccessibleHypertext@AccessBridgeJavaEntryPoints@@QAEHPAV_jobject@@PAUAccessibleHypertextInfoTag@@@Z 10004524 f   AccessBridgeJavaEntryPoints.obj
 0001:000038b8       ?getAccessibleHypertextExt@AccessBridgeJavaEntryPoints@@QAEHQAV_jobject@@JPAUAccessibleHypertextInfoTag@@@Z 100048b8 f   AccessBridgeJavaEntryPoints.obj
 0001:00003c5a       ?getAccessibleHypertextLinkIndex@AccessBridgeJavaEntryPoints@@QAEJQAV_jobject@@J@Z 10004c5a f   AccessBridgeJavaEntryPoints.obj
 0001:00003ce3       ?getAccessibleIcons@AccessBridgeJavaEntryPoints@@QAEHPAV_jobject@@PAUAccessibleIconsTag@@@Z 10004ce3 f   AccessBridgeJavaEntryPoints.obj
 0001:00003fa7       ?getAccessibleKeyBindings@AccessBridgeJavaEntryPoints@@QAEHPAV_jobject@@PAUAccessibleKeyBindingsTag@@@Z 10004fa7 f   AccessBridgeJavaEntryPoints.obj
 0001:000040e8       ?getAccessibleParentFromContext@AccessBridgeJavaEntryPoints@@QAEPAV_jobject@@PAV2@@Z 100050e8 f   AccessBridgeJavaEntryPoints.obj
 0001:000041b3       ?getAccessibleRelationSet@AccessBridgeJavaEntryPoints@@QAEHPAV_jobject@@PAUAccessibleRelationSetInfoTag@@@Z 100051b3 f   AccessBridgeJavaEntryPoints.obj
 0001:000044a8       ?getAccessibleSelectionCountFromContext@AccessBridgeJavaEntryPoints@@QAEHPAV_jobject@@@Z 100054a8 f   AccessBridgeJavaEntryPoints.obj
 0001:0000452e       ?getAccessibleSelectionFromContext@AccessBridgeJavaEntryPoints@@QAEPAV_jobject@@PAV2@H@Z 1000552e f   AccessBridgeJavaEntryPoints.obj
 0001:000045ff       ?getAccessibleTableCellInfo@AccessBridgeJavaEntryPoints@@QAEHPAV_jobject@@JJPAUAccessibleTableCellInfoTag@@@Z 100055ff f   AccessBridgeJavaEntryPoints.obj
 0001:0000482a       ?getAccessibleTableColumn@AccessBridgeJavaEntryPoints@@QAEJPAV_jobject@@J@Z 1000582a f   AccessBridgeJavaEntryPoints.obj
 0001:000048bc       ?getAccessibleTableColumnDescription@AccessBridgeJavaEntryPoints@@QAEPAV_jobject@@PAV2@J@Z 100058bc f   AccessBridgeJavaEntryPoints.obj
 0001:0000498d       ?getAccessibleTableColumnHeader@AccessBridgeJavaEntryPoints@@QAEHPAV_jobject@@PAUAccessibleTableInfoTag@@@Z 1000598d f   AccessBridgeJavaEntryPoints.obj
 0001:00004af0       ?getAccessibleTableColumnSelectionCount@AccessBridgeJavaEntryPoints@@QAEJPAV_jobject@@@Z 10005af0 f   AccessBridgeJavaEntryPoints.obj
 0001:00004b77       ?getAccessibleTableColumnSelections@AccessBridgeJavaEntryPoints@@QAEHPAV_jobject@@JPAJ@Z 10005b77 f   AccessBridgeJavaEntryPoints.obj
 0001:00004c28       ?getAccessibleTableIndex@AccessBridgeJavaEntryPoints@@QAEJPAV_jobject@@JJ@Z 10005c28 f   AccessBridgeJavaEntryPoints.obj
 0001:00004cc0       ?getAccessibleTableInfo@AccessBridgeJavaEntryPoints@@QAEHPAV_jobject@@PAUAccessibleTableInfoTag@@@Z 10005cc0 f   AccessBridgeJavaEntryPoints.obj
 0001:00004eb0       ?getAccessibleTableRow@AccessBridgeJavaEntryPoints@@QAEJPAV_jobject@@J@Z 10005eb0 f   AccessBridgeJavaEntryPoints.obj
 0001:00004f42       ?getAccessibleTableRowDescription@AccessBridgeJavaEntryPoints@@QAEPAV_jobject@@PAV2@J@Z 10005f42 f   AccessBridgeJavaEntryPoints.obj
 0001:00005013       ?getAccessibleTableRowHeader@AccessBridgeJavaEntryPoints@@QAEHPAV_jobject@@PAUAccessibleTableInfoTag@@@Z 10006013 f   AccessBridgeJavaEntryPoints.obj
 0001:00005176       ?getAccessibleTableRowSelectionCount@AccessBridgeJavaEntryPoints@@QAEJPAV_jobject@@@Z 10006176 f   AccessBridgeJavaEntryPoints.obj
 0001:000051fd       ?getAccessibleTableRowSelections@AccessBridgeJavaEntryPoints@@QAEHPAV_jobject@@JPAJ@Z 100061fd f   AccessBridgeJavaEntryPoints.obj
 0001:000052ae       ?getAccessibleTextAttributes@AccessBridgeJavaEntryPoints@@QAEHPAV_jobject@@JPAUAccessibleTextAttributesInfoTag@@@Z 100062ae f   AccessBridgeJavaEntryPoints.obj
 0001:0000649a       ?getAccessibleTextInfo@AccessBridgeJavaEntryPoints@@QAEHPAV_jobject@@PAUAccessibleTextInfoTag@@JJ@Z 1000749a f   AccessBridgeJavaEntryPoints.obj
 0001:000065f0       ?getAccessibleTextItems@AccessBridgeJavaEntryPoints@@QAEHPAV_jobject@@PAUAccessibleTextItemsInfoTag@@J@Z 100075f0 f   AccessBridgeJavaEntryPoints.obj
 0001:00006a35       ?getAccessibleTextLineBounds@AccessBridgeJavaEntryPoints@@QAEHPAV_jobject@@JPAJ1@Z 10007a35 f   AccessBridgeJavaEntryPoints.obj
 0001:00006b26       ?getAccessibleTextRange@AccessBridgeJavaEntryPoints@@QAEHPAV_jobject@@JJPAGF@Z 10007b26 f   AccessBridgeJavaEntryPoints.obj
 0001:00006d25       ?getAccessibleTextRect@AccessBridgeJavaEntryPoints@@QAEHPAV_jobject@@PAUAccessibleTextRectInfoTag@@J@Z 10007d25 f   AccessBridgeJavaEntryPoints.obj
 0001:00006eb8       ?getAccessibleTextSelectionInfo@AccessBridgeJavaEntryPoints@@QAEHPAV_jobject@@PAUAccessibleTextSelectionInfoTag@@@Z 10007eb8 f   AccessBridgeJavaEntryPoints.obj
 0001:000070ff       ?getActiveDescendent@AccessBridgeJavaEntryPoints@@QAEPAV_jobject@@QAV2@@Z 100080ff f   AccessBridgeJavaEntryPoints.obj
 0001:000071bb       ?getCaretLocation@AccessBridgeJavaEntryPoints@@QAEHPAV_jobject@@PAUAccessibleTextRectInfoTag@@J@Z 100081bb f   AccessBridgeJavaEntryPoints.obj
 0001:0000734e       ?getCurrentAccessibleValueFromContext@AccessBridgeJavaEntryPoints@@QAEHPAV_jobject@@PAGF@Z 1000834e f   AccessBridgeJavaEntryPoints.obj
 0001:000074ea       ?getHWNDFromAccessibleContext@AccessBridgeJavaEntryPoints@@QAEPAUHWND__@@PAV_jobject@@@Z 100084ea f   AccessBridgeJavaEntryPoints.obj
 0001:0000756f       ?getMaximumAccessibleValueFromContext@AccessBridgeJavaEntryPoints@@QAEHPAV_jobject@@PAGF@Z 1000856f f   AccessBridgeJavaEntryPoints.obj
 0001:0000770b       ?getMinimumAccessibleValueFromContext@AccessBridgeJavaEntryPoints@@QAEHPAV_jobject@@PAGF@Z 1000870b f   AccessBridgeJavaEntryPoints.obj
 0001:000078a7       ?getObjectDepth@AccessBridgeJavaEntryPoints@@QAEJQAV_jobject@@@Z 100088a7 f   AccessBridgeJavaEntryPoints.obj
 0001:0000792f       ?getParentWithRole@AccessBridgeJavaEntryPoints@@QAEPAV_jobject@@QAV2@PBG@Z 1000892f f   AccessBridgeJavaEntryPoints.obj
 0001:00007a19       ?getParentWithRoleElseRoot@AccessBridgeJavaEntryPoints@@QAEPAV_jobject@@QAV2@PBG@Z 10008a19 f   AccessBridgeJavaEntryPoints.obj
 0001:00007b03       ?getTextAttributesInRange@AccessBridgeJavaEntryPoints@@QAEHQAV_jobject@@HHPAUAccessibleTextAttributesInfoTag@@PAF@Z 10008b03 f   AccessBridgeJavaEntryPoints.obj
 0001:00007d7d       ?getTopLevelObject@AccessBridgeJavaEntryPoints@@QAEPAV_jobject@@QAV2@@Z 10008d7d f   AccessBridgeJavaEntryPoints.obj
 0001:00007e39       ?getVersionInfo@AccessBridgeJavaEntryPoints@@QAEHPAUAccessBridgeVersionInfoTag@@@Z 10008e39 f   AccessBridgeJavaEntryPoints.obj
 0001:00008032       ?getVirtualAccessibleName@AccessBridgeJavaEntryPoints@@QAEHQAV_jobject@@PAGH@Z 10009032 f   AccessBridgeJavaEntryPoints.obj
 0001:000081db       ?getVisibleChildren@AccessBridgeJavaEntryPoints@@QAEHQAV_jobject@@HPAUVisibleChildenInfoTag@@@Z 100091db f   AccessBridgeJavaEntryPoints.obj
 0001:00008339       ?getVisibleChildrenCount@AccessBridgeJavaEntryPoints@@QAEHQAV_jobject@@@Z 10009339 f   AccessBridgeJavaEntryPoints.obj
 0001:000083ac       ?isAccessibleChildSelectedFromContext@AccessBridgeJavaEntryPoints@@QAEHPAV_jobject@@H@Z 100093ac f   AccessBridgeJavaEntryPoints.obj
 0001:0000843a       ?isAccessibleTableColumnSelected@AccessBridgeJavaEntryPoints@@QAEHPAV_jobject@@J@Z 1000943a f   AccessBridgeJavaEntryPoints.obj
 0001:000084cb       ?isAccessibleTableRowSelected@AccessBridgeJavaEntryPoints@@QAEHPAV_jobject@@J@Z 100094cb f   AccessBridgeJavaEntryPoints.obj
 0001:0000855c       ?isJavaWindow@AccessBridgeJavaEntryPoints@@QAEHJ@Z 1000955c f   AccessBridgeJavaEntryPoints.obj
 0001:000085d5       ?isSameObject@AccessBridgeJavaEntryPoints@@QAEHPAV_jobject@@0@Z 100095d5 f   AccessBridgeJavaEntryPoints.obj
 0001:00008649       ?removeAccessibilityEventNotification@AccessBridgeJavaEntryPoints@@QAEH_J@Z 10009649 f   AccessBridgeJavaEntryPoints.obj
 0001:000086c9       ?removeAccessibleSelectionFromContext@AccessBridgeJavaEntryPoints@@QAEXPAV_jobject@@H@Z 100096c9 f   AccessBridgeJavaEntryPoints.obj
 0001:00008741       ?removeJavaEventNotification@AccessBridgeJavaEntryPoints@@QAEH_J@Z 10009741 f   AccessBridgeJavaEntryPoints.obj
 0001:000087c1       ?requestFocus@AccessBridgeJavaEntryPoints@@QAEHQAV_jobject@@@Z 100097c1 f   AccessBridgeJavaEntryPoints.obj
 0001:00008849       ?selectAllAccessibleSelectionFromContext@AccessBridgeJavaEntryPoints@@QAEXPAV_jobject@@@Z 10009849 f   AccessBridgeJavaEntryPoints.obj
 0001:000088bd       ?selectTextRange@AccessBridgeJavaEntryPoints@@QAEHQAV_jobject@@HH@Z 100098bd f   AccessBridgeJavaEntryPoints.obj
 0001:00008954       ?setCaretPosition@AccessBridgeJavaEntryPoints@@QAEHQAV_jobject@@H@Z 10009954 f   AccessBridgeJavaEntryPoints.obj
 0001:000089e5       ?setTextContents@AccessBridgeJavaEntryPoints@@QAEHQAV_jobject@@PBG@Z 100099e5 f   AccessBridgeJavaEntryPoints.obj
 0001:00008aa0       ?verifyAccessibleText@AccessBridgeJavaEntryPoints@@QAEHPAV_jobject@@@Z 10009aa0 f   AccessBridgeJavaEntryPoints.obj
 0001:00008b8b       ?initBroadcastMessageIDs@@YAHXZ 10009b8b f   AccessBridgeMessages.obj
 0001:00008bbd       ??0JavaAccessBridge@@QAE@PAUHINSTANCE__@@@Z 10009bbd f   JavaAccessBridge.obj
 0001:00008be0       ??1JavaAccessBridge@@QAE@XZ 10009be0 f   JavaAccessBridge.obj
 0001:00008c8b       ?MemoryMappedFileCreated@JavaAccessBridge@@QAEJPAUHWND__@@PAD@Z 10009c8b f   JavaAccessBridge.obj
 0001:00008d07       ?WindowsATDestroyed@JavaAccessBridge@@QAEXPAUHWND__@@@Z 10009d07 f   JavaAccessBridge.obj
 0001:00008d93       ?addAccessibilityEventNotification@JavaAccessBridge@@QAEX_JPAUHWND__@@@Z 10009d93 f   JavaAccessBridge.obj
 0001:00008e25       ?addJavaEventNotification@JavaAccessBridge@@QAEX_JPAUHWND__@@@Z 10009e25 f   JavaAccessBridge.obj
 0001:00008eb7       ?fireCaretUpdate@JavaAccessBridge@@QAEXPAUJNIEnv_@@PAV_jobject@@11@Z 10009eb7 f   JavaAccessBridge.obj
 0001:00008fa6       ?fireFocusGained@JavaAccessBridge@@QAEXPAUJNIEnv_@@PAV_jobject@@11@Z 10009fa6 f   JavaAccessBridge.obj
 0001:00009095       ?fireFocusLost@JavaAccessBridge@@QAEXPAUJNIEnv_@@PAV_jobject@@11@Z 1000a095 f   JavaAccessBridge.obj
 0001:00009184       ?fireMenuCanceled@JavaAccessBridge@@QAEXPAUJNIEnv_@@PAV_jobject@@11@Z 1000a184 f   JavaAccessBridge.obj
 0001:0000927f       ?fireMenuDeselected@JavaAccessBridge@@QAEXPAUJNIEnv_@@PAV_jobject@@11@Z 1000a27f f   JavaAccessBridge.obj
 0001:0000937a       ?fireMenuSelected@JavaAccessBridge@@QAEXPAUJNIEnv_@@PAV_jobject@@11@Z 1000a37a f   JavaAccessBridge.obj
 0001:00009475       ?fireMouseClicked@JavaAccessBridge@@QAEXPAUJNIEnv_@@PAV_jobject@@11@Z 1000a475 f   JavaAccessBridge.obj
 0001:00009564       ?fireMouseEntered@JavaAccessBridge@@QAEXPAUJNIEnv_@@PAV_jobject@@11@Z 1000a564 f   JavaAccessBridge.obj
 0001:00009653       ?fireMouseExited@JavaAccessBridge@@QAEXPAUJNIEnv_@@PAV_jobject@@11@Z 1000a653 f   JavaAccessBridge.obj
 0001:00009742       ?fireMousePressed@JavaAccessBridge@@QAEXPAUJNIEnv_@@PAV_jobject@@11@Z 1000a742 f   JavaAccessBridge.obj
 0001:0000983a       ?fireMouseReleased@JavaAccessBridge@@QAEXPAUJNIEnv_@@PAV_jobject@@11@Z 1000a83a f   JavaAccessBridge.obj
 0001:00009935       ?firePopupMenuCanceled@JavaAccessBridge@@QAEXPAUJNIEnv_@@PAV_jobject@@11@Z 1000a935 f   JavaAccessBridge.obj
 0001:00009a30       ?firePopupMenuWillBecomeInvisible@JavaAccessBridge@@QAEXPAUJNIEnv_@@PAV_jobject@@11@Z 1000aa30 f   JavaAccessBridge.obj
 0001:00009b2b       ?firePopupMenuWillBecomeVisible@JavaAccessBridge@@QAEXPAUJNIEnv_@@PAV_jobject@@11@Z 1000ab2b f   JavaAccessBridge.obj
 0001:00009c26       ?firePropertyActiveDescendentChange@JavaAccessBridge@@QAEXPAUJNIEnv_@@PAV_jobject@@1111@Z 1000ac26 f   JavaAccessBridge.obj
 0001:00009d2f       ?firePropertyCaretChange@JavaAccessBridge@@QAEXPAUJNIEnv_@@PAV_jobject@@11JJ@Z 1000ad2f f   JavaAccessBridge.obj
 0001:00009e11       ?firePropertyChildChange@JavaAccessBridge@@QAEXPAUJNIEnv_@@PAV_jobject@@1111@Z 1000ae11 f   JavaAccessBridge.obj
 0001:00009f1a       ?firePropertyDescriptionChange@JavaAccessBridge@@QAEXPAUJNIEnv_@@PAV_jobject@@11PAV_jstring@@2@Z 1000af1a f   JavaAccessBridge.obj
 0001:0000a0fd       ?firePropertyNameChange@JavaAccessBridge@@QAEXPAUJNIEnv_@@PAV_jobject@@11PAV_jstring@@2@Z 1000b0fd f   JavaAccessBridge.obj
 0001:0000a2e0       ?firePropertySelectionChange@JavaAccessBridge@@QAEXPAUJNIEnv_@@PAV_jobject@@11@Z 1000b2e0 f   JavaAccessBridge.obj
 0001:0000a3aa       ?firePropertyStateChange@JavaAccessBridge@@QAEXPAUJNIEnv_@@PAV_jobject@@11PAV_jstring@@2@Z 1000b3aa f   JavaAccessBridge.obj
 0001:0000a58d       ?firePropertyTableModelChange@JavaAccessBridge@@QAEXPAUJNIEnv_@@PAV_jobject@@11PAV_jstring@@2@Z 1000b58d f   JavaAccessBridge.obj
 0001:0000a776       ?firePropertyTextChange@JavaAccessBridge@@QAEXPAUJNIEnv_@@PAV_jobject@@11@Z 1000b776 f   JavaAccessBridge.obj
 0001:0000a840       ?firePropertyValueChange@JavaAccessBridge@@QAEXPAUJNIEnv_@@PAV_jobject@@11PAV_jstring@@2@Z 1000b840 f   JavaAccessBridge.obj
 0001:0000aa23       ?firePropertyVisibleDataChange@JavaAccessBridge@@QAEXPAUJNIEnv_@@PAV_jobject@@11@Z 1000ba23 f   JavaAccessBridge.obj
 0001:0000aaf0       ?initWindow@JavaAccessBridge@@QAEHXZ 1000baf0 f   JavaAccessBridge.obj
 0001:0000ab1c       ?javaRun@JavaAccessBridge@@QAEXPAUJNIEnv_@@PAV_jobject@@@Z 1000bb1c f   JavaAccessBridge.obj
 0001:0000ac8b       ?javaShutdown@JavaAccessBridge@@QAEXPAUJNIEnv_@@PAV_jobject@@@Z 1000bc8b f   JavaAccessBridge.obj
 0001:0000ad1c       ?postHelloToWindowsDLLMsg@JavaAccessBridge@@QAEXPAUHWND__@@@Z 1000bd1c f   JavaAccessBridge.obj
 0001:0000ad60       ?processPackage@JavaAccessBridge@@QAEJPADH@Z 1000bd60 f   JavaAccessBridge.obj
 0001:0000bd40       ?receiveMemoryPackage@JavaAccessBridge@@QAEHPAUHWND__@@J@Z 1000cd40 f   JavaAccessBridge.obj
 0001:0000bdb3       ?releaseJavaObject@JavaAccessBridge@@QAEXPAV_jobject@@@Z 1000cdb3 f   JavaAccessBridge.obj
 0001:0000be02       ?removeAccessibilityEventNotification@JavaAccessBridge@@QAEX_JPAUHWND__@@@Z 1000ce02 f   JavaAccessBridge.obj
 0001:0000be97       ?removeJavaEventNotification@JavaAccessBridge@@QAEX_JPAUHWND__@@@Z 1000ce97 f   JavaAccessBridge.obj
 0001:0000bf2c       _AccessBridgeDialogProc@16 1000cf2c f   JavaAccessBridge.obj
 0001:0000c030       _DllMain@12                1000d030 f   JavaAccessBridge.obj
 0001:0000c099       _Java_com_sun_java_accessibility_internal_AccessBridge_caretUpdate@16 1000d099 f   JavaAccessBridge.obj
 0001:0000c0a4       _Java_com_sun_java_accessibility_internal_AccessBridge_focusGained@16 1000d0a4 f   JavaAccessBridge.obj
 0001:0000c0af       _Java_com_sun_java_accessibility_internal_AccessBridge_focusLost@16 1000d0af f   JavaAccessBridge.obj
 0001:0000c0ba       _Java_com_sun_java_accessibility_internal_AccessBridge_javaShutdown@8 1000d0ba f   JavaAccessBridge.obj
 0001:0000c0c5       _Java_com_sun_java_accessibility_internal_AccessBridge_jawtGetComponentFromNativeWindowHandle@12 1000d0c5 f   JavaAccessBridge.obj
 0001:0000c0f4       _Java_com_sun_java_accessibility_internal_AccessBridge_jawtGetNativeWindowHandleFromComponent@12 1000d0f4 f   JavaAccessBridge.obj
 0001:0000c140       _Java_com_sun_java_accessibility_internal_AccessBridge_menuCanceled@16 1000d140 f   JavaAccessBridge.obj
 0001:0000c14b       _Java_com_sun_java_accessibility_internal_AccessBridge_menuDeselected@16 1000d14b f   JavaAccessBridge.obj
 0001:0000c156       _Java_com_sun_java_accessibility_internal_AccessBridge_menuSelected@16 1000d156 f   JavaAccessBridge.obj
 0001:0000c161       _Java_com_sun_java_accessibility_internal_AccessBridge_mouseClicked@16 1000d161 f   JavaAccessBridge.obj
 0001:0000c16c       _Java_com_sun_java_accessibility_internal_AccessBridge_mouseEntered@16 1000d16c f   JavaAccessBridge.obj
 0001:0000c177       _Java_com_sun_java_accessibility_internal_AccessBridge_mouseExited@16 1000d177 f   JavaAccessBridge.obj
 0001:0000c182       _Java_com_sun_java_accessibility_internal_AccessBridge_mousePressed@16 1000d182 f   JavaAccessBridge.obj
 0001:0000c18d       _Java_com_sun_java_accessibility_internal_AccessBridge_mouseReleased@16 1000d18d f   JavaAccessBridge.obj
 0001:0000c198       _Java_com_sun_java_accessibility_internal_AccessBridge_popupMenuCanceled@16 1000d198 f   JavaAccessBridge.obj
 0001:0000c1a3       _Java_com_sun_java_accessibility_internal_AccessBridge_popupMenuWillBecomeInvisible@16 1000d1a3 f   JavaAccessBridge.obj
 0001:0000c1ae       _Java_com_sun_java_accessibility_internal_AccessBridge_popupMenuWillBecomeVisible@16 1000d1ae f   JavaAccessBridge.obj
 0001:0000c1b9       _Java_com_sun_java_accessibility_internal_AccessBridge_propertyActiveDescendentChange@24 1000d1b9 f   JavaAccessBridge.obj
 0001:0000c1c8       _Java_com_sun_java_accessibility_internal_AccessBridge_propertyCaretChange@24 1000d1c8 f   JavaAccessBridge.obj
 0001:0000c1d7       _Java_com_sun_java_accessibility_internal_AccessBridge_propertyChildChange@24 1000d1d7 f   JavaAccessBridge.obj
 0001:0000c1e6       _Java_com_sun_java_accessibility_internal_AccessBridge_propertyDescriptionChange@24 1000d1e6 f   JavaAccessBridge.obj
 0001:0000c1f5       _Java_com_sun_java_accessibility_internal_AccessBridge_propertyNameChange@24 1000d1f5 f   JavaAccessBridge.obj
 0001:0000c204       _Java_com_sun_java_accessibility_internal_AccessBridge_propertySelectionChange@16 1000d204 f   JavaAccessBridge.obj
 0001:0000c20f       _Java_com_sun_java_accessibility_internal_AccessBridge_propertyStateChange@24 1000d20f f   JavaAccessBridge.obj
 0001:0000c21e       _Java_com_sun_java_accessibility_internal_AccessBridge_propertyTableModelChange@24 1000d21e f   JavaAccessBridge.obj
 0001:0000c22d       _Java_com_sun_java_accessibility_internal_AccessBridge_propertyTextChange@16 1000d22d f   JavaAccessBridge.obj
 0001:0000c238       _Java_com_sun_java_accessibility_internal_AccessBridge_propertyValueChange@24 1000d238 f   JavaAccessBridge.obj
 0001:0000c247       _Java_com_sun_java_accessibility_internal_AccessBridge_propertyVisibleDataChange@16 1000d247 f   JavaAccessBridge.obj
 0001:0000c252       _Java_com_sun_java_accessibility_internal_AccessBridge_runDLL@8 1000d252 f   JavaAccessBridge.obj
 0001:0000c268       _Java_com_sun_java_accessibility_internal_AccessBridge_sendDebugString@12 1000d268 f   JavaAccessBridge.obj
 0001:0000c2c9       ??2@YAPAXI@Z               1000d2c9 f   MSVCRT:new_scalar.obj
 0001:0000c2f9       ??3@YAXPAXI@Z              1000d2f9 f   MSVCRT:delete_scalar_size.obj
 0001:0000c307       ??_U@YAPAXI@Z              1000d307 f   MSVCRT:new_array.obj
 0001:0000c310       ??_V@YAXPAX@Z              1000d310 f   MSVCRT:delete_array.obj
 0001:0000c320       __aulldiv                  1000d320 f   MSVCRT:ulldiv.obj
 0001:0000c388       @__security_check_cookie@4 1000d388 f   MSVCRT:secchk.obj
 0001:0000c6b9       __DllMainCRTStartup@12     1000d6b9 f   MSVCRT:dll_dllmain.obj
 0001:0000c6dc       ??0bad_alloc@std@@QAE@ABV01@@Z 1000d6dc f i MSVCRT:throw_bad_alloc.obj
 0001:0000c6f7       ??0bad_alloc@std@@QAE@XZ   1000d6f7 f i MSVCRT:throw_bad_alloc.obj
 0001:0000c70f       ??0bad_array_new_length@std@@QAE@ABV01@@Z 1000d70f f i MSVCRT:throw_bad_alloc.obj
 0001:0000c72a       ??0bad_array_new_length@std@@QAE@XZ 1000d72a f i MSVCRT:throw_bad_alloc.obj
 0001:0000c742       ??0exception@std@@QAE@ABV01@@Z 1000d742 f i MSVCRT:throw_bad_alloc.obj
 0001:0000c76e       ??1bad_array_new_length@std@@UAE@XZ 1000d76e f i MSVCRT:throw_bad_alloc.obj
 0001:0000c76e       ??1bad_alloc@std@@UAE@XZ   1000d76e f i MSVCRT:throw_bad_alloc.obj
 0001:0000c77f       ??_Ebad_alloc@std@@UAEPAXI@Z 1000d77f f i MSVCRT:throw_bad_alloc.obj
 0001:0000c77f       ??_Gbad_array_new_length@std@@UAEPAXI@Z 1000d77f f i MSVCRT:throw_bad_alloc.obj
 0001:0000c77f       ??_Gexception@std@@UAEPAXI@Z 1000d77f f i MSVCRT:throw_bad_alloc.obj
 0001:0000c77f       ??_Ebad_array_new_length@std@@UAEPAXI@Z 1000d77f f i MSVCRT:throw_bad_alloc.obj
 0001:0000c77f       ??_Gbad_alloc@std@@UAEPAXI@Z 1000d77f f i MSVCRT:throw_bad_alloc.obj
 0001:0000c77f       ??_Eexception@std@@UAEPAXI@Z 1000d77f f i MSVCRT:throw_bad_alloc.obj
 0001:0000c7ac       ?__scrt_throw_std_bad_alloc@@YAXXZ 1000d7ac f   MSVCRT:throw_bad_alloc.obj
 0001:0000c7c9       ?__scrt_throw_std_bad_array_new_length@@YAXXZ 1000d7c9 f   MSVCRT:throw_bad_alloc.obj
 0001:0000c7e6       ?what@exception@std@@UBEPBDXZ 1000d7e6 f i MSVCRT:throw_bad_alloc.obj
 0001:0000c7f3       ??3@YAXPAX@Z               1000d7f3 f   MSVCRT:delete_scalar.obj
 0001:0000c7f8       ___raise_securityfailure   1000d7f8 f   MSVCRT:gs_report.obj
 0001:0000c820       ___report_gsfailure        1000d820 f   MSVCRT:gs_report.obj
 0001:0000c966       ___security_init_cookie    1000d966 f   MSVCRT:gs_support.obj
 0001:0000c9b1       ?__scrt_initialize_type_info@@YAXXZ 1000d9b1 f   MSVCRT:tncleanup.obj
 0001:0000c9bd       ?__scrt_uninitialize_type_info@@YAXXZ 1000d9bd f   MSVCRT:tncleanup.obj
 0001:0000c9c9       ___local_stdio_scanf_options 1000d9c9 f i MSVCRT:default_local_stdio_options.obj
 0001:0000c9cf       ___scrt_initialize_default_local_stdio_options 1000d9cf f   MSVCRT:default_local_stdio_options.obj
 0001:0000ca30       ___scrt_acquire_startup_lock 1000da30 f   MSVCRT:utility.obj
 0001:0000ca62       ___scrt_dllmain_after_initialize_c 1000da62 f   MSVCRT:utility.obj
 0001:0000ca8d       ___scrt_dllmain_before_initialize_c 1000da8d f   MSVCRT:utility.obj
 0001:0000ca9b       ___scrt_dllmain_crt_thread_attach 1000da9b f   MSVCRT:utility.obj
 0001:0000caba       ___scrt_dllmain_crt_thread_detach 1000daba f   MSVCRT:utility.obj
 0001:0000cac7       ___scrt_dllmain_exception_filter 1000dac7 f   MSVCRT:utility.obj
 0001:0000cafb       ___scrt_dllmain_uninitialize_c 1000dafb f   MSVCRT:utility.obj
 0001:0000cb1e       ___scrt_dllmain_uninitialize_critical 1000db1e f   MSVCRT:utility.obj
 0001:0000cb2b       ___scrt_initialize_crt     1000db2b f   MSVCRT:utility.obj
 0001:0000cb64       ___scrt_initialize_onexit_tables 1000db64 f   MSVCRT:utility.obj
 0001:0000cc09       ___scrt_is_nonwritable_in_current_image 1000dc09 f   MSVCRT:utility.obj
 0001:0000cc9d       ___scrt_release_startup_lock 1000dc9d f   MSVCRT:utility.obj
 0001:0000ccba       ___scrt_uninitialize_crt   1000dcba f   MSVCRT:utility.obj
 0001:0000cce2       ___scrt_get_dyn_tls_init_callback 1000dce2 f   MSVCRT:dyn_tls_init.obj
 0001:0000cce8       ___scrt_fastfail           1000dce8 f   MSVCRT:utility_desktop.obj
 0001:0000ce02       __crt_debugger_hook        1000de02 f   MSVCRT:utility_desktop.obj
 0001:0000ce0a       __RTC_Initialize           1000de0a f   MSVCRT:initsect.obj
 0001:0000ce36       __RTC_Terminate            1000de36 f   MSVCRT:initsect.obj
 0001:0000ce70       __SEH_prolog4              1000de70 f   MSVCRT:sehprolg4.obj
 0001:0000ceb6       __SEH_epilog4              1000deb6 f   MSVCRT:sehprolg4.obj
 0001:0000cecb       __except_handler4          1000decb f   MSVCRT:chandler4gs.obj
 0001:0000ceee       @_guard_check_icall_nop@4  1000deee f i MSVCRT:guard_support.obj
 0001:0000ceef       ??_Gtype_info@@UAEPAXI@Z   1000deef f i MSVCRT:std_type_info_static.obj
 0001:0000ceef       ??_Etype_info@@UAEPAXI@Z   1000deef f i MSVCRT:std_type_info_static.obj
 0001:0000cf12       ___isa_available_init      1000df12 f   MSVCRT:cpu_disp.obj
 0001:0000d0a9       __get_startup_argv_mode    1000e0a9 f   MSVCRT:argv_mode.obj
 0001:0000d0ad       ___scrt_is_ucrt_dll_in_use 1000e0ad f   MSVCRT:ucrt_detection.obj
 0001:0000d0b9       _memcpy                    1000e0b9 f   vcruntime:VCRUNTIME140.dll
 0001:0000d0bf       _memset                    1000e0bf f   vcruntime:VCRUNTIME140.dll
 0001:0000d0c5       ___std_exception_copy      1000e0c5 f   vcruntime:VCRUNTIME140.dll
 0001:0000d0cb       ___std_exception_destroy   1000e0cb f   vcruntime:VCRUNTIME140.dll
 0001:0000d0d1       __CxxThrowException@8      1000e0d1 f   vcruntime:VCRUNTIME140.dll
 0001:0000d0d7       ___std_type_info_destroy_list 1000e0d7 f   vcruntime:VCRUNTIME140.dll
 0001:0000d0dd       __except_handler4_common   1000e0dd f   vcruntime:VCRUNTIME140.dll
 0001:0000d0e3       _strcmp                    1000e0e3 f   ucrt:api-ms-win-crt-string-l1-1-0.dll
 0001:0000d0e9       _strcpy                    1000e0e9 f   ucrt:api-ms-win-crt-string-l1-1-0.dll
 0001:0000d0ef       _strlen                    1000e0ef f   ucrt:api-ms-win-crt-string-l1-1-0.dll
 0001:0000d0f5       __callnewh                 1000e0f5 f   ucrt:api-ms-win-crt-heap-l1-1-0.dll
 0001:0000d0fb       _malloc                    1000e0fb f   ucrt:api-ms-win-crt-heap-l1-1-0.dll
 0001:0000d101       __initterm                 1000e101 f   ucrt:api-ms-win-crt-runtime-l1-1-0.dll
 0001:0000d107       __initterm_e               1000e107 f   ucrt:api-ms-win-crt-runtime-l1-1-0.dll
 0001:0000d10d       _free                      1000e10d f   ucrt:api-ms-win-crt-heap-l1-1-0.dll
 0001:0000d113       __seh_filter_dll           1000e113 f   ucrt:api-ms-win-crt-runtime-l1-1-0.dll
 0001:0000d119       __configure_narrow_argv    1000e119 f   ucrt:api-ms-win-crt-runtime-l1-1-0.dll
 0001:0000d11f       __initialize_narrow_environment 1000e11f f   ucrt:api-ms-win-crt-runtime-l1-1-0.dll
 0001:0000d125       __initialize_onexit_table  1000e125 f   ucrt:api-ms-win-crt-runtime-l1-1-0.dll
 0001:0000d12b       __execute_onexit_table     1000e12b f   ucrt:api-ms-win-crt-runtime-l1-1-0.dll
 0001:0000d131       __cexit                    1000e131 f   ucrt:api-ms-win-crt-runtime-l1-1-0.dll
 0001:0000d137       _IsProcessorFeaturePresent@4 1000e137 f   kernel32:KERNEL32.dll
 0001:0000d13d       ___scrt_stub_for_acrt_thread_attach 1000e13d f   MSVCRT:ucrt_stubs.obj
 0001:0000d13d       ___acrt_uninitialize_critical 1000e13d f   MSVCRT:ucrt_stubs.obj
 0001:0000d13d       ___acrt_thread_attach      1000e13d f   MSVCRT:ucrt_stubs.obj
 0001:0000d13d       ___scrt_stub_for_acrt_thread_detach 1000e13d f   MSVCRT:ucrt_stubs.obj
 0001:0000d13d       ___acrt_thread_detach      1000e13d f   MSVCRT:ucrt_stubs.obj
 0001:0000d13d       ___acrt_uninitialize       1000e13d f   MSVCRT:ucrt_stubs.obj
 0001:0000d13d       ___vcrt_thread_attach      1000e13d f   MSVCRT:ucrt_stubs.obj
 0001:0000d13d       ___acrt_initialize         1000e13d f   MSVCRT:ucrt_stubs.obj
 0001:0000d13d       ___scrt_stub_for_acrt_initialize 1000e13d f   MSVCRT:ucrt_stubs.obj
 0001:0000d13d       ___scrt_stub_for_acrt_uninitialize_critical 1000e13d f   MSVCRT:ucrt_stubs.obj
 0001:0000d13d       ___vcrt_thread_detach      1000e13d f   MSVCRT:ucrt_stubs.obj
 0001:0000d13d       ___vcrt_initialize         1000e13d f   MSVCRT:ucrt_stubs.obj
 0001:0000d13d       ___vcrt_uninitialize       1000e13d f   MSVCRT:ucrt_stubs.obj
 0001:0000d13d       ___vcrt_uninitialize_critical 1000e13d f   MSVCRT:ucrt_stubs.obj
 0001:0000d13d       ___scrt_stub_for_acrt_uninitialize 1000e13d f   MSVCRT:ucrt_stubs.obj
 0001:0000d140       __is_c_termination_complete 1000e140 f   MSVCRT:ucrt_stubs.obj
 0001:0000d140       ___scrt_stub_for_is_c_termination_complete 1000e140 f   MSVCRT:ucrt_stubs.obj
 0002:00000000       __imp__CloseHandle@4       1000f000     kernel32:KERNEL32.dll
 0002:00000004       __imp__GetLastError@0      1000f004     kernel32:KERNEL32.dll
 0002:00000008       __imp__MapViewOfFile@20    1000f008     kernel32:KERNEL32.dll
 0002:0000000c       __imp__UnmapViewOfFile@4   1000f00c     kernel32:KERNEL32.dll
 0002:00000010       __imp__OpenFileMappingA@12 1000f010     kernel32:KERNEL32.dll
 0002:00000014       __imp__GetSystemTimeAsFileTime@4 1000f014     kernel32:KERNEL32.dll
 0002:00000018       __imp__InitializeCriticalSection@4 1000f018     kernel32:KERNEL32.dll
 0002:0000001c       __imp__EnterCriticalSection@4 1000f01c     kernel32:KERNEL32.dll
 0002:00000020       __imp__LeaveCriticalSection@4 1000f020     kernel32:KERNEL32.dll
 0002:00000024       __imp__DeleteCriticalSection@4 1000f024     kernel32:KERNEL32.dll
 0002:00000028       __imp__Sleep@4             1000f028     kernel32:KERNEL32.dll
 0002:0000002c       __imp__IsDebuggerPresent@0 1000f02c     kernel32:KERNEL32.dll
 0002:00000030       __imp__InitializeSListHead@4 1000f030     kernel32:KERNEL32.dll
 0002:00000034       __imp__GetCurrentThreadId@0 1000f034     kernel32:KERNEL32.dll
 0002:00000038       __imp__GetCurrentProcessId@0 1000f038     kernel32:KERNEL32.dll
 0002:0000003c       __imp__QueryPerformanceCounter@4 1000f03c     kernel32:KERNEL32.dll
 0002:00000040       __imp__IsProcessorFeaturePresent@4 1000f040     kernel32:KERNEL32.dll
 0002:00000044       __imp__TerminateProcess@8  1000f044     kernel32:KERNEL32.dll
 0002:00000048       __imp__GetCurrentProcess@0 1000f048     kernel32:KERNEL32.dll
 0002:0000004c       __imp__SetUnhandledExceptionFilter@4 1000f04c     kernel32:KERNEL32.dll
 0002:00000050       __imp__UnhandledExceptionFilter@4 1000f050     kernel32:KERNEL32.dll
 0002:00000054       \177KERNEL32_NULL_THUNK_DATA 1000f054     kernel32:KERNEL32.dll
 0002:00000058       __imp__TranslateMessage@4  1000f058     user32:USER32.dll
 0002:0000005c       __imp__CreateDialogParamA@20 1000f05c     user32:USER32.dll
 0002:00000060       __imp__RegisterWindowMessageA@4 1000f060     user32:USER32.dll
 0002:00000064       __imp__PostQuitMessage@4   1000f064     user32:USER32.dll
 0002:00000068       __imp__PostThreadMessageA@16 1000f068     user32:USER32.dll
 0002:0000006c       __imp__PostMessageA@16     1000f06c     user32:USER32.dll
 0002:00000070       __imp__SendMessageA@16     1000f070     user32:USER32.dll
 0002:00000074       __imp__GetMessageA@16      1000f074     user32:USER32.dll
 0002:00000078       __imp__DispatchMessageA@4  1000f078     user32:USER32.dll
 0002:0000007c       \177USER32_NULL_THUNK_DATA 1000f07c     user32:USER32.dll
 0002:00000080       __imp____std_type_info_destroy_list 1000f080     vcruntime:VCRUNTIME140.dll
 0002:00000084       __imp___CxxThrowException@8 1000f084     vcruntime:VCRUNTIME140.dll
 0002:00000088       __imp____std_exception_destroy 1000f088     vcruntime:VCRUNTIME140.dll
 0002:0000008c       __imp___except_handler4_common 1000f08c     vcruntime:VCRUNTIME140.dll
 0002:00000090       __imp__memset              1000f090     vcruntime:VCRUNTIME140.dll
 0002:00000094       __imp____std_exception_copy 1000f094     vcruntime:VCRUNTIME140.dll
 0002:00000098       __imp__memcpy              1000f098     vcruntime:VCRUNTIME140.dll
 0002:0000009c       \177VCRUNTIME140_NULL_THUNK_DATA 1000f09c     vcruntime:VCRUNTIME140.dll
 0002:000000a0       __imp__getenv              1000f0a0     ucrt:api-ms-win-crt-environment-l1-1-0.dll
 0002:000000a4       \177api-ms-win-crt-environment-l1-1-0_NULL_THUNK_DATA 1000f0a4     ucrt:api-ms-win-crt-environment-l1-1-0.dll
 0002:000000a8       __imp__free                1000f0a8     ucrt:api-ms-win-crt-heap-l1-1-0.dll
 0002:000000ac       __imp__malloc              1000f0ac     ucrt:api-ms-win-crt-heap-l1-1-0.dll
 0002:000000b0       __imp___callnewh           1000f0b0     ucrt:api-ms-win-crt-heap-l1-1-0.dll
 0002:000000b4       \177api-ms-win-crt-heap-l1-1-0_NULL_THUNK_DATA 1000f0b4     ucrt:api-ms-win-crt-heap-l1-1-0.dll
 0002:000000b8       __imp___beginthreadex      1000f0b8     ucrt:api-ms-win-crt-runtime-l1-1-0.dll
 0002:000000bc       __imp___initterm           1000f0bc     ucrt:api-ms-win-crt-runtime-l1-1-0.dll
 0002:000000c0       __imp___initterm_e         1000f0c0     ucrt:api-ms-win-crt-runtime-l1-1-0.dll
 0002:000000c4       __imp___seh_filter_dll     1000f0c4     ucrt:api-ms-win-crt-runtime-l1-1-0.dll
 0002:000000c8       __imp___configure_narrow_argv 1000f0c8     ucrt:api-ms-win-crt-runtime-l1-1-0.dll
 0002:000000cc       __imp___initialize_narrow_environment 1000f0cc     ucrt:api-ms-win-crt-runtime-l1-1-0.dll
 0002:000000d0       __imp___initialize_onexit_table 1000f0d0     ucrt:api-ms-win-crt-runtime-l1-1-0.dll
 0002:000000d4       __imp___execute_onexit_table 1000f0d4     ucrt:api-ms-win-crt-runtime-l1-1-0.dll
 0002:000000d8       __imp___cexit              1000f0d8     ucrt:api-ms-win-crt-runtime-l1-1-0.dll
 0002:000000dc       \177api-ms-win-crt-runtime-l1-1-0_NULL_THUNK_DATA 1000f0dc     ucrt:api-ms-win-crt-runtime-l1-1-0.dll
 0002:000000e0       __imp__fclose              1000f0e0     ucrt:api-ms-win-crt-stdio-l1-1-0.dll
 0002:000000e4       __imp____acrt_iob_func     1000f0e4     ucrt:api-ms-win-crt-stdio-l1-1-0.dll
 0002:000000e8       __imp__fopen               1000f0e8     ucrt:api-ms-win-crt-stdio-l1-1-0.dll
 0002:000000ec       __imp____stdio_common_vfprintf 1000f0ec     ucrt:api-ms-win-crt-stdio-l1-1-0.dll
 0002:000000f0       __imp____stdio_common_vfwprintf 1000f0f0     ucrt:api-ms-win-crt-stdio-l1-1-0.dll
 0002:000000f4       \177api-ms-win-crt-stdio-l1-1-0_NULL_THUNK_DATA 1000f0f4     ucrt:api-ms-win-crt-stdio-l1-1-0.dll
 0002:000000f8       __imp__strcmp              1000f0f8     ucrt:api-ms-win-crt-string-l1-1-0.dll
 0002:000000fc       __imp__wcsncpy             1000f0fc     ucrt:api-ms-win-crt-string-l1-1-0.dll
 0002:00000100       __imp__wcslen              1000f100     ucrt:api-ms-win-crt-string-l1-1-0.dll
 0002:00000104       __imp__wcscmp              1000f104     ucrt:api-ms-win-crt-string-l1-1-0.dll
 0002:00000108       __imp__strcpy              1000f108     ucrt:api-ms-win-crt-string-l1-1-0.dll
 0002:0000010c       __imp__strlen              1000f10c     ucrt:api-ms-win-crt-string-l1-1-0.dll
 0002:00000110       __imp__strncpy             1000f110     ucrt:api-ms-win-crt-string-l1-1-0.dll
 0002:00000114       \177api-ms-win-crt-string-l1-1-0_NULL_THUNK_DATA 1000f114     ucrt:api-ms-win-crt-string-l1-1-0.dll
 0002:00000118       __imp__JAWT_GetAWT@8       1000f118     jawt:jawt.dll
 0002:0000011c       \177jawt_NULL_THUNK_DATA   1000f11c     jawt:jawt.dll
 0002:00000120       ___guard_check_icall_fptr  1000f120     MSVCRT:guard_support.obj
 0002:00000124       ___xc_a                    1000f124     MSVCRT:initializers.obj
 0002:00000128       ___xc_z                    1000f128     MSVCRT:initializers.obj
 0002:0000012c       ___xi_a                    1000f12c     MSVCRT:initializers.obj
 0002:00000130       ___xi_z                    1000f130     MSVCRT:initializers.obj
 0002:00000134       ___xp_a                    1000f134     MSVCRT:initializers.obj
 0002:00000138       ___xp_z                    1000f138     MSVCRT:initializers.obj
 0002:0000013c       ___xt_a                    1000f13c     MSVCRT:initializers.obj
 0002:00000140       ___xt_z                    1000f140     MSVCRT:initializers.obj
 0002:00000150       ??_C@_0DL@PNCLIPJM@?$FLINFO?$FN?3?5in?5AccessBridgeATInstan@ 1000f150     AccessBridgeATInstance.obj
 0002:0000018c       ??_C@_0DA@ILNDDPNA@?$FLINFO?$FN?3?5?5?5unmapping?5memoryMappe@ 1000f18c     AccessBridgeATInstance.obj
 0002:000001bc       ??_C@_0DJ@FCAPEKK@?$FLINFO?$FN?3?5?5?5closing?5memoryMappedF@ 1000f1bc     AccessBridgeATInstance.obj
 0002:000001f8       ??_C@_0DB@BBBKEEOJ@?$FLINFO?$FN?3?5In?5AccessBridgeATInstan@ 1000f1f8     AccessBridgeATInstance.obj
 0002:0000022c       ??_C@_0DJ@HCNGCGLH@?$FLERROR?$FN?3?5?5?5Failed?5to?5CreateFile@ 1000f22c     AccessBridgeATInstance.obj
 0002:00000268       ??_C@_0DC@INNGAKAO@?$FLINFO?$FN?3?5?5?5CreateFileMapping?5wor@ 1000f268     AccessBridgeATInstance.obj
 0002:0000029c       ??_C@_0DF@EKLGABNF@?$FLERROR?$FN?3?5?5?5Failed?5to?5MapViewOfF@ 1000f29c     AccessBridgeATInstance.obj
 0002:000002d4       ??_C@_0CK@LMLFEIHL@?$FLINFO?$FN?3?5?5?5MapViewOfFile?5worked?5@ 1000f2d4     AccessBridgeATInstance.obj
 0002:00000300       ??_C@_03DJNNCAJF@OK?$DP@   1000f300     AccessBridgeATInstance.obj
 0002:00000304       ??_C@_0DL@FPNEIEFH@?$FLERROR?$FN?3?5?5?5JavaVM?5failed?5to?5wri@ 1000f304     AccessBridgeATInstance.obj
 0002:00000340       ??_C@_0CN@CCHCHAPN@?$FLINFO?$FN?3?5?5?5JavaVM?5successfully?5w@ 1000f340     AccessBridgeATInstance.obj
 0002:00000370       ??_C@_03ONJMBPEK@OK?$CB@   1000f370     AccessBridgeATInstance.obj
 0002:00000378       ??_C@_0EE@MNPDBEBN@?$FLINFO?$FN?3?5AccessBridgeATInstance?3@ 1000f378     AccessBridgeATInstance.obj
 0002:000003c0       ??_C@_0FI@KACFLKHC@?$FLINFO?$FN?3?5AccessBridgeATInstance?3@ 1000f3c0     AccessBridgeATInstance.obj
 0002:00000418       ??_C@_0EN@DDCKACNO@?$FLINFO?$FN?3?5AccessBridgeATInstance?3@ 1000f418     AccessBridgeATInstance.obj
 0002:00000468       ??_C@_0BJ@FKCDJFDK@JAVA_ACCESSBRIDGE_LOGDIR@ 1000f468     AccessBridgeDebug.obj
 0002:00000484       ??_C@_04FPOLKAEB@?4log@    1000f484     AccessBridgeDebug.obj
 0002:0000048c       ??_C@_01NOFIACDB@w@        1000f48c     AccessBridgeDebug.obj
 0002:00000490       ??_C@_04EINJHBMM@?6?$CFs?6@ 1000f490     AccessBridgeDebug.obj
 0002:00000498       ??_C@_0BH@PPBGFLKL@Could?5not?5open?5file?5?$CFs@ 1000f498     AccessBridgeDebug.obj
 0002:000004b0       ??_C@_07IBOBEFLP@?$FL?$CFllu?$FN?5@ 1000f4b0     AccessBridgeDebug.obj
 0002:000004b8       ??_C@_02PCIJFNDE@?$AN?6@   1000f4b8     AccessBridgeDebug.obj
 0002:000004bc       ??_C@_0DD@HABIDLLD@?$FLINFO?$FN?3?5AccessBridgeJavaEntryPo@ 1000f4bc     AccessBridgeJavaEntryPoints.obj
 0002:000004f0       ??_C@_0CI@FJHGEAOO@?$FLINFO?$FN?3?5Calling?5BuildJavaEntryP@ 1000f4f0     AccessBridgeJavaEntryPoints.obj
 0002:00000518       ??_C@_0DB@PHGNIPBB@com?1sun?1java?1accessibility?1inte@ 1000f518     AccessBridgeJavaEntryPoints.obj
 0002:0000054c       ??_C@_0CP@OJHOIDNH@?$FLERROR?$FN?3?5?5FindClass?$CI?$CFs?$CJ?5failed?$CB@ 1000f54c     AccessBridgeJavaEntryPoints.obj
 0002:0000057c       ??_C@_0DE@FJPDGHPE@?$FLERROR?$FN?3?5FindClass?$CI?$CFs?$CJ?5failed?$CB?5@ 1000f57c     AccessBridgeJavaEntryPoints.obj
 0002:000005b0       ??_C@_0BG@JLFLBLJI@?$CILjava?1lang?1Object?$DL?$CJV@ 1000f5b0     AccessBridgeJavaEntryPoints.obj
 0002:000005c8       ??_C@_0BD@PAIEAHIF@decrementReference@ 1000f5c8     AccessBridgeJavaEntryPoints.obj
 0002:000005dc       ??_C@_0DP@BBIEPKKN@?$FLERROR?$FN?3?5GetMethodID?$CI?$CFs?$CJ?5failed@ 1000f5dc     AccessBridgeJavaEntryPoints.obj
 0002:0000061c       ??_C@_0BF@FOHFOJOB@?$CI?$CJLjava?1lang?1String?$DL@ 1000f61c     AccessBridgeJavaEntryPoints.obj
 0002:00000634       ??_C@_0BH@KKNMIJGK@getJavaVersionProperty@ 1000f634     AccessBridgeJavaEntryPoints.obj
 0002:0000064c       ??_C@_04FJLILDCB@?$CII?$CJZ@ 1000f64c     AccessBridgeJavaEntryPoints.obj
 0002:00000654       ??_C@_0N@MHDJENGP@isJavaWindow@ 1000f654     AccessBridgeJavaEntryPoints.obj
 0002:00000664       ??_C@_0CL@DDDHKJEI@?$CII?$CJLjavax?1accessibility?1Accessi@ 1000f664     AccessBridgeJavaEntryPoints.obj
 0002:00000690       ??_C@_0CB@JPFPCEPL@getContextFromNativeWindowHandl@ 1000f690     AccessBridgeJavaEntryPoints.obj
 0002:000006b4       ??_C@_0CL@LNFAHLDN@?$CILjavax?1accessibility?1Accessibl@ 1000f6b4     AccessBridgeJavaEntryPoints.obj
 0002:000006e0       ??_C@_0CB@OGDNEJKI@getNativeWindowHandleFromContex@ 1000f6e0     AccessBridgeJavaEntryPoints.obj
 0002:00000708       ??_C@_0FB@EAOFMHCM@?$CILjavax?1accessibility?1Accessibl@ 1000f708     AccessBridgeJavaEntryPoints.obj
 0002:0000075c       ??_C@_0BP@OKMFCEDC@getAccessibleParentFromContext@ 1000f75c     AccessBridgeJavaEntryPoints.obj
 0002:0000077c       ??_C@_0DN@EHCPLCMJ@?$CILjavax?1accessibility?1Accessibl@ 1000f77c     AccessBridgeJavaEntryPoints.obj
 0002:000007bc       ??_C@_0BA@NNDOMDNC@setTextContents@ 1000f7bc     AccessBridgeJavaEntryPoints.obj
 0002:000007d0       ??_C@_0GD@DBHMDOGO@?$CILjavax?1accessibility?1Accessibl@ 1000f7d0     AccessBridgeJavaEntryPoints.obj
 0002:00000834       ??_C@_0BC@EHMJEOIE@getParentWithRole@ 1000f834     AccessBridgeJavaEntryPoints.obj
 0002:00000848       ??_C@_0BC@CBIPDOMM@getTopLevelObject@ 1000f848     AccessBridgeJavaEntryPoints.obj
 0002:0000085c       ??_C@_0BK@KAMHKCND@getParentWithRoleElseRoot@ 1000f85c     AccessBridgeJavaEntryPoints.obj
 0002:00000878       ??_C@_0P@POFHEAF@getObjectDepth@ 1000f878     AccessBridgeJavaEntryPoints.obj
 0002:00000888       ??_C@_0BE@CDLLPKAM@getActiveDescendent@ 1000f888     AccessBridgeJavaEntryPoints.obj
 0002:000008a0       ??_C@_0FD@CINPJKCJ@?$CIIILjavax?1accessibility?1Accessi@ 1000f8a0     AccessBridgeJavaEntryPoints.obj
 0002:000008f4       ??_C@_0BH@BIEKBJIN@getAccessibleContextAt@ 1000f8f4     AccessBridgeJavaEntryPoints.obj
 0002:0000090c       ??_C@_0CK@DOBCJGDO@?$CI?$CJLjavax?1accessibility?1Accessib@ 1000f90c     AccessBridgeJavaEntryPoints.obj
 0002:00000938       ??_C@_0BO@BAFCPPBG@getAccessibleContextWithFocus@ 1000f938     AccessBridgeJavaEntryPoints.obj
 0002:00000958       ??_C@_0DM@JMIIJMDP@?$CILjavax?1accessibility?1Accessibl@ 1000f958     AccessBridgeJavaEntryPoints.obj
 0002:00000994       ??_C@_0BN@DPBDCOIO@getAccessibleNameFromContext@ 1000f994     AccessBridgeJavaEntryPoints.obj
 0002:000009b4       ??_C@_0CE@IOFJICIE@getAccessibleDescriptionFromCon@ 1000f9b4     AccessBridgeJavaEntryPoints.obj
 0002:000009d8       ??_C@_0CD@DDGCACMP@getAccessibleRoleStringFromCont@ 1000f9d8     AccessBridgeJavaEntryPoints.obj
 0002:000009fc       ??_C@_0CJ@OOFFKIOD@getAccessibleRoleStringFromCont@ 1000f9fc     AccessBridgeJavaEntryPoints.obj
 0002:00000a28       ??_C@_0CF@JIKEBCCK@getAccessibleStatesStringFromCo@ 1000fa28     AccessBridgeJavaEntryPoints.obj
 0002:00000a50       ??_C@_0CL@EODHLGAL@getAccessibleStatesStringFromCo@ 1000fa50     AccessBridgeJavaEntryPoints.obj
 0002:00000a7c       ??_C@_0CG@LAIPJCLP@getAccessibleIndexInParentFromC@ 1000fa7c     AccessBridgeJavaEntryPoints.obj
 0002:00000aa4       ??_C@_0CG@KMCKGMOL@getAccessibleChildrenCountFromC@ 1000faa4     AccessBridgeJavaEntryPoints.obj
 0002:00000ad0       ??_C@_0FC@MAPACPFB@?$CILjavax?1accessibility?1Accessibl@ 1000fad0     AccessBridgeJavaEntryPoints.obj
 0002:00000b24       ??_C@_0BO@BJCAFAFF@getAccessibleChildFromContext@ 1000fb24     AccessBridgeJavaEntryPoints.obj
 0002:00000b44       ??_C@_0DO@DCCADJME@?$CILjavax?1accessibility?1Accessibl@ 1000fb44     AccessBridgeJavaEntryPoints.obj
 0002:00000b84       ??_C@_0CH@EEFIDNHA@getAccessibleBoundsOnScreenFrom@ 1000fb84     AccessBridgeJavaEntryPoints.obj
 0002:00000bac       ??_C@_0BP@FJIKBALD@getAccessibleXcoordFromContext@ 1000fbac     AccessBridgeJavaEntryPoints.obj
 0002:00000bcc       ??_C@_0BP@LGNIKGFC@getAccessibleYcoordFromContext@ 1000fbcc     AccessBridgeJavaEntryPoints.obj
 0002:00000bec       ??_C@_0BP@EMIHBOON@getAccessibleHeightFromContext@ 1000fbec     AccessBridgeJavaEntryPoints.obj
 0002:00000c0c       ??_C@_0BO@OAEOJGNL@getAccessibleWidthFromContext@ 1000fc0c     AccessBridgeJavaEntryPoints.obj
 0002:00000c30       ??_C@_0FD@DOBAJOLJ@?$CILjavax?1accessibility?1Accessibl@ 1000fc30     AccessBridgeJavaEntryPoints.obj
 0002:00000c84       ??_C@_0CC@MHPILDJI@getAccessibleComponentFromConte@ 1000fc84     AccessBridgeJavaEntryPoints.obj
 0002:00000ca8       ??_C@_0FA@DEIINAGF@?$CILjavax?1accessibility?1Accessibl@ 1000fca8     AccessBridgeJavaEntryPoints.obj
 0002:00000cf8       ??_C@_0BP@PKDLLPIG@getAccessibleActionFromContext@ 1000fcf8     AccessBridgeJavaEntryPoints.obj
 0002:00000d18       ??_C@_0FD@KNPEAGPM@?$CILjavax?1accessibility?1Accessibl@ 1000fd18     AccessBridgeJavaEntryPoints.obj
 0002:00000d6c       ??_C@_0CC@BHJMNIGA@getAccessibleSelectionFromConte@ 1000fd6c     AccessBridgeJavaEntryPoints.obj
 0002:00000d90       ??_C@_0EO@JMGLFFGI@?$CILjavax?1accessibility?1Accessibl@ 1000fd90     AccessBridgeJavaEntryPoints.obj
 0002:00000de0       ??_C@_0BN@CMHLOCAB@getAccessibleTextFromContext@ 1000fde0     AccessBridgeJavaEntryPoints.obj
 0002:00000e00       ??_C@_0EP@DILHGLKF@?$CILjavax?1accessibility?1Accessibl@ 1000fe00     AccessBridgeJavaEntryPoints.obj
 0002:00000e50       ??_C@_0BO@BFBIPFI@getAccessibleValueFromContext@ 1000fe50     AccessBridgeJavaEntryPoints.obj
 0002:00000e70       ??_C@_0EP@DNAJNMPI@?$CILjavax?1accessibility?1Accessibl@ 1000fe70     AccessBridgeJavaEntryPoints.obj
 0002:00000ec0       ??_C@_0BO@PAPKMEMG@getAccessibleTableFromContext@ 1000fec0     AccessBridgeJavaEntryPoints.obj
 0002:00000ee0       ??_C@_0EP@HGIIMPLK@?$CILjavax?1accessibility?1Accessibl@ 1000fee0     AccessBridgeJavaEntryPoints.obj
 0002:00000f30       ??_C@_0BO@PDGALDAF@getContextFromAccessibleTable@ 1000ff30     AccessBridgeJavaEntryPoints.obj
 0002:00000f50       ??_C@_0BM@FOJGHDMD@getAccessibleTableRowHeader@ 1000ff50     AccessBridgeJavaEntryPoints.obj
 0002:00000f6c       ??_C@_0BP@FNCIHNLO@getAccessibleTableColumnHeader@ 1000ff6c     AccessBridgeJavaEntryPoints.obj
 0002:00000f8c       ??_C@_0BL@FHMDFDAE@getAccessibleTableRowCount@ 1000ff8c     AccessBridgeJavaEntryPoints.obj
 0002:00000fa8       ??_C@_0BO@FPCPCCIG@getAccessibleTableColumnCount@ 1000ffa8     AccessBridgeJavaEntryPoints.obj
 0002:00000fc8       ??_C@_0FB@MHAEKEPL@?$CILjavax?1accessibility?1Accessibl@ 1000ffc8     AccessBridgeJavaEntryPoints.obj
 0002:0000101c       ??_C@_0CI@CIBBMNLI@getAccessibleTableCellAccessibl@ 1001001c     AccessBridgeJavaEntryPoints.obj
 0002:00001044       ??_C@_0CL@HMHFCPKO@?$CILjavax?1accessibility?1Accessibl@ 10010044     AccessBridgeJavaEntryPoints.obj
 0002:00001070       ??_C@_0BM@BBCGJJGP@getAccessibleTableCellIndex@ 10010070     AccessBridgeJavaEntryPoints.obj
 0002:0000108c       ??_C@_0CA@MEOFLNBC@getAccessibleTableCellRowExtent@ 1001008c     AccessBridgeJavaEntryPoints.obj
 0002:000010ac       ??_C@_0CD@GOAKABO@getAccessibleTableCellColumnExt@ 100100ac     AccessBridgeJavaEntryPoints.obj
 0002:000010d0       ??_C@_0CL@BNJKGODM@?$CILjavax?1accessibility?1Accessibl@ 100100d0     AccessBridgeJavaEntryPoints.obj
 0002:000010fc       ??_C@_0BO@KIDDCDEB@isAccessibleTableCellSelected@ 100100fc     AccessBridgeJavaEntryPoints.obj
 0002:0000111c       ??_C@_0CE@NOEAKJPM@getAccessibleTableRowHeaderRowC@ 1001011c     AccessBridgeJavaEntryPoints.obj
 0002:00001140       ??_C@_0CH@NOEKFODF@getAccessibleTableColumnHeaderR@ 10010140     AccessBridgeJavaEntryPoints.obj
 0002:00001168       ??_C@_0CH@HOBKNLMK@getAccessibleTableRowHeaderColu@ 10010168     AccessBridgeJavaEntryPoints.obj
 0002:00001190       ??_C@_0CK@FLEMOIGB@getAccessibleTableColumnHeaderC@ 10010190     AccessBridgeJavaEntryPoints.obj
 0002:000011c0       ??_C@_0FA@NJKKHECI@?$CILjavax?1accessibility?1Accessibl@ 100101c0     AccessBridgeJavaEntryPoints.obj
 0002:00001210       ??_C@_0CB@KCKFJBAJ@getAccessibleTableRowDescriptio@ 10010210     AccessBridgeJavaEntryPoints.obj
 0002:00001234       ??_C@_0CE@KHNFECJN@getAccessibleTableColumnDescrip@ 10010234     AccessBridgeJavaEntryPoints.obj
 0002:00001258       ??_C@_0CJ@HGNCMOOJ@?$CILjavax?1accessibility?1Accessibl@ 10010258     AccessBridgeJavaEntryPoints.obj
 0002:00001284       ??_C@_0CE@CDNGIBEK@getAccessibleTableRowSelectionC@ 10010284     AccessBridgeJavaEntryPoints.obj
 0002:000012a8       ??_C@_0CK@OKAFABOP@?$CILjavax?1accessibility?1Accessibl@ 100102a8     AccessBridgeJavaEntryPoints.obj
 0002:000012d4       ??_C@_0BN@PCLDBBIG@isAccessibleTableRowSelected@ 100102d4     AccessBridgeJavaEntryPoints.obj
 0002:000012f4       ??_C@_0CK@ILOKEAHN@?$CILjavax?1accessibility?1Accessibl@ 100102f4     AccessBridgeJavaEntryPoints.obj
 0002:00001320       ??_C@_0CA@CNAAIKJJ@getAccessibleTableRowSelections@ 10010320     AccessBridgeJavaEntryPoints.obj
 0002:00001340       ??_C@_0CH@CDNMHGID@getAccessibleTableColumnSelecti@ 10010340     AccessBridgeJavaEntryPoints.obj
 0002:00001368       ??_C@_0CA@NFOBJKJN@isAccessibleTableColumnSelected@ 10010368     AccessBridgeJavaEntryPoints.obj
 0002:00001388       ??_C@_0CD@FNIEANFO@getAccessibleTableColumnSelecti@ 10010388     AccessBridgeJavaEntryPoints.obj
 0002:000013ac       ??_C@_0BG@JNIAKEE@getAccessibleTableRow@ 100103ac     AccessBridgeJavaEntryPoints.obj
 0002:000013c4       ??_C@_0BJ@DEHNOIGE@getAccessibleTableColumn@ 100103c4     AccessBridgeJavaEntryPoints.obj
 0002:000013e0       ??_C@_0BI@MLOHLDGL@getAccessibleTableIndex@ 100103e0     AccessBridgeJavaEntryPoints.obj
 0002:000013f8       ??_C@_0BL@NLFDIBPJ@getAccessibleRelationCount@ 100103f8     AccessBridgeJavaEntryPoints.obj
 0002:00001414       ??_C@_0DN@BLNOMAFI@?$CILjavax?1accessibility?1Accessibl@ 10010414     AccessBridgeJavaEntryPoints.obj
 0002:00001454       ??_C@_0BJ@DOGHLHFJ@getAccessibleRelationKey@ 10010454     AccessBridgeJavaEntryPoints.obj
 0002:00001470       ??_C@_0CM@KJPNEAF@?$CILjavax?1accessibility?1Accessibl@ 10010470     AccessBridgeJavaEntryPoints.obj
 0002:0000149c       ??_C@_0CB@ONJFHOJM@getAccessibleRelationTargetCoun@ 1001049c     AccessBridgeJavaEntryPoints.obj
 0002:000014c0       ??_C@_0FD@OOMEDHDI@?$CILjavax?1accessibility?1Accessibl@ 100104c0     AccessBridgeJavaEntryPoints.obj
 0002:00001514       ??_C@_0BM@MFFGDMCG@getAccessibleRelationTarget@ 10010514     AccessBridgeJavaEntryPoints.obj
 0002:00001530       ??_C@_0FD@IPGDKGIL@?$CILjavax?1accessibility?1Accessibl@ 10010530     AccessBridgeJavaEntryPoints.obj
 0002:00001584       ??_C@_0BH@IPNEFMCF@getAccessibleHypertext@ 10010584     AccessBridgeJavaEntryPoints.obj
 0002:000015a0       ??_C@_0FE@PMDDAMJI@?$CILjavax?1accessibility?1Accessibl@ 100105a0     AccessBridgeJavaEntryPoints.obj
 0002:000015f4       ??_C@_0BM@JMCFFMCN@activateAccessibleHyperlink@ 100105f4     AccessBridgeJavaEntryPoints.obj
 0002:00001610       ??_C@_0BM@IADLHNKN@getAccessibleHyperlinkCount@ 10010610     AccessBridgeJavaEntryPoints.obj
 0002:00001630       ??_C@_0FG@JAOELFOA@?$CILjavax?1accessibility?1Accessibl@ 10010630     AccessBridgeJavaEntryPoints.obj
 0002:00001688       ??_C@_0BH@EAGDOOIC@getAccessibleHyperlink@ 10010688     AccessBridgeJavaEntryPoints.obj
 0002:000016a0       ??_C@_0DO@OBGKICOI@?$CILjavax?1accessibility?1Accessibl@ 100106a0     AccessBridgeJavaEntryPoints.obj
 0002:000016e0       ??_C@_0BL@MPKBBMO@getAccessibleHyperlinkText@ 100106e0     AccessBridgeJavaEntryPoints.obj
 0002:000016fc       ??_C@_0BK@DJNACEGJ@getAccessibleHyperlinkURL@ 100106fc     AccessBridgeJavaEntryPoints.obj
 0002:00001718       ??_C@_0CN@CAHDBMA@?$CILjavax?1accessibility?1Accessibl@ 10010718     AccessBridgeJavaEntryPoints.obj
 0002:00001748       ??_C@_0CB@LKDEDAHI@getAccessibleHyperlinkStartInde@ 10010748     AccessBridgeJavaEntryPoints.obj
 0002:0000176c       ??_C@_0BP@KJGEOOIO@getAccessibleHyperlinkEndIndex@ 1001076c     AccessBridgeJavaEntryPoints.obj
 0002:0000178c       ??_C@_0CO@HPBFOBHC@?$CILjavax?1accessibility?1Accessibl@ 1001078c     AccessBridgeJavaEntryPoints.obj
 0002:000017bc       ??_C@_0CA@FBPINCJA@getAccessibleHypertextLinkIndex@ 100107bc     AccessBridgeJavaEntryPoints.obj
 0002:000017dc       ??_C@_0BO@KGNEMCMH@getAccessibleKeyBindingsCount@ 100107dc     AccessBridgeJavaEntryPoints.obj
 0002:000017fc       ??_C@_0CM@PAHADMIP@?$CILjavax?1accessibility?1Accessibl@ 100107fc     AccessBridgeJavaEntryPoints.obj
 0002:00001828       ??_C@_0BM@HBNEDKIN@getAccessibleKeyBindingChar@ 10010828     AccessBridgeJavaEntryPoints.obj
 0002:00001844       ??_C@_0CB@CIMFEKNG@getAccessibleKeyBindingModifier@ 10010844     AccessBridgeJavaEntryPoints.obj
 0002:00001868       ??_C@_0BI@MJKKDJIF@getAccessibleIconsCount@ 10010868     AccessBridgeJavaEntryPoints.obj
 0002:00001880       ??_C@_0BN@CJEBMOD@getAccessibleIconDescription@ 10010880     AccessBridgeJavaEntryPoints.obj
 0002:000018a0       ??_C@_0BI@MDOGDIAA@getAccessibleIconHeight@ 100108a0     AccessBridgeJavaEntryPoints.obj
 0002:000018b8       ??_C@_0BH@GGKEIMGD@getAccessibleIconWidth@ 100108b8     AccessBridgeJavaEntryPoints.obj
 0002:000018d0       ??_C@_0BK@PKOFGGNC@getAccessibleActionsCount@ 100108d0     AccessBridgeJavaEntryPoints.obj
 0002:000018ec       ??_C@_0BI@DODALGBC@getAccessibleActionName@ 100108ec     AccessBridgeJavaEntryPoints.obj
 0002:00001904       ??_C@_0BE@CCPKEBNJ@doAccessibleActions@ 10010904     AccessBridgeJavaEntryPoints.obj
 0002:00001918       ??_C@_0CC@JCBADKJK@getAccessibleCharCountFromConte@ 10010918     AccessBridgeJavaEntryPoints.obj
 0002:0000193c       ??_C@_0CG@KPDPNIKI@getAccessibleCaretPositionFromC@ 1001093c     AccessBridgeJavaEntryPoints.obj
 0002:00001964       ??_C@_0CN@CCCKKDDE@?$CILjavax?1accessibility?1Accessibl@ 10010964     AccessBridgeJavaEntryPoints.obj
 0002:00001994       ??_C@_0CF@IPJFBKEC@getAccessibleIndexAtPointFromCo@ 10010994     AccessBridgeJavaEntryPoints.obj
 0002:000019bc       ??_C@_0CG@CGEAMPNI@getAccessibleLetterAtIndexFromC@ 100109bc     AccessBridgeJavaEntryPoints.obj
 0002:000019e4       ??_C@_0CE@CLNANFEE@getAccessibleWordAtIndexFromCon@ 100109e4     AccessBridgeJavaEntryPoints.obj
 0002:00001a08       ??_C@_0CI@BJNPGKMI@getAccessibleSentenceAtIndexFro@ 10010a08     AccessBridgeJavaEntryPoints.obj
 0002:00001a30       ??_C@_0CL@HGHPNDH@getAccessibleTextSelectionStart@ 10010a30     AccessBridgeJavaEntryPoints.obj
 0002:00001a5c       ??_C@_0CJ@IPEBCNBB@getAccessibleTextSelectionEndFr@ 10010a5c     AccessBridgeJavaEntryPoints.obj
 0002:00001a88       ??_C@_0CJ@IBCLFAFA@getAccessibleTextSelectedTextFr@ 10010a88     AccessBridgeJavaEntryPoints.obj
 0002:00001ab4       ??_C@_0CK@JLPCFBLN@getAccessibleAttributesAtIndexF@ 10010ab4     AccessBridgeJavaEntryPoints.obj
 0002:00001ae0       ??_C@_0EK@JEPLCIJI@?$CILjavax?1accessibility?1Accessibl@ 10010ae0     AccessBridgeJavaEntryPoints.obj
 0002:00001b2c       ??_C@_0CM@LKNKHCB@getAccessibleAttributeSetAtInde@ 10010b2c     AccessBridgeJavaEntryPoints.obj
 0002:00001b58       ??_C@_0DP@HKEBFOCN@?$CILjavax?1accessibility?1Accessibl@ 10010b58     AccessBridgeJavaEntryPoints.obj
 0002:00001b98       ??_C@_0CI@IIHCGONP@getAccessibleTextRectAtIndexFro@ 10010b98     AccessBridgeJavaEntryPoints.obj
 0002:00001bc0       ??_C@_0CO@OMLKOFDL@getAccessibleXcoordTextRectAtIn@ 10010bc0     AccessBridgeJavaEntryPoints.obj
 0002:00001bf0       ??_C@_0CO@NKEIHFMI@getAccessibleYcoordTextRectAtIn@ 10010bf0     AccessBridgeJavaEntryPoints.obj
 0002:00001c20       ??_C@_0CO@JHFMLGGO@getAccessibleHeightTextRectAtIn@ 10010c20     AccessBridgeJavaEntryPoints.obj
 0002:00001c50       ??_C@_0CN@COKFHFFE@getAccessibleWidthTextRectAtInd@ 10010c50     AccessBridgeJavaEntryPoints.obj
 0002:00001c80       ??_C@_0BC@NPONPPPN@getCaretLocationX@ 10010c80     AccessBridgeJavaEntryPoints.obj
 0002:00001c94       ??_C@_0BC@MGPGMOLM@getCaretLocationY@ 10010c94     AccessBridgeJavaEntryPoints.obj
 0002:00001ca8       ??_C@_0BH@MJJIPGPF@getCaretLocationHeight@ 10010ca8     AccessBridgeJavaEntryPoints.obj
 0002:00001cc0       ??_C@_0BG@BIMEFOON@getCaretLocationWidth@ 10010cc0     AccessBridgeJavaEntryPoints.obj
 0002:00001cd8       ??_C@_0CL@JPPFAPAC@getAccessibleTextLineLeftBounds@ 10010cd8     AccessBridgeJavaEntryPoints.obj
 0002:00001d04       ??_C@_0CM@IBNKHADJ@getAccessibleTextLineRightBound@ 10010d04     AccessBridgeJavaEntryPoints.obj
 0002:00001d30       ??_C@_0DO@MIIPGCPP@?$CILjavax?1accessibility?1Accessibl@ 10010d30     AccessBridgeJavaEntryPoints.obj
 0002:00001d70       ??_C@_0CC@CIBLKPOK@getAccessibleTextRangeFromConte@ 10010d70     AccessBridgeJavaEntryPoints.obj
 0002:00001d94       ??_C@_0CF@CJIJHKPD@getCurrentAccessibleValueFromCo@ 10010d94     AccessBridgeJavaEntryPoints.obj
 0002:00001dbc       ??_C@_0CF@PMHBGBIN@getMaximumAccessibleValueFromCo@ 10010dbc     AccessBridgeJavaEntryPoints.obj
 0002:00001de4       ??_C@_0CF@MEICJJIC@getMinimumAccessibleValueFromCo@ 10010de4     AccessBridgeJavaEntryPoints.obj
 0002:00001e0c       ??_C@_0CM@MHMFNKJL@?$CILjavax?1accessibility?1Accessibl@ 10010e0c     AccessBridgeJavaEntryPoints.obj
 0002:00001e38       ??_C@_0CC@OHDKMAMO@addAccessibleSelectionFromConte@ 10010e38     AccessBridgeJavaEntryPoints.obj
 0002:00001e5c       ??_C@_0CL@HAAKHFKD@?$CILjavax?1accessibility?1Accessibl@ 10010e5c     AccessBridgeJavaEntryPoints.obj
 0002:00001e88       ??_C@_0CE@JAJNKBKJ@clearAccessibleSelectionFromCon@ 10010e88     AccessBridgeJavaEntryPoints.obj
 0002:00001eac       ??_C@_0CH@GOOENNPE@getAccessibleSelectionCountFrom@ 10010eac     AccessBridgeJavaEntryPoints.obj
 0002:00001ed4       ??_C@_0CM@GLHAJFJH@?$CILjavax?1accessibility?1Accessibl@ 10010ed4     AccessBridgeJavaEntryPoints.obj
 0002:00001f00       ??_C@_0CF@PFGNJKHP@isAccessibleChildSelectedFromCo@ 10010f00     AccessBridgeJavaEntryPoints.obj
 0002:00001f28       ??_C@_0CF@LNEMJFKL@removeAccessibleSelectionFromCo@ 10010f28     AccessBridgeJavaEntryPoints.obj
 0002:00001f50       ??_C@_0CI@GIPFHPKO@selectAllAccessibleSelectionFro@ 10010f50     AccessBridgeJavaEntryPoints.obj
 0002:00001f78       ??_C@_04OHLIFDMD@?$CIJ?$CJV@ 10010f78     AccessBridgeJavaEntryPoints.obj
 0002:00001f80       ??_C@_0BJ@MPIBKFAO@addJavaEventNotification@ 10010f80     AccessBridgeJavaEntryPoints.obj
 0002:00001f9c       ??_C@_0BM@FNBBPCEJ@removeJavaEventNotification@ 10010f9c     AccessBridgeJavaEntryPoints.obj
 0002:00001fb8       ??_C@_0CC@MPLKGCBM@addAccessibilityEventNotificati@ 10010fb8     AccessBridgeJavaEntryPoints.obj
 0002:00001fdc       ??_C@_0CF@JFMMDHHJ@removeAccessibilityEventNotific@ 10010fdc     AccessBridgeJavaEntryPoints.obj
 0002:00002004       ??_C@_0CD@PFBLKFGD@?$CILjavax?1swing?1text?1AttributeSet@ 10011004     AccessBridgeJavaEntryPoints.obj
 0002:00002028       ??_C@_0BI@PMOBPKB@getBoldFromAttributeSet@ 10011028     AccessBridgeJavaEntryPoints.obj
 0002:00002040       ??_C@_0BK@HMLEJNMA@getItalicFromAttributeSet@ 10011040     AccessBridgeJavaEntryPoints.obj
 0002:0000205c       ??_C@_0BN@BGEODKID@getUnderlineFromAttributeSet@ 1001105c     AccessBridgeJavaEntryPoints.obj
 0002:0000207c       ??_C@_0CB@BICMGOJK@getStrikethroughFromAttributeSe@ 1001107c     AccessBridgeJavaEntryPoints.obj
 0002:000020a0       ??_C@_0BP@BNLEAGAN@getSuperscriptFromAttributeSet@ 100110a0     AccessBridgeJavaEntryPoints.obj
 0002:000020c0       ??_C@_0BN@FENOLEGG@getSubscriptFromAttributeSet@ 100110c0     AccessBridgeJavaEntryPoints.obj
 0002:000020e0       ??_C@_0DE@PFGGMCPM@?$CILjavax?1swing?1text?1AttributeSet@ 100110e0     AccessBridgeJavaEntryPoints.obj
 0002:00002114       ??_C@_0CD@MGNACFJA@getBackgroundColorFromAttribute@ 10011114     AccessBridgeJavaEntryPoints.obj
 0002:00002138       ??_C@_0CD@JFAEMBOF@getForegroundColorFromAttribute@ 10011138     AccessBridgeJavaEntryPoints.obj
 0002:0000215c       ??_C@_0BO@JFHBDDGD@getFontFamilyFromAttributeSet@ 1001115c     AccessBridgeJavaEntryPoints.obj
 0002:0000217c       ??_C@_0CD@JEPEOEPB@?$CILjavax?1swing?1text?1AttributeSet@ 1001117c     AccessBridgeJavaEntryPoints.obj
 0002:000021a0       ??_C@_0BM@OMIOBJPB@getFontSizeFromAttributeSet@ 100111a0     AccessBridgeJavaEntryPoints.obj
 0002:000021bc       ??_C@_0BN@BAFOGOJK@getAlignmentFromAttributeSet@ 100111bc     AccessBridgeJavaEntryPoints.obj
 0002:000021dc       ??_C@_0BN@DEDFHCOP@getBidiLevelFromAttributeSet@ 100111dc     AccessBridgeJavaEntryPoints.obj
 0002:000021fc       ??_C@_0CD@BDGMPIDO@?$CILjavax?1swing?1text?1AttributeSet@ 100111fc     AccessBridgeJavaEntryPoints.obj
 0002:00002220       ??_C@_0CD@EJOOBJDB@getFirstLineIndentFromAttribute@ 10011220     AccessBridgeJavaEntryPoints.obj
 0002:00002244       ??_C@_0BO@KCBIJLNO@getLeftIndentFromAttributeSet@ 10011244     AccessBridgeJavaEntryPoints.obj
 0002:00002264       ??_C@_0BP@KEIFBKEA@getRightIndentFromAttributeSet@ 10011264     AccessBridgeJavaEntryPoints.obj
 0002:00002284       ??_C@_0BP@ICDNCHPN@getLineSpacingFromAttributeSet@ 10011284     AccessBridgeJavaEntryPoints.obj
 0002:000022a4       ??_C@_0BO@CHPMHCHE@getSpaceAboveFromAttributeSet@ 100112a4     AccessBridgeJavaEntryPoints.obj
 0002:000022c4       ??_C@_0BO@DOLMIFOK@getSpaceBelowFromAttributeSet@ 100112c4     AccessBridgeJavaEntryPoints.obj
 0002:000022e4       ??_C@_0CL@NMLPDKKP@?$CILjavax?1accessibility?1Accessibl@ 100112e4     AccessBridgeJavaEntryPoints.obj
 0002:00002310       ??_C@_0N@CEMKNPGL@requestFocus@ 10011310     AccessBridgeJavaEntryPoints.obj
 0002:00002320       ??_C@_0CN@EDMFOCKG@?$CILjavax?1accessibility?1Accessibl@ 10011320     AccessBridgeJavaEntryPoints.obj
 0002:00002350       ??_C@_0BA@JKPGAJFL@selectTextRange@ 10011350     AccessBridgeJavaEntryPoints.obj
 0002:00002360       ??_C@_0BI@IIOLCPFK@getVisibleChildrenCount@ 10011360     AccessBridgeJavaEntryPoints.obj
 0002:00002378       ??_C@_0BA@JIDLMKH@getVisibleChild@ 10011378     AccessBridgeJavaEntryPoints.obj
 0002:00002388       ??_C@_0BB@ENIAPGBO@setCaretPosition@ 10011388     AccessBridgeJavaEntryPoints.obj
 0002:0000239c       ??_C@_0CE@MELACKPN@getVirtualAccessibleNameFromCon@ 1001139c     AccessBridgeJavaEntryPoints.obj
 0002:000023c0       ??_C@_0DP@ODHDIMGL@?$FLINFO?$FN?3?5Calling?5AccessBridgeJav@ 100113c0     AccessBridgeJavaEntryPoints.obj
 0002:00002400       ??_C@_0DD@INJPOCHE@Getting?5isJavaWindow?5?9?5call?5to?5@ 10011400     AccessBridgeJavaEntryPoints.obj
 0002:00002434       ??_C@_0DN@ENCLOLFG@?$FLERROR?$FN?3?5?$CK?$CK?$CK?5Exception?5occured?5@ 10011434     AccessBridgeJavaEntryPoints.obj
 0002:00002474       ??_C@_0DH@DHJJKMLN@?$FLERROR?$FN?3?5either?5jniEnv?5?$DN?$DN?50?5or?5@ 10011474     AccessBridgeJavaEntryPoints.obj
 0002:000024ac       ??_C@_0DN@GKGIBPBO@?$FLINFO?$FN?3?5In?5AccessBridgeJavaEntr@ 100114ac     AccessBridgeJavaEntryPoints.obj
 0002:000024ec       ??_C@_0BF@LOIOEBHF@Calling?5IsSameObject@ 100114ec     AccessBridgeJavaEntryPoints.obj
 0002:00002504       ??_C@_0CE@PJOLBDKG@?$FLINFO?$FN?3?5?5?5isSameObject?5returnin@ 10011504     AccessBridgeJavaEntryPoints.obj
 0002:00002528       ??_C@_0EK@MPPKLDGH@?$FLINFO?$FN?3?5In?5AccessBridgeJavaEntr@ 10011528     AccessBridgeJavaEntryPoints.obj
 0002:00002574       ??_C@_0DP@INBKCEII@Getting?5AccessibleContextFromHW@ 10011574     AccessBridgeJavaEntryPoints.obj
 0002:000025b8       ??_C@_0EI@POHJNOIF@?$FLERROR?$FN?3?5?5either?5jniEnv?5?$DN?$DN?50?5or@ 100115b8     AccessBridgeJavaEntryPoints.obj
 0002:00002600       ??_C@_0EK@KGPHBKLN@?$FLINFO?$FN?3?5In?5AccessBridgeJavaEntr@ 10011600     AccessBridgeJavaEntryPoints.obj
 0002:0000264c       ??_C@_0DM@OPKABADC@Getting?5HWNDFromAccessibleConte@ 1001164c     AccessBridgeJavaEntryPoints.obj
 0002:00002688       ??_C@_0BD@NKFEMHLM@?$FLINFO?$FN?3?5rHWND?5?$DN?5?$CFX@ 10011688     AccessBridgeJavaEntryPoints.obj
 0002:000026a0       ??_C@_0EH@MFPOIGJN@?$FLERROR?$FN?3?5either?5jniEnv?5?$DN?$DN?50?5or?5@ 100116a0     AccessBridgeJavaEntryPoints.obj
 0002:000026e8       ??_C@_0EC@BPPANMDJ@?$FLINFO?$FN?3?5In?5AccessBridgeJavaEntr@ 100116e8     AccessBridgeJavaEntryPoints.obj
 0002:0000272c       ??_C@_0BN@LGGMDMGD@?$FLERROR?$FN?3?5?5?5?5NewString?5failed@ 1001172c     AccessBridgeJavaEntryPoints.obj
 0002:0000274c       ??_C@_0CO@NCDGKPGB@setTextContents?5?9?5call?5to?5CallB@ 1001174c     AccessBridgeJavaEntryPoints.obj
 0002:0000277c       ??_C@_0BI@IMHMFAIB@?$FLINFO?$FN?3?5?5?5?5?5result?5?$DN?5?$CFd@ 1001177c     AccessBridgeJavaEntryPoints.obj
 0002:00002794       ??_C@_0DK@MGDAPF@?$FLERROR?$FN?3?5either?5jniEnv?5?$DN?$DN?50?5or?5@ 10011794     AccessBridgeJavaEntryPoints.obj
 0002:000027d0       ??_C@_0DP@LHNNHOD@?$FLINFO?$FN?3?5In?5AccessBridgeJavaEntr@ 100117d0     AccessBridgeJavaEntryPoints.obj
 0002:00002810       ??_C@_0BO@LLFKIHLA@?$FLERROR?$FN?3?5?5?5?5?5NewString?5failed@ 10011810     AccessBridgeJavaEntryPoints.obj
 0002:00002830       ??_C@_0DE@KBFMBJPI@Getting?5ParentWithRole?5?9?5call?5t@ 10011830     AccessBridgeJavaEntryPoints.obj
 0002:00002864       ??_C@_0CE@LNEDINGM@?$FLINFO?$FN?3?5?5?5?5?5rAccessibleContext?5@ 10011864     AccessBridgeJavaEntryPoints.obj
 0002:00002888       ??_C@_0DA@OMNPGENP@Getting?5ParentWithRole?5?9?5call?5t@ 10011888     AccessBridgeJavaEntryPoints.obj
 0002:000028b8       ??_C@_0EF@LHAMKGPK@?$FLINFO?$FN?3?5?5?5Returning?5?9?5returnedA@ 100118b8     AccessBridgeJavaEntryPoints.obj
 0002:00002900       ??_C@_0DM@OLEIFDLG@?$FLERROR?$FN?3?5either?5jniEnv?5?$DN?$DN?50?5or?5@ 10011900     AccessBridgeJavaEntryPoints.obj
 0002:0000293c       ??_C@_0DP@EPHBFJKE@?$FLINFO?$FN?3?5In?5AccessBridgeJavaEntr@ 1001193c     AccessBridgeJavaEntryPoints.obj
 0002:0000297c       ??_C@_0DE@FDIFCLEM@Getting?5TopLevelObject?5?9?5call?5t@ 1001197c     AccessBridgeJavaEntryPoints.obj
 0002:000029b0       ??_C@_0CB@GDMCCFCK@?$FLINFO?$FN?3?5?5rAccessibleContext?5?$DN?5?$CF@ 100119b0     AccessBridgeJavaEntryPoints.obj
 0002:000029d4       ??_C@_0DA@ELIJHKN@Getting?5TopLevelObject?5?9?5call?5t@ 100119d4     AccessBridgeJavaEntryPoints.obj
 0002:00002a04       ??_C@_0DM@MKIGPNDF@?$FLERROR?$FN?3?5either?5jniEnv?5?$DN?$DN?50?5or?5@ 10011a04     AccessBridgeJavaEntryPoints.obj
 0002:00002a40       ??_C@_0EH@MCHGGFNF@?$FLINFO?$FN?3?5In?5AccessBridgeJavaEntr@ 10011a40     AccessBridgeJavaEntryPoints.obj
 0002:00002a88       ??_C@_0DM@IKNMPPHI@Getting?5ParentWithRoleElseRoot?5@ 10011a88     AccessBridgeJavaEntryPoints.obj
 0002:00002ac4       ??_C@_0DI@CDJCPAOF@Getting?5ParentWithRoleElseRoot?5@ 10011ac4     AccessBridgeJavaEntryPoints.obj
 0002:00002b00       ??_C@_0EF@MODADMKL@?$FLERROR?$FN?3?5?5either?5jniEnv?5?$DN?$DN?50?5or@ 10011b00     AccessBridgeJavaEntryPoints.obj
 0002:00002b48       ??_C@_0DM@EBONPKNN@?$FLINFO?$FN?3?5In?5AccessBridgeJavaEntr@ 10011b48     AccessBridgeJavaEntryPoints.obj
 0002:00002b84       ??_C@_0CO@CCBFEFG@Getting?5ObjectDepth?5?9?5call?5to?5C@ 10011b84     AccessBridgeJavaEntryPoints.obj
 0002:00002bb4       ??_C@_0BJ@KJFHIGKC@?$FLINFO?$FN?3?5?5?5?5?5rResult?5?$DN?5?$CFd@ 10011bb4     AccessBridgeJavaEntryPoints.obj
 0002:00002bd0       ??_C@_0DJ@NCMDONA@?$FLERROR?$FN?3?5either?5jniEnv?5?$DN?$DN?50?5or?5@ 10011bd0     AccessBridgeJavaEntryPoints.obj
 0002:00002c10       ??_C@_0EB@OJAHMNKI@?$FLINFO?$FN?3?5In?5AccessBridgeJavaEntr@ 10011c10     AccessBridgeJavaEntryPoints.obj
 0002:00002c54       ??_C@_0DG@FKCKDOAD@Getting?5ActiveDescendent?5?9?5call@ 10011c54     AccessBridgeJavaEntryPoints.obj
 0002:00002c8c       ??_C@_0DC@DOJHNKHC@Getting?5ActiveDescendant?5?9?5call@ 10011c8c     AccessBridgeJavaEntryPoints.obj
 0002:00002cc0       ??_C@_0DO@FBKMCPK@?$FLERROR?$FN?3?5either?5jniEnv?5?$DN?$DN?50?5or?5@ 10011cc0     AccessBridgeJavaEntryPoints.obj
 0002:00002d00       ??_C@_0CK@IFAHAOG@?$FLINFO?$FN?3?5?5getVirtualAccessibleNa@ 10011d00     AccessBridgeJavaEntryPoints.obj
 0002:00002d2c       ??_C@_0DE@GLGPLDPG@Getting?5AccessibleName?5?9?5call?5t@ 10011d2c     AccessBridgeJavaEntryPoints.obj
 0002:00002d60       ??_C@_0DC@LMABNHGH@Getting?5AccessibleName?5?9?5call?5t@ 10011d60     AccessBridgeJavaEntryPoints.obj
 0002:00002d94       ??_C@_0DD@FODFLNBM@Getting?5AccessibleName?5?9?5call?5t@ 10011d94     AccessBridgeJavaEntryPoints.obj
 0002:00002dc8       ??_C@_0DG@LKNGBJAO@Getting?5AccessibleName?5?9?5call?5t@ 10011dc8     AccessBridgeJavaEntryPoints.obj
 0002:00002e00       ??_C@_0DC@MBCPGFEL@Getting?5AccessibleName?5?9?5call?5t@ 10011e00     AccessBridgeJavaEntryPoints.obj
 0002:00002e34       ??_C@_1DA@BACBNKJB@?$AA?5?$AA?5?$AAA?$AAc?$AAc?$AAe?$AAs?$AAs?$AAi?$AAb?$AAl?$AAe?$AA?5?$AAN?$AAa@ 10011e34     AccessBridgeJavaEntryPoints.obj
 0002:00002e64       ??_C@_0DC@HCPEBFPJ@Getting?5AccessibleName?5?9?5call?5t@ 10011e64     AccessBridgeJavaEntryPoints.obj
 0002:00002e98       ??_C@_0CD@JNOMKFNM@?$FLINFO?$FN?3?5?5?5Accessible?5Name?5is?5nu@ 10011e98     AccessBridgeJavaEntryPoints.obj
 0002:00002ec0       ??_C@_0EN@LBGKPBFG@?$FLINFO?$FN?3?5either?5jniEnv?5?$DN?$DN?50?5or?5g@ 10011ec0     AccessBridgeJavaEntryPoints.obj
 0002:00002f10       ??_C@_0DK@COLMCNJL@?$FLINFO?$FN?3?5In?5AccessBridgeJavaEntr@ 10011f10     AccessBridgeJavaEntryPoints.obj
 0002:00002f4c       ??_C@_0CL@OHFNFEAE@requestFocus?5?9?5call?5to?5CallBool@ 10011f4c     AccessBridgeJavaEntryPoints.obj
 0002:00002f78       ??_C@_0BH@JOKEJIHH@?$FLINFO?$FN?3?5?5?5?5result?5?$DN?5?$CFd@ 10011f78     AccessBridgeJavaEntryPoints.obj
 0002:00002f90       ??_C@_0DH@OADKFKDG@?$FLERROR?$FN?3?5either?5jniEnv?5?$DN?$DN?50?5or?5@ 10011f90     AccessBridgeJavaEntryPoints.obj
 0002:00002fc8       ??_C@_0FB@HEEEBDKB@?$FLINFO?$FN?3?5In?5AccessBridgeJavaEntr@ 10011fc8     AccessBridgeJavaEntryPoints.obj
 0002:0000301c       ??_C@_0CO@NOPLEGNC@selectTextRange?5?9?5call?5to?5CallB@ 1001201c     AccessBridgeJavaEntryPoints.obj
 0002:0000304c       ??_C@_0DK@EDLAMPCD@?$FLERROR?$FN?3?5either?5jniEnv?5?$DN?$DN?50?5or?5@ 1001204c     AccessBridgeJavaEntryPoints.obj
 0002:00003088       ??_C@_0FK@CBBPCLFD@?$FLINFO?$FN?3?5In?5AccessBridgeJavaEntr@ 10012088     AccessBridgeJavaEntryPoints.obj
 0002:000030e4       ??_C@_0DN@CIOOGMLK@?$FLINFO?$FN?3?5?5Getting?5full?5test_attr@ 100120e4     AccessBridgeJavaEntryPoints.obj
 0002:00003128       ??_C@_0EB@FNOCJLAN@Getting?5AccessibleAttributesAtI@ 10012128     AccessBridgeJavaEntryPoints.obj
 0002:0000316c       ??_C@_0DE@NPIJKEOK@?$FLINFO?$FN?3?5?5?5returned?5from?5CallObj@ 1001216c     AccessBridgeJavaEntryPoints.obj
 0002:000031a0       ??_C@_0DP@GAODIEPK@Getting?5AccessibleAttributesAtI@ 100121a0     AccessBridgeJavaEntryPoints.obj
 0002:000031e0       ??_C@_0EA@NAFHLALG@Getting?5AccessibleAttributesAtI@ 100121e0     AccessBridgeJavaEntryPoints.obj
 0002:00003220       ??_C@_0ED@HICLLPAP@Getting?5AccessibleAttributesAtI@ 10012220     AccessBridgeJavaEntryPoints.obj
 0002:00003264       ??_C@_0DP@BNMNDGNG@Getting?5AccessibleAttributesAtI@ 10012264     AccessBridgeJavaEntryPoints.obj
 0002:000032a8       ??_C@_1FE@NAFGNNMA@?$AA?$FL?$AAI?$AAN?$AAF?$AAO?$AA?$FN?$AA?3?$AA?5?$AA?5?$AAA?$AAc?$AAc?$AAe?$AAs?$AAs@ 100122a8     AccessBridgeJavaEntryPoints.obj
 0002:000032fc       ??_C@_0DP@KOBGEGGE@Getting?5AccessibleAttributesAtI@ 100122fc     AccessBridgeJavaEntryPoints.obj
 0002:0000333c       ??_C@_0CO@GBFCDBDB@?$FLWARN?$FN?3?5?5?5Accessible?5Text?5attri@ 1001233c     AccessBridgeJavaEntryPoints.obj
 0002:00003370       ??_C@_0FB@DKHOICMI@?$FLERROR?$FN?3?5either?5env?5?$DN?$DN?50?5or?5get@ 10012370     AccessBridgeJavaEntryPoints.obj
 0002:000033c8       ??_C@_0EH@KKFBHMJC@?$FLINFO?$FN?3?5?$CD?$CD?$CD?$CD?$CD?5AccessBridgeJavaE@ 100123c8     AccessBridgeJavaEntryPoints.obj
 0002:00003410       ??_C@_0DP@MHLDKAGF@?$CD?$CD?$CD?$CD?$CD?5Getting?5visible?5children?5@ 10012410     AccessBridgeJavaEntryPoints.obj
 0002:00003450       ??_C@_0CM@JAPBNGLO@?$FLINFO?$FN?3?5?5?5?$CD?$CD?$CD?$CD?$CD?5visible?5childre@ 10012450     AccessBridgeJavaEntryPoints.obj
 0002:00003480       ??_C@_0FD@GLIPOPHN@?$FLINFO?$FN?3?5?$CD?$CD?$CD?$CD?$CD?5AccessBridgeJavaE@ 10012480     AccessBridgeJavaEntryPoints.obj
 0002:000034d4       ??_C@_0CH@ONKDDCMN@?$FLINFO?$FN?3?5?5?5getting?5visible?5child@ 100124d4     AccessBridgeJavaEntryPoints.obj
 0002:000034fc       ??_C@_0DJ@HGPLCHEB@?$CD?$CD?$CD?$CD?$CD?5getVisibleChildMethod?5?9?5c@ 100124fc     AccessBridgeJavaEntryPoints.obj
 0002:00003538       ??_C@_0DF@JHJIJJH@?$CD?$CD?$CD?$CD?$CD?5getVisibleChildMethod?5?9?5c@ 10012538     AccessBridgeJavaEntryPoints.obj
 0002:00003570       ??_C@_0CD@ECMHOCH@?$FLINFO?$FN?3?5?5?5?$CD?$CD?$CD?$CD?$CD?5visible?5child?5?$DN@ 10012570     AccessBridgeJavaEntryPoints.obj
 0002:00003598       ??_C@_0EK@GNPPBBMN@?$FLINFO?$FN?3?5?5?5?$CD?$CD?$CD?$CD?$CD?5AccessBridgeJav@ 10012598     AccessBridgeJavaEntryPoints.obj
 0002:000035e8       ??_C@_0EL@OPKFGOFA@?$FLINFO?$FN?3?5In?5AccessBridgeJavaEntr@ 100125e8     AccessBridgeJavaEntryPoints.obj
 0002:00003634       ??_C@_0CO@BDNAFHGG@setCaretPostion?5?9?5call?5to?5CallB@ 10012634     AccessBridgeJavaEntryPoints.obj
 0002:00003664       ??_C@_0BJ@PGHBDIPI@?$FLERROR?$FN?3?5?5?5?5?5result?5?$DN?5?$CFd@ 10012664     AccessBridgeJavaEntryPoints.obj
 0002:00003680       ??_C@_0DL@CBEPMOL@?$FLERROR?$FN?3?5either?5jniEnv?5?$DN?$DN?50?5or?5@ 10012680     AccessBridgeJavaEntryPoints.obj
 0002:000036bc       ??_C@_0DP@DPLDEGDE@?$FLINFO?$FN?3?5Calling?5AccessBridgeJav@ 100126bc     AccessBridgeJavaEntryPoints.obj
 0002:000036fc       ??_C@_0DJ@EBEOKJAG@Getting?5JavaVersionProperty?5?9?5c@ 100126fc     AccessBridgeJavaEntryPoints.obj
 0002:00003738       ??_C@_0FC@KFJABCDE@?$FLERROR?$FN?3?5?5?$CK?$CK?$CK?5Exception?5when?5ge@ 10012738     AccessBridgeJavaEntryPoints.obj
 0002:0000378c       ??_C@_0DL@FDAICLOI@Getting?5JavaVersionProperty?5?9?5c@ 1001278c     AccessBridgeJavaEntryPoints.obj
 0002:000037c8       ??_C@_0DH@PEMIMKKJ@Getting?5JavaVersionProperty?5?9?5c@ 100127c8     AccessBridgeJavaEntryPoints.obj
 0002:00003800       ??_C@_1CK@PFPDBLJ@?$AA?5?$AA?5?$AAJ?$AAa?$AAv?$AAa?$AA?5?$AAv?$AAe?$AAr?$AAs?$AAi?$AAo?$AAn?$AA?5@ 10012800     AccessBridgeJavaEntryPoints.obj
 0002:0000382c       ??_C@_0DH@EHBDLKBL@Getting?5JavaVersionProperty?5?9?5c@ 1001282c     AccessBridgeJavaEntryPoints.obj
 0002:00003864       ??_C@_0CA@KOJKOLB@?$FLWARN?$FN?3?5?5?5Java?5version?5is?5null?4@ 10012864     AccessBridgeJavaEntryPoints.obj
 0002:00003884       ??_C@_0DP@FHBJPJDO@?$FLERROR?$FN?3?5?5either?5env?5?$DN?$DN?50?5or?5ge@ 10012884     AccessBridgeJavaEntryPoints.obj
 0002:000038c8       ??_C@_0EC@OAJCCJEK@?$FLINFO?$FN?3?5Calling?5AccessBridgeJav@ 100128c8     AccessBridgeJavaEntryPoints.obj
 0002:0000390c       ??_C@_0BF@MJCCCBHB@?$FLERROR?$FN?3?5?5No?5Java?5VM@ 1001290c     AccessBridgeJavaEntryPoints.obj
 0002:00003924       ??_C@_0BH@PCLEJECO@?$FLERROR?$FN?3?5?5Null?5jobject@ 10012924     AccessBridgeJavaEntryPoints.obj
 0002:0000393c       ??_C@_0DE@FOOENAKM@Getting?5AccessibleText?5?9?5call?5t@ 1001293c     AccessBridgeJavaEntryPoints.obj
 0002:00003970       ??_C@_0BP@NHKMDDHI@?$FLERROR?$FN?3?5?5?5AccessibleText?5?$DN?5?$CFp@ 10012970     AccessBridgeJavaEntryPoints.obj
 0002:00003990       ??_C@_0DC@NHCDOGBO@Getting?5AccessibleText?5?9?5call?5t@ 10012990     AccessBridgeJavaEntryPoints.obj
 0002:000039c8       ??_C@_0EF@KPMHECBJ@?$FLERROR?$FN?3?5?5either?5env?5?$DN?$DN?50?5or?5ge@ 100129c8     AccessBridgeJavaEntryPoints.obj
 0002:00003a10       ??_C@_0CL@OMBEMJIM@?$FLERROR?$FN?3?5?5jobject?5is?5not?5an?5Acc@ 10012a10     AccessBridgeJavaEntryPoints.obj
 0002:00003a40       ??_C@_0FB@IMPDGAOD@?$FLINFO?$FN?3?5Calling?5AccessBridgeJav@ 10012a40     AccessBridgeJavaEntryPoints.obj
 0002:00003a94       ??_C@_0DJ@CBKJGOIB@Getting?5AccessibleContextAt?5?9?5c@ 10012a94     AccessBridgeJavaEntryPoints.obj
 0002:00003ad0       ??_C@_0DF@PJCJKGPI@Getting?5AccessibleContextAt?5?9?5c@ 10012ad0     AccessBridgeJavaEntryPoints.obj
 0002:00003b08       ??_C@_0DP@LFOACNJN@?$FLERROR?$FN?3?5?5either?5env?5?$DN?$DN?50?5or?5ge@ 10012b08     AccessBridgeJavaEntryPoints.obj
 0002:00003b48       ??_C@_0EN@LHFHLFOC@?$FLINFO?$FN?3?5Calling?5AccessBridgeJav@ 10012b48     AccessBridgeJavaEntryPoints.obj
 0002:00003b98       ??_C@_0EA@NLINILPH@Getting?5AccessibleContextWithFo@ 10012b98     AccessBridgeJavaEntryPoints.obj
 0002:00003bd8       ??_C@_0DM@IJDJLPBO@Getting?5AccessibleContextWithFo@ 10012bd8     AccessBridgeJavaEntryPoints.obj
 0002:00003c18       ??_C@_0EJ@KBIILIHA@?$FLERROR?$FN?3?5?5either?5jniEnv?5?$DN?$DN?50?5or@ 10012c18     AccessBridgeJavaEntryPoints.obj
 0002:00003c68       ??_C@_0FB@NNGDGCK@?$FLINFO?$FN?3?5?$CD?$CD?$CD?$CD?$CD?5Calling?5AccessBri@ 10012c68     AccessBridgeJavaEntryPoints.obj
 0002:00003cbc       ??_C@_0DF@BABIDEMG@?$FLWARN?$FN?3?5?5passed?5in?5AccessibleCo@ 10012cbc     AccessBridgeJavaEntryPoints.obj
 0002:00003cf8       ??_C@_1EA@IPHAHEJA@?$AA?$FL?$AAI?$AAN?$AAF?$AAO?$AA?$FN?$AA?3?$AA?5?$AA?5?$AA?5?$AAA?$AAc?$AAc?$AAe?$AAs@ 10012cf8     AccessBridgeJavaEntryPoints.obj
 0002:00003d38       ??_C@_0CD@BCDIDKCI@?$FLWARN?$FN?3?5?5?5Accessible?5Name?5is?5nu@ 10012d38     AccessBridgeJavaEntryPoints.obj
 0002:00003d60       ??_C@_0EF@DMNCHIBL@?$FLERROR?$FN?3?5?5either?5env?5?$DN?$DN?50?5or?5ge@ 10012d60     AccessBridgeJavaEntryPoints.obj
 0002:00003da8       ??_C@_0DL@IPNAGHCP@Getting?5AccessibleDescription?5?9@ 10012da8     AccessBridgeJavaEntryPoints.obj
 0002:00003de8       ??_C@_1EO@NBFBPIFN@?$AA?$FL?$AAI?$AAN?$AAF?$AAO?$AA?$FN?$AA?3?$AA?5?$AA?5?$AA?5?$AAA?$AAc?$AAc?$AAe?$AAs@ 10012de8     AccessBridgeJavaEntryPoints.obj
 0002:00003e38       ??_C@_0CK@KNEKOBNE@?$FLWARN?$FN?3?5?5?5Accessible?5Descriptio@ 10012e38     AccessBridgeJavaEntryPoints.obj
 0002:00003e68       ??_C@_0EM@LPILGNDD@?$FLERROR?$FN?3?5?5either?5env?5?$DN?$DN?50?5or?5ge@ 10012e68     AccessBridgeJavaEntryPoints.obj
 0002:00003eb4       ??_C@_0DE@IKDIHCF@Getting?5AccessibleRole?5?9?5call?5t@ 10012eb4     AccessBridgeJavaEntryPoints.obj
 0002:00003ee8       ??_C@_0DC@FOMJEAJG@Getting?5AccessibleRole?5?9?5call?5t@ 10012ee8     AccessBridgeJavaEntryPoints.obj
 0002:00003f1c       ??_C@_0DD@JEGNLHAB@Getting?5AccessibleRole?5?9?5call?5t@ 10012f1c     AccessBridgeJavaEntryPoints.obj
 0002:00003f50       ??_C@_0DG@DBHHBIKL@Getting?5AccessibleRole?5?9?5call?5t@ 10012f50     AccessBridgeJavaEntryPoints.obj
 0002:00003f88       ??_C@_0DC@CDOHPCLK@Getting?5AccessibleRole?5?9?5call?5t@ 10012f88     AccessBridgeJavaEntryPoints.obj
 0002:00003fc0       ??_C@_1EA@DFMPHGFH@?$AA?$FL?$AAI?$AAN?$AAF?$AAO?$AA?$FN?$AA?3?$AA?5?$AA?5?$AA?5?$AAA?$AAc?$AAc?$AAe?$AAs@ 10012fc0     AccessBridgeJavaEntryPoints.obj
 0002:00004000       ??_C@_0DC@JADMICAI@Getting?5AccessibleRole?5?9?5call?5t@ 10013000     AccessBridgeJavaEntryPoints.obj
 0002:00004034       ??_C@_0CD@DPDMNHLG@?$FLWARN?$FN?3?5?5?5Accessible?5Role?5is?5nu@ 10013034     AccessBridgeJavaEntryPoints.obj
 0002:00004058       ??_C@_0EL@ENOHPPLP@?$FLERROR?$FN?3?5?5either?5env?5?$DN?$DN?50?5or?5ge@ 10013058     AccessBridgeJavaEntryPoints.obj
 0002:000040a4       ??_C@_0DK@OPAANMJH@Getting?5AccessibleRole_en_US?5?9?5@ 100130a4     AccessBridgeJavaEntryPoints.obj
 0002:000040e0       ??_C@_0DI@CJNJDFMD@Getting?5AccessibleRole_en_US?5?9?5@ 100130e0     AccessBridgeJavaEntryPoints.obj
 0002:00004118       ??_C@_0DJ@IPBLACAP@Getting?5AccessibleRole_en_US?5?9?5@ 10013118     AccessBridgeJavaEntryPoints.obj
 0002:00004154       ??_C@_0DM@BLDNLLEO@Getting?5AccessibleRole_en_US?5?9?5@ 10013154     AccessBridgeJavaEntryPoints.obj
 0002:00004190       ??_C@_0DI@FEPHIHOP@Getting?5AccessibleRole_en_US?5?9?5@ 10013190     AccessBridgeJavaEntryPoints.obj
 0002:000041c8       ??_C@_1EM@ICLLIBMO@?$AA?$FL?$AAI?$AAN?$AAF?$AAO?$AA?$FN?$AA?3?$AA?5?$AA?5?$AA?5?$AAA?$AAc?$AAc?$AAe?$AAs@ 100131c8     AccessBridgeJavaEntryPoints.obj
 0002:00004214       ??_C@_0DI@OHCMPHFN@Getting?5AccessibleRole_en_US?5?9?5@ 10013214     AccessBridgeJavaEntryPoints.obj
 0002:0000424c       ??_C@_0CJ@JHFOCCMF@?$FLWARN?$FN?3?5?5?5Accessible?5Role?5en_US@ 1001324c     AccessBridgeJavaEntryPoints.obj
 0002:00004278       ??_C@_0FA@EDCBAJIO@?$FLERROR?$FN?3?5either?5env?5?$DN?$DN?50?5or?5get@ 10013278     AccessBridgeJavaEntryPoints.obj
 0002:000042c8       ??_C@_0DF@HNCNCNCA@Getting?5AccessibleState?5?9?5call?5@ 100132c8     AccessBridgeJavaEntryPoints.obj
 0002:00004300       ??_C@_0DD@FJJPIJBK@Getting?5AccessibleState?5?9?5call?5@ 10013300     AccessBridgeJavaEntryPoints.obj
 0002:00004334       ??_C@_0DE@HAGECOMD@Getting?5AccessibleState?5?9?5call?5@ 10013334     AccessBridgeJavaEntryPoints.obj
 0002:00004368       ??_C@_0DH@HKADNDJG@Getting?5AccessibleState?5?9?5call?5@ 10013368     AccessBridgeJavaEntryPoints.obj
 0002:000043a0       ??_C@_0DD@CELBDLDG@Getting?5AccessibleState?5?9?5call?5@ 100133a0     AccessBridgeJavaEntryPoints.obj
 0002:000043d8       ??_C@_1EE@DCJFHGCM@?$AA?$FL?$AAI?$AAN?$AAF?$AAO?$AA?$FN?$AA?3?$AA?5?$AA?5?$AA?5?$AAA?$AAc?$AAc?$AAe?$AAs@ 100133d8     AccessBridgeJavaEntryPoints.obj
 0002:0000441c       ??_C@_0DD@JHGKELIE@Getting?5AccessibleState?5?9?5call?5@ 1001341c     AccessBridgeJavaEntryPoints.obj
 0002:00004450       ??_C@_0CF@EJIKBPCF@?$FLWARN?$FN?3?5?5?5Accessible?5States?5is?5@ 10013450     AccessBridgeJavaEntryPoints.obj
 0002:00004478       ??_C@_0EN@PLJCLDAI@?$FLERROR?$FN?3?5?5either?5env?5?$DN?$DN?50?5or?5ge@ 10013478     AccessBridgeJavaEntryPoints.obj
 0002:000044c8       ??_C@_0DL@NKOGKBKA@Getting?5AccessibleState_en_US?5?9@ 100134c8     AccessBridgeJavaEntryPoints.obj
 0002:00004504       ??_C@_0DJ@EPIHCNDB@Getting?5AccessibleState_en_US?5?9@ 10013504     AccessBridgeJavaEntryPoints.obj
 0002:00004540       ??_C@_0DK@NMMOMPCH@Getting?5AccessibleState_en_US?5?9@ 10013540     AccessBridgeJavaEntryPoints.obj
 0002:0000457c       ??_C@_0DN@KFIOCDBN@Getting?5AccessibleState_en_US?5?9@ 1001357c     AccessBridgeJavaEntryPoints.obj
 0002:000045bc       ??_C@_0DJ@DCKJJPBN@Getting?5AccessibleState_en_US?5?9@ 100135bc     AccessBridgeJavaEntryPoints.obj
 0002:000045f8       ??_C@_1FA@BNDENPHM@?$AA?$FL?$AAI?$AAN?$AAF?$AAO?$AA?$FN?$AA?3?$AA?5?$AA?5?$AA?5?$AAA?$AAc?$AAc?$AAe?$AAs@ 100135f8     AccessBridgeJavaEntryPoints.obj
 0002:00004648       ??_C@_0DJ@IBHCOPKP@Getting?5AccessibleState_en_US?5?9@ 10013648     AccessBridgeJavaEntryPoints.obj
 0002:00004684       ??_C@_0CL@LNKMOAJG@?$FLWARN?$FN?3?5?5?5Accessible?5States?5en_@ 10013684     AccessBridgeJavaEntryPoints.obj
 0002:000046b0       ??_C@_0FC@KNGBOCJI@?$FLERROR?$FN?3?5either?5env?5?$DN?$DN?50?5or?5get@ 100136b0     AccessBridgeJavaEntryPoints.obj
 0002:00004704       ??_C@_0DK@NAACLIEE@Getting?5AccessibleIndexInParent@ 10013704     AccessBridgeJavaEntryPoints.obj
 0002:00004740       ??_C@_0BP@LDKDBFNM@?$FLINFO?$FN?3?5?5?5Index?5in?5Parent?5?$DN?5?$CFd@ 10013740     AccessBridgeJavaEntryPoints.obj
 0002:00004760       ??_C@_0EO@FMBHNIPI@?$FLERROR?$FN?3?5?5either?5env?5?$DN?$DN?50?5or?5ge@ 10013760     AccessBridgeJavaEntryPoints.obj
 0002:000047b0       ??_C@_0EK@BLALEJAL@?$FLINFO?$FN?3?5?$CK?$CK?$CK?5jniEnv?3?5?$CFp?$DL?5accessB@ 100137b0     AccessBridgeJavaEntryPoints.obj
 0002:000047fc       ??_C@_0DK@HBEJENLO@Getting?5AccessibleChildrenCount@ 100137fc     AccessBridgeJavaEntryPoints.obj
 0002:00004838       ??_C@_0BO@INNKBLPE@?$FLINFO?$FN?3?5?5?5Children?5count?5?$DN?5?$CFd@ 10013838     AccessBridgeJavaEntryPoints.obj
 0002:00004858       ??_C@_0EO@BPNCCJLD@?$FLERROR?$FN?3?5?5either?5env?5?$DN?$DN?50?5or?5ge@ 10013858     AccessBridgeJavaEntryPoints.obj
 0002:000048a8       ??_C@_0EK@PAPEMOFA@?$FLINFO?$FN?3?5?$CK?$CK?$CK?5jniEnv?3?5?$CFp?$DL?5accessB@ 100138a8     AccessBridgeJavaEntryPoints.obj
 0002:000048f4       ??_C@_0DD@EIHALEFK@Getting?5AccessibleXcoord?5?9?5call@ 100138f4     AccessBridgeJavaEntryPoints.obj
 0002:00004928       ??_C@_0BH@EMDFCPBA@?$FLINFO?$FN?3?5?5?5X?5coord?5?$DN?5?$CFd@ 10013928     AccessBridgeJavaEntryPoints.obj
 0002:00004940       ??_C@_0EH@EAAFBPMN@?$FLERROR?$FN?3?5?5either?5env?5?$DN?$DN?50?5or?5ge@ 10013940     AccessBridgeJavaEntryPoints.obj
 0002:00004988       ??_C@_0EK@PIPPCCAB@?$FLINFO?$FN?3?5?$CK?$CK?$CK?5jniEnv?3?5?$CFX?$DL?5accessB@ 10013988     AccessBridgeJavaEntryPoints.obj
 0002:000049d4       ??_C@_0DD@HOICCEKJ@Getting?5AccessibleYcoord?5?9?5call@ 100139d4     AccessBridgeJavaEntryPoints.obj
 0002:00004a08       ??_C@_0BH@JBKDPGJF@?$FLINFO?$FN?3?5?5?5Y?5coord?5?$DN?5?$CFd@ 10013a08     AccessBridgeJavaEntryPoints.obj
 0002:00004a20       ??_C@_0EH@CDACMGOJ@?$FLERROR?$FN?3?5?5either?5env?5?$DN?$DN?50?5or?5ge@ 10013a20     AccessBridgeJavaEntryPoints.obj
 0002:00004a68       ??_C@_0DC@IECDLNHB@Getting?5AccessibleWidth?5?9?5call?5@ 10013a68     AccessBridgeJavaEntryPoints.obj
 0002:00004a9c       ??_C@_0BF@EEAFCLIB@?$FLINFO?$FN?3?5?5?5Width?5?$DN?5?$CFd@ 10013a9c     AccessBridgeJavaEntryPoints.obj
 0002:00004ab8       ??_C@_0EG@HOHNFBDJ@?$FLERROR?$FN?3?5?5either?5env?5?$DN?$DN?50?5or?5ge@ 10013ab8     AccessBridgeJavaEntryPoints.obj
 0002:00004b00       ??_C@_0DD@DDJGOHAP@Getting?5AccessibleHeight?5?9?5call@ 10013b00     AccessBridgeJavaEntryPoints.obj
 0002:00004b34       ??_C@_0BG@DJGLJFGH@?$FLINFO?$FN?3?5?5?5Height?5?$DN?5?$CFd@ 10013b34     AccessBridgeJavaEntryPoints.obj
 0002:00004b50       ??_C@_0EH@LBBAABEE@?$FLERROR?$FN?3?5?5either?5env?5?$DN?$DN?50?5or?5ge@ 10013b50     AccessBridgeJavaEntryPoints.obj
 0002:00004b98       ??_C@_0DJ@LNCBBGOH@Getting?5AccessibleComponent?5?9?5c@ 10013b98     AccessBridgeJavaEntryPoints.obj
 0002:00004bd4       ??_C@_0CD@PFGFGKFI@?$FLINFO?$FN?3?5?5?5AccessibleComponent?5?$DN@ 10013bd4     AccessBridgeJavaEntryPoints.obj
 0002:00004bf8       ??_C@_0DH@KGCNAJLL@Getting?5AccessibleComponent?5?9?5c@ 10013bf8     AccessBridgeJavaEntryPoints.obj
 0002:00004c30       ??_C@_0EK@MOFEFKAP@?$FLERROR?$FN?3?5?5either?5env?5?$DN?$DN?50?5or?5ge@ 10013c30     AccessBridgeJavaEntryPoints.obj
 0002:00004c7c       ??_C@_0DG@DACOODAE@Getting?5AccessibleAction?5?9?5call@ 10013c7c     AccessBridgeJavaEntryPoints.obj
 0002:00004cb4       ??_C@_0CA@PJFDOLN@?$FLINFO?$FN?3?5?5?5AccessibleAction?5?$DN?5?$CFp@ 10013cb4     AccessBridgeJavaEntryPoints.obj
 0002:00004cd4       ??_C@_0DE@DDPPAPLP@Getting?5AccessibleAction?5?9?5call@ 10013cd4     AccessBridgeJavaEntryPoints.obj
 0002:00004d08       ??_C@_0EH@DKLGJNHO@?$FLERROR?$FN?3?5?5either?5env?5?$DN?$DN?50?5or?5ge@ 10013d08     AccessBridgeJavaEntryPoints.obj
 0002:00004d50       ??_C@_0DJ@CGHCFMLP@Getting?5AccessibleSelection?5?9?5c@ 10013d50     AccessBridgeJavaEntryPoints.obj
 0002:00004d8c       ??_C@_0CD@PJLLNPAJ@?$FLINFO?$FN?3?5?5?5AccessibleSelection?5?$DN@ 10013d8c     AccessBridgeJavaEntryPoints.obj
 0002:00004db0       ??_C@_0DH@PGPODJFA@Getting?5AccessibleSelection?5?9?5c@ 10013db0     AccessBridgeJavaEntryPoints.obj
 0002:00004de8       ??_C@_0EK@NDMBIFBF@?$FLERROR?$FN?3?5?5either?5env?5?$DN?$DN?50?5or?5ge@ 10013de8     AccessBridgeJavaEntryPoints.obj
 0002:00004e34       ??_C@_0DO@EELLKHNA@?$FLINFO?$FN?3?5?$CD?$CD?$CD?$CD?$CD?5Calling?5getAccess@ 10013e34     AccessBridgeJavaEntryPoints.obj
 0002:00004e78       ??_C@_0EE@BBNKAGDP@?$FLINFO?$FN?3?5?$CD?$CD?$CD?$CD?$CD?5?4?4?4?5Returned?5from@ 10013e78     AccessBridgeJavaEntryPoints.obj
 0002:00004ebc       ??_C@_0DL@DIOKBKHD@?$CD?$CD?$CD?$CD?$CD?5Getting?5AccessibleTable?5?9@ 10013ebc     AccessBridgeJavaEntryPoints.obj
 0002:00004ef8       ??_C@_0CF@KFOMFGJG@?$FLINFO?$FN?3?5?5?5?$CD?$CD?$CD?$CD?$CD?5AccessibleTable@ 10013ef8     AccessBridgeJavaEntryPoints.obj
 0002:00004f20       ??_C@_0DJ@ELALBBFD@?$CD?$CD?$CD?$CD?$CD?5Getting?5AccessibleTable?5?9@ 10013f20     AccessBridgeJavaEntryPoints.obj
 0002:00004f60       ??_C@_0EF@MKDIKDJP@?$FLERROR?$FN?3?5either?5env?5?$DN?$DN?50?5or?5get@ 10013f60     AccessBridgeJavaEntryPoints.obj
 0002:00004fa8       ??_C@_0BO@PJMPGGKG@?$FLINFO?$FN?3?5?5?5AccessibleText?5?$DN?5?$CFp@ 10013fa8     AccessBridgeJavaEntryPoints.obj
 0002:00004fc8       ??_C@_0DF@NJBDDCEL@Getting?5AccessibleValue?5?9?5call?5@ 10013fc8     AccessBridgeJavaEntryPoints.obj
 0002:00005000       ??_C@_0BP@BANALONE@?$FLINFO?$FN?3?5?5?5AccessibleValue?5?$DN?5?$CFp@ 10014000     AccessBridgeJavaEntryPoints.obj
 0002:00005020       ??_C@_0DD@JJHMAHMH@Getting?5AccessibleValue?5?9?5call?5@ 10014020     AccessBridgeJavaEntryPoints.obj
 0002:00005058       ??_C@_0EG@HHMGAANK@?$FLERROR?$FN?3?5?5either?5env?5?$DN?$DN?50?5or?5ge@ 10014058     AccessBridgeJavaEntryPoints.obj
 0002:000050a0       ??_C@_0DJ@EACHBMMF@Getting?5AccessibleHypertext?5?9?5c@ 100140a0     AccessBridgeJavaEntryPoints.obj
 0002:000050dc       ??_C@_0CD@DNELEHHF@?$FLINFO?$FN?3?5?5?5AccessibleHypertext?5?$DN@ 100140dc     AccessBridgeJavaEntryPoints.obj
 0002:00005100       ??_C@_0DH@DONNNDKC@Getting?5AccessibleHypertext?5?9?5c@ 10014100     AccessBridgeJavaEntryPoints.obj
 0002:00005138       ??_C@_0FA@DGBOEHHP@?$FLINFO?$FN?3?5Calling?5AccessBridgeJav@ 10014138     AccessBridgeJavaEntryPoints.obj
 0002:00005188       ??_C@_0DF@OGEEIIFE@Getting?5AccessibleChild?5?9?5call?5@ 10014188     AccessBridgeJavaEntryPoints.obj
 0002:000051c0       ??_C@_0DB@OOCPCHE@Getting?5AccessibleChild?5?9?5call?5@ 100141c0     AccessBridgeJavaEntryPoints.obj
 0002:000051f4       ??_C@_0DD@JNMELFAO@Getting?5AccessibleChild?5?9?5call?5@ 100141f4     AccessBridgeJavaEntryPoints.obj
 0002:00005228       ??_C@_0EC@MDNHELGM@?$FLERROR?$FN?3?5?5either?5env?5?$DN?$DN?50?5or?5ge@ 10014228     AccessBridgeJavaEntryPoints.obj
 0002:00005270       ??_C@_0FB@PNLEIBEF@?$FLINFO?$FN?3?5Calling?5AccessBridgeJav@ 10014270     AccessBridgeJavaEntryPoints.obj
 0002:000052c4       ??_C@_0DG@BJCEEHCN@Getting?5AccessibleParent?5?9?5call@ 100142c4     AccessBridgeJavaEntryPoints.obj
 0002:000052fc       ??_C@_0DC@MKLJMCBC@Getting?5AccessibleParent?5?9?5call@ 100142fc     AccessBridgeJavaEntryPoints.obj
 0002:00005330       ??_C@_0DE@IILKINNI@Getting?5AccessibleParent?5?9?5call@ 10014330     AccessBridgeJavaEntryPoints.obj
 0002:00005368       ??_C@_0EH@MOCAMKEC@?$FLERROR?$FN?3?5?5either?5env?5?$DN?$DN?50?5or?5ge@ 10014368     AccessBridgeJavaEntryPoints.obj
 0002:000053b0       ??_C@_0EP@IDGNPODK@?$FLINFO?$FN?3?5?$CD?$CD?$CD?$CD?$CD?5Calling?5AccessBri@ 100143b0     AccessBridgeJavaEntryPoints.obj
 0002:00005400       ??_C@_0EA@HDPDLION@?$CD?$CD?$CD?$CD?$CD?5Getting?5AccessibleTableRo@ 10014400     AccessBridgeJavaEntryPoints.obj
 0002:00005440       ??_C@_0CF@OMEBMMOI@?$FLINFO?$FN?3?5?5?5?$CD?$CD?$CD?$CD?$CD?5table?5row?5count@ 10014440     AccessBridgeJavaEntryPoints.obj
 0002:00005468       ??_C@_0DN@MNMKPHBJ@?$FLERROR?$FN?3?5either?5env?5?$DN?$DN?50?5or?5get@ 10014468     AccessBridgeJavaEntryPoints.obj
 0002:000054a8       ??_C@_0DN@LHDBHOOP@Getting?5AccessibleTableColumnCo@ 100144a8     AccessBridgeJavaEntryPoints.obj
 0002:000054e8       ??_C@_0CI@GJGENPPF@?$FLINFO?$FN?3?5?5?5?$CD?$CD?$CD?$CD?$CD?5table?5column?5co@ 100144e8     AccessBridgeJavaEntryPoints.obj
 0002:00005510       ??_C@_0EF@LHBDGBA@?$FLERROR?$FN?3?5either?5env?5?$DN?$DN?50?5or?5get@ 10014510     AccessBridgeJavaEntryPoints.obj
 0002:00005558       ??_C@_0DH@GFGBCDOC@?$CD?$CD?$CD?$CD?$CD?5Getting?5AccessibleTable?5?9@ 10014558     AccessBridgeJavaEntryPoints.obj
 0002:00005590       ??_C@_0CF@DCCEHDEO@?$FLINFO?$FN?3?5?5?5?$CD?$CD?$CD?$CD?$CD?5accessibleTable@ 10014590     AccessBridgeJavaEntryPoints.obj
 0002:000055b8       ??_C@_0DP@FLHLIILD@?$FLINFO?$FN?3?5?$CD?$CD?$CD?$CD?$CD?5Calling?5getContex@ 100145b8     AccessBridgeJavaEntryPoints.obj
 0002:000055f8       ??_C@_0EF@JOJDMPNM@?$FLINFO?$FN?3?5?$CD?$CD?$CD?$CD?$CD?5?4?4?4?5Returned?5from@ 100145f8     AccessBridgeJavaEntryPoints.obj
 0002:00005640       ??_C@_0CH@GEKEKGKL@?$FLINFO?$FN?3?5?5?5?$CD?$CD?$CD?$CD?$CD?5accessibleConte@ 10014640     AccessBridgeJavaEntryPoints.obj
 0002:00005668       ??_C@_0EG@CNEBJJDJ@?$FLERROR?$FN?3?5either?5env?5?$DN?$DN?50?5or?5get@ 10014668     AccessBridgeJavaEntryPoints.obj
 0002:000056b0       ??_C@_0FE@GFOFNDOE@?$FLINFO?$FN?3?5?$CD?$CD?$CD?$CD?$CD?5Calling?5AccessBri@ 100146b0     AccessBridgeJavaEntryPoints.obj
 0002:00005708       ??_C@_0GF@GDALOMIB@?$FLINFO?$FN?3?5?$CD?$CD?$CD?$CD?$CD?5Calling?5AccessBri@ 10014708     AccessBridgeJavaEntryPoints.obj
 0002:00005770       ??_C@_0EB@IFJOCDDE@?$CD?$CD?$CD?$CD?$CD?5Getting?5AccessibleTableCe@ 10014770     AccessBridgeJavaEntryPoints.obj
 0002:000057b4       ??_C@_0CG@KKOMOEPJ@?$FLINFO?$FN?3?5?5?5?$CD?$CD?$CD?$CD?$CD?5table?5cell?5inde@ 100147b4     AccessBridgeJavaEntryPoints.obj
 0002:000057e0       ??_C@_0ED@MJPDAFIJ@?$FLERROR?$FN?3?5either?5env?5?$DN?$DN?50?5or?5get@ 100147e0     AccessBridgeJavaEntryPoints.obj
 0002:00005828       ??_C@_0EK@HFAIKGKI@?$CD?$CD?$CD?$CD?$CD?5Getting?5AccessibleTableCe@ 10014828     AccessBridgeJavaEntryPoints.obj
 0002:00005874       ??_C@_0CL@CDCOGIJD@?$FLINFO?$FN?3?5?5?5?$CD?$CD?$CD?$CD?$CD?5table?5cell?5row?5@ 10014874     AccessBridgeJavaEntryPoints.obj
 0002:000058a0       ??_C@_0EH@MFABNFMJ@?$FLERROR?$FN?3?5either?5env?5?$DN?$DN?50?5or?5get@ 100148a0     AccessBridgeJavaEntryPoints.obj
 0002:000058e8       ??_C@_0EN@GIPGNDGO@?$CD?$CD?$CD?$CD?$CD?5Getting?5AccessibleTableCe@ 100148e8     AccessBridgeJavaEntryPoints.obj
 0002:00005938       ??_C@_0CN@JHPAHOLB@?$FLINFO?$FN?3?5?5?$CD?$CD?$CD?$CD?$CD?5table?5cell?5colum@ 10014938     AccessBridgeJavaEntryPoints.obj
 0002:00005968       ??_C@_0EK@MCJJFMIG@?$FLERROR?$FN?3?5either?5env?5?$DN?$DN?50?5or?5get@ 10014968     AccessBridgeJavaEntryPoints.obj
 0002:000059b8       ??_C@_0EK@OAKDMNFI@?$CD?$CD?$CD?$CD?$CD?5Getting?5isAccessibleTable@ 100149b8     AccessBridgeJavaEntryPoints.obj
 0002:00005a04       ??_C@_0CL@FGJJGBAG@?$FLINFO?$FN?3?5?5?5?$CD?$CD?$CD?$CD?$CD?5table?5cell?5isSe@ 10014a04     AccessBridgeJavaEntryPoints.obj
 0002:00005a30       ??_C@_0EF@NDHLMIOL@?$FLERROR?$FN?3?5either?5env?5?$DN?$DN?50?5or?5isA@ 10014a30     AccessBridgeJavaEntryPoints.obj
 0002:00005a78       ??_C@_0FA@PNFLEDNO@?$CD?$CD?$CD?$CD?$CD?5Getting?5AccessibleTableCe@ 10014a78     AccessBridgeJavaEntryPoints.obj
 0002:00005ac8       ??_C@_0EM@CCOLAKIM@?$CD?$CD?$CD?$CD?$CD?5Getting?5AccessibleTableCe@ 10014ac8     AccessBridgeJavaEntryPoints.obj
 0002:00005b14       ??_C@_0DC@NHIEBBHC@?$FLINFO?$FN?3?5?5?5?$CD?$CD?$CD?$CD?$CD?5table?5cell?5Acce@ 10014b14     AccessBridgeJavaEntryPoints.obj
 0002:00005b48       ??_C@_0EP@BAKELAEL@?$FLERROR?$FN?3?5either?5env?5?$DN?$DN?50?5or?5get@ 10014b48     AccessBridgeJavaEntryPoints.obj
 0002:00005b98       ??_C@_0FJ@JCFFKNHH@?$FLINFO?$FN?3?5?5?$CD?$CD?$CD?$CD?$CD?5Calling?5AccessBr@ 10014b98     AccessBridgeJavaEntryPoints.obj
 0002:00005bf8       ??_C@_0FE@DGILOPPB@?$FLINFO?$FN?3?5?$CD?$CD?$CD?$CD?$CD?5Calling?5AccessBri@ 10014bf8     AccessBridgeJavaEntryPoints.obj
 0002:00005c50       ??_C@_0EJ@OONHAJKO@?$CD?$CD?$CD?$CD?$CD?5Getting?5AccessibleTableRo@ 10014c50     AccessBridgeJavaEntryPoints.obj
 0002:00005ca0       ??_C@_0EG@NDBCAEFO@?$FLERROR?$FN?3?5either?5env?5?$DN?$DN?50?5or?5get@ 10014ca0     AccessBridgeJavaEntryPoints.obj
 0002:00005ce8       ??_C@_0EG@DALLPPNJ@Getting?5AccessibleTableRowHeade@ 10014ce8     AccessBridgeJavaEntryPoints.obj
 0002:00005d30       ??_C@_0EO@OOHGOEEK@?$FLERROR?$FN?3?5either?5env?5?$DN?$DN?50?5or?5get@ 10014d30     AccessBridgeJavaEntryPoints.obj
 0002:00005d80       ??_C@_0EE@GCIECGJK@?$CD?$CD?$CD?$CD?$CD?5Getting?5AccessibleTableRo@ 10014d80     AccessBridgeJavaEntryPoints.obj
 0002:00005dc8       ??_C@_0EA@OEOKKCMN@?$CD?$CD?$CD?$CD?$CD?5Getting?5AccessibleTableRo@ 10014dc8     AccessBridgeJavaEntryPoints.obj
 0002:00005e08       ??_C@_0DA@BEAKBEEG@?$FLINFO?$FN?3?5?5?5?$CD?$CD?$CD?$CD?$CD?5row?5header?5Acce@ 10014e08     AccessBridgeJavaEntryPoints.obj
 0002:00005e38       ??_C@_0ED@KKINKAGC@?$FLERROR?$FN?3?5either?5env?5?$DN?$DN?50?5or?5get@ 10014e38     AccessBridgeJavaEntryPoints.obj
 0002:00005e80       ??_C@_0FL@PPBJDPIL@?$FLINFO?$FN?3?5?5?5?$CD?$CD?$CD?$CD?$CD?5Calling?5AccessB@ 10014e80     AccessBridgeJavaEntryPoints.obj
 0002:00005ee0       ??_C@_0FH@EJOHBEGH@?$FLINFO?$FN?3?5?$CD?$CD?$CD?$CD?$CD?5Calling?5AccessBri@ 10014ee0     AccessBridgeJavaEntryPoints.obj
 0002:00005f38       ??_C@_0EM@ILKGOFLG@?$CD?$CD?$CD?$CD?$CD?5Getting?5AccessibleTableCo@ 10014f38     AccessBridgeJavaEntryPoints.obj
 0002:00005f88       ??_C@_0EK@LPGMLANE@?$FLERROR?$FN?3?5?5either?5env?5?$DN?$DN?50?5or?5ge@ 10014f88     AccessBridgeJavaEntryPoints.obj
 0002:00005fd8       ??_C@_0EJ@CKEIFDID@Getting?5AccessibleTableColumnHe@ 10014fd8     AccessBridgeJavaEntryPoints.obj
 0002:00006028       ??_C@_0FB@LHNIAEHP@?$FLERROR?$FN?3?5either?5env?5?$DN?$DN?50?5or?5get@ 10015028     AccessBridgeJavaEntryPoints.obj
 0002:00006080       ??_C@_0EH@JIOGAIC@?$CD?$CD?$CD?$CD?$CD?5Getting?5AccessibleTableCo@ 10015080     AccessBridgeJavaEntryPoints.obj
 0002:000060c8       ??_C@_0ED@DCBGPFPL@?$CD?$CD?$CD?$CD?$CD?5Getting?5AccessibleTableCo@ 100150c8     AccessBridgeJavaEntryPoints.obj
 0002:0000610c       ??_C@_0DD@JPNBDACB@?$FLINFO?$FN?3?5?5?5?$CD?$CD?$CD?$CD?$CD?5column?5header?5A@ 1001510c     AccessBridgeJavaEntryPoints.obj
 0002:00006140       ??_C@_0EG@EHCJNLHA@?$FLERROR?$FN?3?5either?5env?5?$DN?$DN?50?5or?5get@ 10015140     AccessBridgeJavaEntryPoints.obj
 0002:00006188       ??_C@_0FO@DKAHOFOA@?$FLINFO?$FN?3?5?5?5?$CD?$CD?$CD?$CD?$CD?5Calling?5AccessB@ 10015188     AccessBridgeJavaEntryPoints.obj
 0002:000061e8       ??_C@_0FJ@IPEPPO@?$FLINFO?$FN?3?5?$CD?$CD?$CD?$CD?$CD?5Calling?5AccessBri@ 100151e8     AccessBridgeJavaEntryPoints.obj
 0002:00006248       ??_C@_0ED@ECGPKBKB@Getting?5AccessibleTableRowDescr@ 10015248     AccessBridgeJavaEntryPoints.obj
 0002:0000628c       ??_C@_0DP@MGPIFPGE@Getting?5AccessibleTableRowDescr@ 1001528c     AccessBridgeJavaEntryPoints.obj
 0002:000062d0       ??_C@_0EB@HPGBLABA@Getting?5AccessibleTableRowDescr@ 100152d0     AccessBridgeJavaEntryPoints.obj
 0002:00006318       ??_C@_0EI@FALMFIJI@?$FLERROR?$FN?3?5either?5env?5?$DN?$DN?50?5or?5get@ 10015318     AccessBridgeJavaEntryPoints.obj
 0002:00006360       ??_C@_0FM@OGMEFLJF@?$FLINFO?$FN?3?5?$CD?$CD?$CD?$CD?$CD?5Calling?5AccessBri@ 10015360     AccessBridgeJavaEntryPoints.obj
 0002:000063c0       ??_C@_0EG@HNHAKGAA@Getting?5AccessibleTableColumnDe@ 100153c0     AccessBridgeJavaEntryPoints.obj
 0002:00006408       ??_C@_0EC@OOIBKPKB@Getting?5AccessibleTableColumnDe@ 10015408     AccessBridgeJavaEntryPoints.obj
 0002:00006450       ??_C@_0EE@HEFBEJHO@Getting?5AccessibleTableColumnDe@ 10015450     AccessBridgeJavaEntryPoints.obj
 0002:00006498       ??_C@_0EL@MDADMDPK@?$FLERROR?$FN?3?5either?5env?5?$DN?$DN?50?5or?5get@ 10015498     AccessBridgeJavaEntryPoints.obj
 0002:000064e8       ??_C@_0FD@NONCILOI@?$FLINFO?$FN?3?5?$CD?$CD?$CD?$CD?$CD?5AccessBridgeJavaE@ 100154e8     AccessBridgeJavaEntryPoints.obj
 0002:00006540       ??_C@_0EJ@CONOFLFI@?$CD?$CD?$CD?$CD?$CD?5Getting?5AccessibleTableRo@ 10015540     AccessBridgeJavaEntryPoints.obj
 0002:0000658c       ??_C@_0CP@GJAEEGNO@?$FLINFO?$FN?3?5?5?5?$CD?$CD?$CD?$CD?$CD?5table?5row?5selec@ 1001558c     AccessBridgeJavaEntryPoints.obj
 0002:000065c0       ??_C@_0EL@JIBDDMIF@?$FLERROR?$FN?3?5either?5env?5?$DN?$DN?50?5or?5get@ 100155c0     AccessBridgeJavaEntryPoints.obj
 0002:00006610       ??_C@_0FA@LAKDEELL@?$FLINFO?$FN?3?5?$CD?$CD?$CD?$CD?$CD?5AccessBridgeJavaE@ 10015610     AccessBridgeJavaEntryPoints.obj
 0002:00006660       ??_C@_0EJ@PAIANDP@?$CD?$CD?$CD?$CD?$CD?5Getting?5isAccessibleTable@ 10015660     AccessBridgeJavaEntryPoints.obj
 0002:000066ac       ??_C@_0CK@ENCKDAKJ@?$FLINFO?$FN?3?5?5?5?$CD?$CD?$CD?$CD?$CD?5table?5row?5isSel@ 100156ac     AccessBridgeJavaEntryPoints.obj
 0002:000066d8       ??_C@_0EE@OPDECGCG@?$FLERROR?$FN?3?5either?5env?5?$DN?$DN?50?5or?5isA@ 100156d8     AccessBridgeJavaEntryPoints.obj
 0002:00006720       ??_C@_0FG@BNGDNOAB@?$FLINFO?$FN?3?5?$CD?$CD?$CD?$CD?$CD?5AccessBridgeJavaE@ 10015720     AccessBridgeJavaEntryPoints.obj
 0002:00006778       ??_C@_0EF@MANEDMPN@?$CD?$CD?$CD?$CD?$CD?5Getting?5AccessibleTableRo@ 10015778     AccessBridgeJavaEntryPoints.obj
 0002:000067c0       ??_C@_0CN@EGDPALEC@?$FLINFO?$FN?3?5?5?5?$CD?$CD?$CD?$CD?$CD?5table?5row?5selec@ 100157c0     AccessBridgeJavaEntryPoints.obj
 0002:000067f0       ??_C@_0FH@IBIGBELL@?$FLINFO?$FN?3?5?5?5?$CD?$CD?$CD?$CD?$CD?5AccessBridgeJav@ 100157f0     AccessBridgeJavaEntryPoints.obj
 0002:00006848       ??_C@_0FG@LAILABJF@?$FLINFO?$FN?3?5?$CD?$CD?$CD?$CD?$CD?5AccessBridgeJavaE@ 10015848     AccessBridgeJavaEntryPoints.obj
 0002:000068a0       ??_C@_0EM@ELKPLHEA@?$CD?$CD?$CD?$CD?$CD?5Getting?5AccessibleTableCo@ 100158a0     AccessBridgeJavaEntryPoints.obj
 0002:000068ec       ??_C@_0DC@EFKBJLFF@?$FLINFO?$FN?3?5?5?5?$CD?$CD?$CD?$CD?$CD?5table?5column?5se@ 100158ec     AccessBridgeJavaEntryPoints.obj
 0002:00006920       ??_C@_0FD@ODFPPIDD@?$FLINFO?$FN?3?5?$CD?$CD?$CD?$CD?$CD?5AccessBridgeJavaE@ 10015920     AccessBridgeJavaEntryPoints.obj
 0002:00006978       ??_C@_0EM@HPIPAKED@?$CD?$CD?$CD?$CD?$CD?5Getting?5isAccessibleTable@ 10015978     AccessBridgeJavaEntryPoints.obj
 0002:000069c4       ??_C@_0CN@OPIEHDOO@?$FLINFO?$FN?3?5?5?5?$CD?$CD?$CD?$CD?$CD?5table?5column?5is@ 100159c4     AccessBridgeJavaEntryPoints.obj
 0002:000069f8       ??_C@_0EI@CBBNNOEE@?$FLERROR?$FN?3?5?5either?5env?5?$DN?$DN?50?5or?5is@ 100159f8     AccessBridgeJavaEntryPoints.obj
 0002:00006a40       ??_C@_0FK@KHEECFFC@?$FLINFO?$FN?3?5?$CD?$CD?$CD?$CD?$CD?5AccessBridgeJavaE@ 10015a40     AccessBridgeJavaEntryPoints.obj
 0002:00006aa0       ??_C@_0EI@NDNDKOON@?$CD?$CD?$CD?$CD?$CD?5Getting?5AccessibleTableCo@ 10015aa0     AccessBridgeJavaEntryPoints.obj
 0002:00006ae8       ??_C@_0DA@FGAFLCDN@?$FLINFO?$FN?3?5?5?5?$CD?$CD?$CD?$CD?$CD?5table?5Column?5se@ 10015ae8     AccessBridgeJavaEntryPoints.obj
 0002:00006b18       ??_C@_0FK@PECCMPIL@?$FLINFO?$FN?3?5?5?5?$CD?$CD?$CD?$CD?$CD?5AccessBridgeJav@ 10015b18     AccessBridgeJavaEntryPoints.obj
 0002:00006b78       ??_C@_0EP@DEKNIMFA@?$FLINFO?$FN?3?5?$CD?$CD?$CD?$CD?$CD?5AccessBridgeJavaE@ 10015b78     AccessBridgeJavaEntryPoints.obj
 0002:00006bc8       ??_C@_0DL@DELNDLCL@?$CD?$CD?$CD?$CD?$CD?5Getting?5AccessibleTableRo@ 10015bc8     AccessBridgeJavaEntryPoints.obj
 0002:00006c04       ??_C@_0BP@MEJOIGMM@?$FLINFO?$FN?3?5?5?5?$CD?$CD?$CD?$CD?$CD?5table?5row?5?$DN?5?$CFd@ 10015c04     AccessBridgeJavaEntryPoints.obj
 0002:00006c24       ??_C@_0DN@DIFOEGJK@?$FLERROR?$FN?3?5either?5env?5?$DN?$DN?50?5or?5get@ 10015c24     AccessBridgeJavaEntryPoints.obj
 0002:00006c68       ??_C@_0FC@BFBAOEGI@?$FLINFO?$FN?3?5?$CD?$CD?$CD?$CD?$CD?5AccessBridgeJavaE@ 10015c68     AccessBridgeJavaEntryPoints.obj
 0002:00006cbc       ??_C@_0DO@MBGEOOOH@?$CD?$CD?$CD?$CD?$CD?5Getting?5AccessibleTableCo@ 10015cbc     AccessBridgeJavaEntryPoints.obj
 0002:00006cfc       ??_C@_0CC@CJBEHFKG@?$FLINFO?$FN?3?5?5?5?$CD?$CD?$CD?$CD?$CD?5table?5column?5?$DN?5@ 10015cfc     AccessBridgeJavaEntryPoints.obj
 0002:00006d20       ??_C@_0EA@IFBLPNLC@?$FLERROR?$FN?3?5either?5env?5?$DN?$DN?50?5or?5get@ 10015d20     AccessBridgeJavaEntryPoints.obj
 0002:00006d60       ??_C@_0FH@GMMGKHHK@?$FLINFO?$FN?3?5?$CD?$CD?$CD?$CD?$CD?5AccessBridgeJavaE@ 10015d60     AccessBridgeJavaEntryPoints.obj
 0002:00006db8       ??_C@_0EA@IDLLLJIK@?$CD?$CD?$CD?$CD?$CD?5Getting?5getAccessibleTabl@ 10015db8     AccessBridgeJavaEntryPoints.obj
 0002:00006df8       ??_C@_0CB@JIHDIDBK@?$FLINFO?$FN?3?5?5?5?$CD?$CD?$CD?$CD?$CD?5table?5index?5?$DN?5?$CF@ 10015df8     AccessBridgeJavaEntryPoints.obj
 0002:00006e1c       ??_C@_0DP@EPGMKJOF@?$FLERROR?$FN?3?5either?5env?5?$DN?$DN?50?5or?5get@ 10015e1c     AccessBridgeJavaEntryPoints.obj
 0002:00006e60       ??_C@_0EM@OMNMKDMF@?$FLINFO?$FN?3?5?$CD?$CD?$CD?$CD?$CD?5AccessBridgeJavaE@ 10015e60     AccessBridgeJavaEntryPoints.obj
 0002:00006eb0       ??_C@_0EA@LPBOBAAO@?$CD?$CD?$CD?$CD?$CD?5Getting?5AccessibleRelatio@ 10015eb0     AccessBridgeJavaEntryPoints.obj
 0002:00006ef0       ??_C@_0CO@JNBGELMK@?$FLINFO?$FN?3?5?5?5?$CD?$CD?$CD?$CD?$CD?5AccessibleRelat@ 10015ef0     AccessBridgeJavaEntryPoints.obj
 0002:00006f20       ??_C@_0DL@KJPPMLJK@Getting?5AccessibleRelationKey?5?9@ 10015f20     AccessBridgeJavaEntryPoints.obj
 0002:00006f5c       ??_C@_0DK@CJPLLCPL@Getting?5AccessibleRelation?5key?5@ 10015f5c     AccessBridgeJavaEntryPoints.obj
 0002:00006f98       ??_C@_0DL@KHBJJIBG@Getting?5AccessibleRelation?5key?5@ 10015f98     AccessBridgeJavaEntryPoints.obj
 0002:00006fd4       ??_C@_0DO@GNGKCACF@Getting?5AccessibleRelation?5key?5@ 10015fd4     AccessBridgeJavaEntryPoints.obj
 0002:00007014       ??_C@_0CL@LKNHIIFA@?$FLINFO?$FN?3?5?$CD?$CD?$CD?$CD?$CD?5AccessibleRelatio@ 10016014     AccessBridgeJavaEntryPoints.obj
 0002:00007040       ??_C@_0DK@OHAOHAGF@Getting?5AccessibleRelation?5key?5@ 10016040     AccessBridgeJavaEntryPoints.obj
 0002:0000707c       ??_C@_0CK@FLLDFIHJ@?$FLWARN?$FN?3?5?5?5AccessibleRelation?5ke@ 1001607c     AccessBridgeJavaEntryPoints.obj
 0002:000070a8       ??_C@_0DL@FOJGEEOM@Getting?5AccessibleRelationSet?5?9@ 100160a8     AccessBridgeJavaEntryPoints.obj
 0002:000070e4       ??_C@_0DH@OOCHFOKL@Getting?5AccessibleRelationSet?5?9@ 100160e4     AccessBridgeJavaEntryPoints.obj
 0002:0000711c       ??_C@_0CA@NHODALDJ@?$FLINFO?$FN?3?5?5?5relation?5set?5item?3?5?$CFp@ 1001611c     AccessBridgeJavaEntryPoints.obj
 0002:00007140       ??_C@_0FA@NBCFFMGI@?$FLINFO?$FN?3?5?5?5?$CD?$CD?$CD?$CD?$CD?5AccessBridgeJav@ 10016140     AccessBridgeJavaEntryPoints.obj
 0002:00007190       ??_C@_0EK@KKPLDFBH@?$FLINFO?$FN?3?5?$CD?$CD?$CD?$CD?$CD?5AccessBridgeJavaE@ 10016190     AccessBridgeJavaEntryPoints.obj
 0002:000071dc       ??_C@_0DP@KAHCJAMC@?$CD?$CD?$CD?$CD?$CD?5Getting?5AccessibleHyperte@ 100161dc     AccessBridgeJavaEntryPoints.obj
 0002:0000721c       ??_C@_0DL@BCGGEGFO@?$CD?$CD?$CD?$CD?$CD?5Getting?5AccessibleHyperte@ 1001621c     AccessBridgeJavaEntryPoints.obj
 0002:00007258       ??_C@_0CJ@KAIOACGL@?$FLINFO?$FN?3?5?5?5?$CD?$CD?$CD?$CD?$CD?5AccessibleHyper@ 10016258     AccessBridgeJavaEntryPoints.obj
 0002:00007284       ??_C@_0DK@IMJHJIPP@?$FLWARN?$FN?3?5?5?5?$CD?$CD?$CD?$CD?$CD?5null?5Accessible@ 10016284     AccessBridgeJavaEntryPoints.obj
 0002:000072c0       ??_C@_0DI@FEBHIMOE@?$CD?$CD?$CD?$CD?$CD?5Getting?5hyperlink?5count?5?9@ 100162c0     AccessBridgeJavaEntryPoints.obj
 0002:000072f8       ??_C@_0CF@OFPNIMKK@?$FLINFO?$FN?3?5?5?5?$CD?$CD?$CD?$CD?$CD?5hyperlink?5count@ 100162f8     AccessBridgeJavaEntryPoints.obj
 0002:00007320       ??_C@_0DP@CIGIOMPM@?$CD?$CD?$CD?$CD?$CD?5Getting?5AccessibleHyperli@ 10016320     AccessBridgeJavaEntryPoints.obj
 0002:00007360       ??_C@_0DL@PDIOCHOJ@?$CD?$CD?$CD?$CD?$CD?5Getting?5AccessibleHyperli@ 10016360     AccessBridgeJavaEntryPoints.obj
 0002:0000739c       ??_C@_0CJ@FJIBOEOI@?$FLINFO?$FN?3?5?5?5?$CD?$CD?$CD?$CD?$CD?5AccessibleHyper@ 1001639c     AccessBridgeJavaEntryPoints.obj
 0002:000073c8       ??_C@_0DE@FAMBBMPD@Getting?5hyperlink?5text?5?9?5call?5t@ 100163c8     AccessBridgeJavaEntryPoints.obj
 0002:000073fc       ??_C@_0DM@FFPIAIEA@Getting?5AccessibleHyperlink?5tex@ 100163fc     AccessBridgeJavaEntryPoints.obj
 0002:00007438       ??_C@_0DN@PLNGPBKI@Getting?5AccessibleHyperlink?5tex@ 10016438     AccessBridgeJavaEntryPoints.obj
 0002:00007478       ??_C@_0EA@BNEOPMKM@Getting?5AccessibleHyperlink?5tex@ 10016478     AccessBridgeJavaEntryPoints.obj
 0002:000074b8       ??_C@_0CN@IIHGCCLN@?$FLINFO?$FN?3?5?$CD?$CD?$CD?$CD?$CD?5AccessibleHyperli@ 100164b8     AccessBridgeJavaEntryPoints.obj
 0002:000074e8       ??_C@_0DM@JLANMKNO@Getting?5AccessibleHyperlink?5tex@ 100164e8     AccessBridgeJavaEntryPoints.obj
 0002:00007524       ??_C@_0CM@DKPAOLF@?$FLWARN?$FN?3?5?5?5AccessibleHyperlink?5t@ 10016524     AccessBridgeJavaEntryPoints.obj
 0002:00007550       ??_C@_0DO@DJICJOGB@?$CD?$CD?$CD?$CD?$CD?5Getting?5hyperlink?5start?5i@ 10016550     AccessBridgeJavaEntryPoints.obj
 0002:00007590       ??_C@_0CL@GNKIIEKN@?$FLINFO?$FN?3?5?5?5?$CD?$CD?$CD?$CD?$CD?5hyperlink?5start@ 10016590     AccessBridgeJavaEntryPoints.obj
 0002:000075bc       ??_C@_0DM@MGHLFEBK@?$CD?$CD?$CD?$CD?$CD?5Getting?5hyperlink?5end?5ind@ 100165bc     AccessBridgeJavaEntryPoints.obj
 0002:000075f8       ??_C@_0CJ@POHPAAGA@?$FLINFO?$FN?3?5?5?5?$CD?$CD?$CD?$CD?$CD?5hyperlink?5end?5i@ 100165f8     AccessBridgeJavaEntryPoints.obj
 0002:00007628       ??_C@_0EO@MCEJOGLJ@?$FLINFO?$FN?3?5?5?5?$CD?$CD?$CD?$CD?$CD?5AccessBridgeJav@ 10016628     AccessBridgeJavaEntryPoints.obj
 0002:00007678       ??_C@_0FC@PJEJEFPL@?$FLINFO?$FN?3?5Calling?5AccessBridgeJav@ 10016678     AccessBridgeJavaEntryPoints.obj
 0002:000076cc       ??_C@_0DK@IAFPEHK@activateAccessibleHyperlink?5?9?5c@ 100166cc     AccessBridgeJavaEntryPoints.obj
 0002:00007708       ??_C@_0EG@NBDJGANF@?$FLERROR?$FN?3?5either?5jniEnv?5?$DN?$DN?50?5or?5@ 10016708     AccessBridgeJavaEntryPoints.obj
 0002:00007750       ??_C@_0FO@LCEKGOMG@?$FLINFO?$FN?3?5?$CD?$CD?$CD?$CD?$CD?5AccessBridgeJavaE@ 10016750     AccessBridgeJavaEntryPoints.obj
 0002:000077b0       ??_C@_0CD@FKJEEIHP@?$FLINFO?$FN?3?5?5?5getting?5hyperlink?5?$CFd?5@ 100167b0     AccessBridgeJavaEntryPoints.obj
 0002:000077d8       ??_C@_0FB@LIBMBPHJ@?$FLINFO?$FN?3?5?5?5?$CD?$CD?$CD?$CD?$CD?5AccessBridgeJav@ 100167d8     AccessBridgeJavaEntryPoints.obj
 0002:00007830       ??_C@_0EL@OJOFGNCE@?$FLINFO?$FN?3?5?$CD?$CD?$CD?$CD?$CD?5AccessBridgeJavaE@ 10016830     AccessBridgeJavaEntryPoints.obj
 0002:00007880       ??_C@_0FL@JFFPJPNI@?$FLINFO?$FN?3?5?$CD?$CD?$CD?$CD?$CD?5AccessBridgeJavaE@ 10016880     AccessBridgeJavaEntryPoints.obj
 0002:000078dc       ??_C@_0DI@MNABDACM@?$CD?$CD?$CD?$CD?$CD?5Getting?5hyperlink?5index?5?9@ 100168dc     AccessBridgeJavaEntryPoints.obj
 0002:00007914       ??_C@_0CF@MJOBJPAA@?$FLINFO?$FN?3?5?5?5?$CD?$CD?$CD?$CD?$CD?5hyperlink?5index@ 10016914     AccessBridgeJavaEntryPoints.obj
 0002:00007940       ??_C@_0FC@MDIFEEKA@?$FLINFO?$FN?3?5?$CD?$CD?$CD?$CD?$CD?5AccessBridgeJavaE@ 10016940     AccessBridgeJavaEntryPoints.obj
 0002:00007998       ??_C@_0EM@DFNHGKKP@?$FLINFO?$FN?3?5?$CD?$CD?$CD?$CD?$CD?5AccessBridgeJavaE@ 10016998     AccessBridgeJavaEntryPoints.obj
 0002:000079e4       ??_C@_0DL@CLKJJKNH@?$CD?$CD?$CD?$CD?$CD?5Getting?5key?5bindings?5coun@ 100169e4     AccessBridgeJavaEntryPoints.obj
 0002:00007a20       ??_C@_0CI@OKJNHPKA@?$FLINFO?$FN?3?5?5?5?$CD?$CD?$CD?$CD?$CD?5key?5bindings?5co@ 10016a20     AccessBridgeJavaEntryPoints.obj
 0002:00007a48       ??_C@_0DP@FMCKMBKC@?$CD?$CD?$CD?$CD?$CD?5Getting?5key?5binding?5chara@ 10016a48     AccessBridgeJavaEntryPoints.obj
 0002:00007a88       ??_C@_0FN@DCEDCNML@?$FLINFO?$FN?3?5?5?5?$CD?$CD?$CD?$CD?$CD?5key?5binding?5cha@ 10016a88     AccessBridgeJavaEntryPoints.obj
 0002:00007ae8       ??_C@_0DO@HKGJEFDO@?$CD?$CD?$CD?$CD?$CD?5Getting?5key?5binding?5modif@ 10016ae8     AccessBridgeJavaEntryPoints.obj
 0002:00007b28       ??_C@_0CK@OFBJGPDI@?$FLINFO?$FN?3?5?5?$CD?$CD?$CD?$CD?$CD?5key?5binding?5modi@ 10016b28     AccessBridgeJavaEntryPoints.obj
 0002:00007b58       ??_C@_0EG@MKCABNJD@?$FLINFO?$FN?3?5?$CD?$CD?$CD?$CD?$CD?5AccessBridgeJavaE@ 10016b58     AccessBridgeJavaEntryPoints.obj
 0002:00007ba0       ??_C@_0CG@IDHCCFPM@?$FLWARN?$FN?3?5?5?5?$CD?$CD?$CD?$CD?$CD?5missing?5method?$CI@ 10016ba0     AccessBridgeJavaEntryPoints.obj
 0002:00007bc8       ??_C@_0DE@JDHACCPK@?$CD?$CD?$CD?$CD?$CD?5Getting?5icons?5count?5?9?5cal@ 10016bc8     AccessBridgeJavaEntryPoints.obj
 0002:00007bfc       ??_C@_0CB@DPKCEABK@?$FLINFO?$FN?3?5?5?5?$CD?$CD?$CD?$CD?$CD?5icons?5count?5?$DN?5?$CF@ 10016bfc     AccessBridgeJavaEntryPoints.obj
 0002:00007c20       ??_C@_0DG@HKLCCMCD@Getting?5icon?5description?5?9?5call@ 10016c20     AccessBridgeJavaEntryPoints.obj
 0002:00007c58       ??_C@_0DO@JICPIJF@Getting?5AccessibleIcon?5descript@ 10016c58     AccessBridgeJavaEntryPoints.obj
 0002:00007c98       ??_C@_0DP@NDDKNAD@Getting?5AccessibleIcon?5descript@ 10016c98     AccessBridgeJavaEntryPoints.obj
 0002:00007cd8       ??_C@_0EC@OANEKHE@Getting?5AccessibleIcon?5descript@ 10016cd8     AccessBridgeJavaEntryPoints.obj
 0002:00007d1c       ??_C@_0CP@OGEOHJKD@?$FLINFO?$FN?3?5?$CD?$CD?$CD?$CD?$CD?5AccessibleIcon?5de@ 10016d1c     AccessBridgeJavaEntryPoints.obj
 0002:00007d4c       ??_C@_0DO@MHHHDKAL@Getting?5AccessibleIcon?5descript@ 10016d4c     AccessBridgeJavaEntryPoints.obj
 0002:00007d8c       ??_C@_0CO@EGEFBBBG@?$FLWARN?$FN?3?5?5?5AccessibleIcon?5descri@ 10016d8c     AccessBridgeJavaEntryPoints.obj
 0002:00007dbc       ??_C@_0DE@GOAGCEO@?$CD?$CD?$CD?$CD?$CD?5Getting?5icon?5height?5?9?5cal@ 10016dbc     AccessBridgeJavaEntryPoints.obj
 0002:00007df0       ??_C@_0CB@BMHPADNP@?$FLINFO?$FN?3?5?5?5?$CD?$CD?$CD?$CD?$CD?5icon?5height?5?$DN?5?$CF@ 10016df0     AccessBridgeJavaEntryPoints.obj
 0002:00007e14       ??_C@_0DD@EHAOAGFJ@?$CD?$CD?$CD?$CD?$CD?5Getting?5icon?5width?5?9?5call@ 10016e14     AccessBridgeJavaEntryPoints.obj
 0002:00007e48       ??_C@_0CA@DPEBDDDD@?$FLINFO?$FN?3?5?5?5?$CD?$CD?$CD?$CD?$CD?5icon?5width?5?$DN?5?$CFd@ 10016e48     AccessBridgeJavaEntryPoints.obj
 0002:00007e68       ??_C@_0DG@DLFAKGJK@?$CD?$CD?$CD?$CD?$CD?5Getting?5actions?5count?5?9?5c@ 10016e68     AccessBridgeJavaEntryPoints.obj
 0002:00007ea0       ??_C@_0CH@EOBAHIJB@?$FLINFO?$FN?3?5?5?5?$CD?$CD?$CD?$CD?$CD?5key?5actions?5cou@ 10016ea0     AccessBridgeJavaEntryPoints.obj
 0002:00007ec8       ??_C@_0DC@LHBGBJKA@Getting?5Action?5Name?5?5?9?5call?5to?5@ 10016ec8     AccessBridgeJavaEntryPoints.obj
 0002:00007efc       ??_C@_0DK@MCEEGDOO@Getting?5AccessibleAction?5Name?5?5@ 10016efc     AccessBridgeJavaEntryPoints.obj
 0002:00007f38       ??_C@_0DL@IBEDPAGK@Getting?5AccessibleAction?5name?5?5@ 10016f38     AccessBridgeJavaEntryPoints.obj
 0002:00007f74       ??_C@_0DO@BGBLOIHC@Getting?5AccessibleAction?5name?5?5@ 10016f74     AccessBridgeJavaEntryPoints.obj
 0002:00007fb4       ??_C@_0CL@LDPKEJLA@?$FLINFO?$FN?3?5?$CD?$CD?$CD?$CD?$CD?5AccessibleAction?5@ 10016fb4     AccessBridgeJavaEntryPoints.obj
 0002:00007fe0       ??_C@_0DK@GEFGKAFF@Getting?5AccessibleAction?5name?5?5@ 10016fe0     AccessBridgeJavaEntryPoints.obj
 0002:0000801c       ??_C@_0CK@GFGPDCKK@?$FLWARN?$FN?3?5?5?5AccessibleAction?5name@ 1001701c     AccessBridgeJavaEntryPoints.obj
 0002:00008048       ??_C@_0FG@HPHLKACM@?$FLINFO?$FN?3?5Calling?5AccessBridgeJav@ 10017048     AccessBridgeJavaEntryPoints.obj
 0002:000080a0       ??_C@_0CB@NAFFMPJL@?$FLINFO?$FN?3?5?5?5?5?5doing?5?$CFd?5actions?5?4?4@ 100170a0     AccessBridgeJavaEntryPoints.obj
 0002:000080c4       ??_C@_0CE@MIPOFJEF@?$FLINFO?$FN?3?5?5?5?5?5doing?5action?5?$CFd?3?5?$CFs@ 100170c4     AccessBridgeJavaEntryPoints.obj
 0002:000080e8       ??_C@_0DC@PKIFPAKH@doAccessibleActions?5?9?5call?5to?5C@ 100170e8     AccessBridgeJavaEntryPoints.obj
 0002:0000811c       ??_C@_0BO@OONLHHCL@?$FLERROR?$FN?3?5?5?5?5?5Action?5?$CFd?5failed@ 1001711c     AccessBridgeJavaEntryPoints.obj
 0002:00008140       ??_C@_0FA@KEPHMGGF@?$FLINFO?$FN?3?5Calling?5AccessBridgeJav@ 10017140     AccessBridgeJavaEntryPoints.obj
 0002:00008190       ??_C@_0DG@GCJDNJFK@Getting?5AccessibleCharCount?5?9?5c@ 10017190     AccessBridgeJavaEntryPoints.obj
 0002:000081c8       ??_C@_0BK@OIDALDPI@?$FLINFO?$FN?3?5?5?5Char?5count?5?$DN?5?$CFd@ 100171c8     AccessBridgeJavaEntryPoints.obj
 0002:000081e8       ??_C@_0EJ@JKPJJPMH@?$FLERROR?$FN?3?5either?5env?5?$DN?$DN?50?5or?5get@ 100171e8     AccessBridgeJavaEntryPoints.obj
 0002:00008234       ??_C@_0DK@EFHALPMO@Getting?5AccessibleCaretPosition@ 10017234     AccessBridgeJavaEntryPoints.obj
 0002:00008270       ??_C@_0BO@CCCENNB@?$FLINFO?$FN?3?5?5?5Index?5at?5caret?5?$DN?5?$CFd@ 10017270     AccessBridgeJavaEntryPoints.obj
 0002:00008290       ??_C@_0EN@DJGOBIMD@?$FLERROR?$FN?3?5either?5env?5?$DN?$DN?50?5or?5get@ 10017290     AccessBridgeJavaEntryPoints.obj
 0002:000082e0       ??_C@_0DJ@MLOJKMJI@Getting?5AccessibleIndexAtPoint?5@ 100172e0     AccessBridgeJavaEntryPoints.obj
 0002:0000831c       ??_C@_0BO@FIAABPFC@?$FLINFO?$FN?3?5?5?5Index?5at?5point?5?$DN?5?$CFd@ 1001731c     AccessBridgeJavaEntryPoints.obj
 0002:00008340       ??_C@_0EM@ENNBLMPC@?$FLERROR?$FN?3?5either?5env?5?$DN?$DN?50?5or?5get@ 10017340     AccessBridgeJavaEntryPoints.obj
 0002:00008390       ??_C@_0EJ@KDHBNGHD@?$FLINFO?$FN?3?5Calling?5AccessBridgeJav@ 10017390     AccessBridgeJavaEntryPoints.obj
 0002:000083dc       ??_C@_0DK@CALJAPAO@Getting?5AccessibleLetterAtIndex@ 100173dc     AccessBridgeJavaEntryPoints.obj
 0002:00008418       ??_C@_0DL@JDJLEMDG@Getting?5AccessibleLetterAtIndex@ 10017418     AccessBridgeJavaEntryPoints.obj
 0002:00008454       ??_C@_0DP@BIFOHJBB@Getting?5AccessibleLetterAtIndex@ 10017454     AccessBridgeJavaEntryPoints.obj
 0002:00008494       ??_C@_0DL@OOLFPOBK@Getting?5AccessibleLetterAtIndex@ 10017494     AccessBridgeJavaEntryPoints.obj
 0002:000084d0       ??_C@_0CG@BAFOKJKC@?$FLINFO?$FN?3?5?5?5Accessible?5Text?5lette@ 100174d0     AccessBridgeJavaEntryPoints.obj
 0002:000084f8       ??_C@_0DL@FNGOIOKI@Getting?5AccessibleLetterAtIndex@ 100174f8     AccessBridgeJavaEntryPoints.obj
 0002:00008534       ??_C@_0CK@KNLDNGDN@?$FLWARN?$FN?3?5?5?5Accessible?5Text?5lette@ 10017534     AccessBridgeJavaEntryPoints.obj
 0002:00008560       ??_C@_0EN@GBFAECFE@?$FLERROR?$FN?3?5either?5env?5?$DN?$DN?50?5or?5get@ 10017560     AccessBridgeJavaEntryPoints.obj
 0002:000085b0       ??_C@_0DI@DFJMLOME@Getting?5AccessibleWordAtIndex?5?9@ 100175b0     AccessBridgeJavaEntryPoints.obj
 0002:000085e8       ??_C@_0DJ@OIDPECCJ@Getting?5AccessibleWordAtIndex?5?9@ 100175e8     AccessBridgeJavaEntryPoints.obj
 0002:00008624       ??_C@_0DK@MPAFOPBO@Getting?5AccessibleWordAtIndex?5?9@ 10017624     AccessBridgeJavaEntryPoints.obj
 0002:00008660       ??_C@_0DN@BHAGMCIL@Getting?5AccessibleWordAtIndex?5?9@ 10017660     AccessBridgeJavaEntryPoints.obj
 0002:000086a0       ??_C@_0DJ@JFBBPAAF@Getting?5AccessibleWordAtIndex?5?9@ 100176a0     AccessBridgeJavaEntryPoints.obj
 0002:000086e0       ??_C@_1EK@ODCBDMFL@?$AA?$FL?$AAI?$AAN?$AAF?$AAO?$AA?$FN?$AA?3?$AA?5?$AA?5?$AA?5?$AAA?$AAc?$AAc?$AAe?$AAs@ 100176e0     AccessBridgeJavaEntryPoints.obj
 0002:0000872c       ??_C@_0DJ@CGMKIALH@Getting?5AccessibleWordAtIndex?5?9@ 1001772c     AccessBridgeJavaEntryPoints.obj
 0002:00008768       ??_C@_0CI@JLGHFNHI@?$FLWARN?$FN?3?5?5?5Accessible?5Text?5word?5@ 10017768     AccessBridgeJavaEntryPoints.obj
 0002:00008790       ??_C@_0EL@NKGFFDIO@?$FLERROR?$FN?3?5either?5env?5?$DN?$DN?50?5or?5get@ 10017790     AccessBridgeJavaEntryPoints.obj
 0002:000087dc       ??_C@_0DP@OGFHHBKC@Getting?5AccessibleSentenceAtInd@ 100177dc     AccessBridgeJavaEntryPoints.obj
 0002:0000881c       ??_C@_0DN@MGFPCBII@Getting?5AccessibleSentenceAtInd@ 1001781c     AccessBridgeJavaEntryPoints.obj
 0002:0000885c       ??_C@_0DO@GOPKBMAD@Getting?5AccessibleSentenceAtInd@ 1001785c     AccessBridgeJavaEntryPoints.obj
 0002:000088a0       ??_C@_0EB@BBGLKPPK@Getting?5AccessibleSentenceAtInd@ 100178a0     AccessBridgeJavaEntryPoints.obj
 0002:000088e4       ??_C@_0DN@LLHBJDKE@Getting?5AccessibleSentenceAtInd@ 100178e4     AccessBridgeJavaEntryPoints.obj
 0002:00008928       ??_C@_1FC@FOIECOHK@?$AA?$FL?$AAI?$AAN?$AAF?$AAO?$AA?$FN?$AA?3?$AA?5?$AA?5?$AA?5?$AAA?$AAc?$AAc?$AAe?$AAs@ 10017928     AccessBridgeJavaEntryPoints.obj
 0002:0000897c       ??_C@_0DN@IKKODBG@Getting?5AccessibleSentenceAtInd@ 1001797c     AccessBridgeJavaEntryPoints.obj
 0002:000089bc       ??_C@_0CM@EBOEJDBD@?$FLWARN?$FN?3?5?5?5Accessible?5Text?5sente@ 100179bc     AccessBridgeJavaEntryPoints.obj
 0002:000089e8       ??_C@_0EP@JMGAHICJ@?$FLERROR?$FN?3?5either?5env?5?$DN?$DN?50?5or?5get@ 100179e8     AccessBridgeJavaEntryPoints.obj
 0002:00008a38       ??_C@_0FB@DGBDAMEN@?$FLINFO?$FN?3?5Calling?5AccessBridgeJav@ 10017a38     AccessBridgeJavaEntryPoints.obj
 0002:00008a8c       ??_C@_0DP@BBIGIAAH@Getting?5AccessibleTextSelection@ 10017a8c     AccessBridgeJavaEntryPoints.obj
 0002:00008acc       ??_C@_0BP@MPEDAFPO@?$FLINFO?$FN?3?5?5?5Selection?5start?5?$DN?5?$CFd@ 10017acc     AccessBridgeJavaEntryPoints.obj
 0002:00008af0       ??_C@_0FD@EDCFOMDB@?$FLERROR?$FN?3?5?5either?5env?5?$DN?$DN?50?5or?5ge@ 10017af0     AccessBridgeJavaEntryPoints.obj
 0002:00008b44       ??_C@_0DN@MBOJJHKP@Getting?5AccessibleTextSelection@ 10017b44     AccessBridgeJavaEntryPoints.obj
 0002:00008b84       ??_C@_0BN@JAKAFPAN@?$FLINFO?$FN?3?5?5?5Selection?5end?5?$DN?5?$CFd@ 10017b84     AccessBridgeJavaEntryPoints.obj
 0002:00008ba8       ??_C@_0FA@HPMPKGDO@?$FLERROR?$FN?3?5either?5env?5?$DN?$DN?50?5or?5get@ 10017ba8     AccessBridgeJavaEntryPoints.obj
 0002:00008bf8       ??_C@_0EA@KGAPFINL@Getting?5AccessibleTextSelectedT@ 10017bf8     AccessBridgeJavaEntryPoints.obj
 0002:00008c38       ??_C@_0DO@OMODBJBJ@Getting?5AccessibleTextSelectedT@ 10017c38     AccessBridgeJavaEntryPoints.obj
 0002:00008c78       ??_C@_0DP@OJNIADOJ@Getting?5AccessibleTextSelectedT@ 10017c78     AccessBridgeJavaEntryPoints.obj
 0002:00008cb8       ??_C@_0EC@KNCELFHB@Getting?5AccessibleTextSelectedT@ 10017cb8     AccessBridgeJavaEntryPoints.obj
 0002:00008cfc       ??_C@_0DO@JBMNKLDF@Getting?5AccessibleTextSelectedT@ 10017cfc     AccessBridgeJavaEntryPoints.obj
 0002:00008d3c       ??_C@_0CK@DDDAABEG@?$FLINFO?$FN?3?5?5?5Accessible?8s?5selected@ 10017d3c     AccessBridgeJavaEntryPoints.obj
 0002:00008d68       ??_C@_0DO@CCBGNLIH@Getting?5AccessibleTextSelectedT@ 10017d68     AccessBridgeJavaEntryPoints.obj
 0002:00008da8       ??_C@_0CO@GAOLMCL@?$FLWARN?$FN?3?5?5?5Accessible?8s?5selected@ 10017da8     AccessBridgeJavaEntryPoints.obj
 0002:00008dd8       ??_C@_0EP@FNBFNNLO@?$FLWARN?$FN?3?5either?5env?5?$DN?$DN?50?5or?5getA@ 10017dd8     AccessBridgeJavaEntryPoints.obj
 0002:00008e28       ??_C@_0EO@HEMIPALC@?$FLINFO?$FN?3?5Calling?5AccessBridgeJav@ 10017e28     AccessBridgeJavaEntryPoints.obj
 0002:00008e78       ??_C@_0CK@OGCGGLCF@?$FLINFO?$FN?3?5?5Getting?5AttributeSet?5a@ 10017e78     AccessBridgeJavaEntryPoints.obj
 0002:00008ea8       ??_C@_0ED@CGONELLD@Getting?5AccessibleAttributeSetA@ 10017ea8     AccessBridgeJavaEntryPoints.obj
 0002:00008ef0       ??_C@_0FD@BNPBOBD@?$FLERROR?$FN?3?5either?5env?5?$DN?$DN?50?5or?5get@ 10017ef0     AccessBridgeJavaEntryPoints.obj
 0002:00008f48       ??_C@_0FG@OPHHFMC@?$FLWARN?$FN?3?5?5AttributeSet?5returned?5@ 10017f48     AccessBridgeJavaEntryPoints.obj
 0002:00008fa0       ??_C@_0CL@BFGDEBIA@?$FLINFO?$FN?3?5?5Getting?5bold?5from?5Attr@ 10017fa0     AccessBridgeJavaEntryPoints.obj
 0002:00008fcc       ??_C@_0DL@NGCGOJOD@Getting?5BoldFromAttributeSet?5?9?5@ 10017fcc     AccessBridgeJavaEntryPoints.obj
 0002:00009008       ??_C@_0DP@GPLAEKHL@?$FLERROR?$FN?3?5either?5env?5?$DN?$DN?50?5or?5get@ 10018008     AccessBridgeJavaEntryPoints.obj
 0002:00009048       ??_C@_0DI@GHAHHMIG@Getting?5BoldFromAttributeSet?5?9?5@ 10018048     AccessBridgeJavaEntryPoints.obj
 0002:00009080       ??_C@_0DI@NENMAMDE@Getting?5BoldFromAttributeSet?5?9?5@ 10018080     AccessBridgeJavaEntryPoints.obj
 0002:000090b8       ??_C@_0CN@DLPNJKCI@?$FLINFO?$FN?3?5?5Getting?5italic?5from?5At@ 100180b8     AccessBridgeJavaEntryPoints.obj
 0002:000090e8       ??_C@_0DN@FALJGLGH@Getting?5ItalicFromAttributeSet?5@ 100180e8     AccessBridgeJavaEntryPoints.obj
 0002:00009128       ??_C@_0EC@PFKOONOF@?$FLERROR?$FN?3?5either?5env?5?$DN?$DN?50?5or?5get@ 10018128     AccessBridgeJavaEntryPoints.obj
 0002:0000916c       ??_C@_0DK@CEDKJPGF@Getting?5ItalicFromAttributeSet?5@ 1001816c     AccessBridgeJavaEntryPoints.obj
 0002:000091a8       ??_C@_0DK@JHOBOPNH@Getting?5ItalicFromAttributeSet?5@ 100181a8     AccessBridgeJavaEntryPoints.obj
 0002:000091e4       ??_C@_0DA@HJAHPBCP@?$FLINFO?$FN?3?5?5Getting?5underline?5from@ 100181e4     AccessBridgeJavaEntryPoints.obj
 0002:00009218       ??_C@_0EA@LFOJMIBN@Getting?5UnderlineFromAttributeS@ 10018218     AccessBridgeJavaEntryPoints.obj
 0002:00009258       ??_C@_0EF@LMCHMLNC@?$FLERROR?$FN?3?5?5either?5env?5?$DN?$DN?50?5or?5ge@ 10018258     AccessBridgeJavaEntryPoints.obj
 0002:000092a0       ??_C@_0DN@GEOGGPCN@Getting?5UnderlineFromAttributeS@ 100182a0     AccessBridgeJavaEntryPoints.obj
 0002:000092e0       ??_C@_0DN@NHDNBPJP@Getting?5UnderlineFromAttributeS@ 100182e0     AccessBridgeJavaEntryPoints.obj
 0002:00009320       ??_C@_0DE@MIAPKOHI@?$FLINFO?$FN?3?5?5Getting?5strikethrough?5@ 10018320     AccessBridgeJavaEntryPoints.obj
 0002:00009358       ??_C@_0EE@DDJIBELI@Getting?5StrikethroughFromAttrib@ 10018358     AccessBridgeJavaEntryPoints.obj
 0002:000093a0       ??_C@_0EI@HMMOGEKC@?$FLERROR?$FN?3?5either?5env?5?$DN?$DN?50?5or?5get@ 100183a0     AccessBridgeJavaEntryPoints.obj
 0002:000093e8       ??_C@_0EB@GCIGLCLO@Getting?5StrikethroughFromAttrib@ 100183e8     AccessBridgeJavaEntryPoints.obj
 0002:00009430       ??_C@_0EB@NBFNMCAM@Getting?5StrikethroughFromAttrib@ 10018430     AccessBridgeJavaEntryPoints.obj
 0002:00009474       ??_C@_0DC@ENJFOBHI@?$FLINFO?$FN?3?5?5Getting?5superscript?5fr@ 10018474     AccessBridgeJavaEntryPoints.obj
 0002:000094a8       ??_C@_0EC@BAJDPNIO@Getting?5SuperscriptFromAttribut@ 100184a8     AccessBridgeJavaEntryPoints.obj
 0002:000094f0       ??_C@_0EH@EIIKEOA@?$FLERROR?$FN?3?5either?5env?5?$DN?$DN?50?5or?5get@ 100184f0     AccessBridgeJavaEntryPoints.obj
 0002:00009538       ??_C@_0DP@LNAJFDKJ@Getting?5SuperscriptFromAttribut@ 10018538     AccessBridgeJavaEntryPoints.obj
 0002:00009578       ??_C@_0DP@ONCCDBL@Getting?5SuperscriptFromAttribut@ 10018578     AccessBridgeJavaEntryPoints.obj
 0002:000095b8       ??_C@_0DA@KLOJONPP@?$FLINFO?$FN?3?5?5Getting?5subscript?5from@ 100185b8     AccessBridgeJavaEntryPoints.obj
 0002:000095e8       ??_C@_0EA@NMFFGPLI@Getting?5SubscriptFromAttributeS@ 100185e8     AccessBridgeJavaEntryPoints.obj
 0002:00009628       ??_C@_0EE@EGHOMMOM@?$FLERROR?$FN?3?5either?5env?5?$DN?$DN?50?5or?5get@ 10018628     AccessBridgeJavaEntryPoints.obj
 0002:0000966c       ??_C@_0DN@NJLPKKJA@Getting?5SubscriptFromAttributeS@ 1001866c     AccessBridgeJavaEntryPoints.obj
 0002:000096ac       ??_C@_0DN@GKGENKCC@Getting?5SubscriptFromAttributeS@ 100186ac     AccessBridgeJavaEntryPoints.obj
 0002:000096ec       ??_C@_0DG@JDMMILDN@?$FLINFO?$FN?3?5?5Getting?5backgroundColo@ 100186ec     AccessBridgeJavaEntryPoints.obj
 0002:00009728       ??_C@_0EF@CPKEHGFF@Getting?5BackgroundColorFromAttr@ 10018728     AccessBridgeJavaEntryPoints.obj
 0002:00009770       ??_C@_0ED@OOEECCFB@Getting?5BackgroundColorFromAttr@ 10018770     AccessBridgeJavaEntryPoints.obj
 0002:000097b8       ??_C@_0EE@JBNNGNHA@Getting?5BackgroundColorFromAttr@ 100187b8     AccessBridgeJavaEntryPoints.obj
 0002:00009800       ??_C@_0EH@NEPCIENA@Getting?5BackgroundColorFromAttr@ 10018800     AccessBridgeJavaEntryPoints.obj
 0002:00009848       ??_C@_0ED@JDGKJAHN@Getting?5BackgroundColorFromAttr@ 10018848     AccessBridgeJavaEntryPoints.obj
 0002:00009890       ??_C@_1GA@PMLMKIMP@?$AA?$FL?$AAI?$AAN?$AAF?$AAO?$AA?$FN?$AA?3?$AA?5?$AA?5?$AA?5?$AAA?$AAt?$AAt?$AAr?$AAi@ 10018890     AccessBridgeJavaEntryPoints.obj
 0002:000098f0       ??_C@_0ED@CALBOAMP@Getting?5BackgroundColorFromAttr@ 100188f0     AccessBridgeJavaEntryPoints.obj
 0002:00009934       ??_C@_0DD@DIMBBLFG@?$FLWARN?$FN?3?5?5?5AttributeSet?8s?5backgr@ 10018934     AccessBridgeJavaEntryPoints.obj
 0002:00009968       ??_C@_0EK@LDLFAHLP@?$FLERROR?$FN?3?5either?5env?5?$DN?$DN?50?5or?5get@ 10018968     AccessBridgeJavaEntryPoints.obj
 0002:000099b4       ??_C@_0DG@OAPFKBJG@?$FLINFO?$FN?3?5?5Getting?5foregroundColo@ 100189b4     AccessBridgeJavaEntryPoints.obj
 0002:000099f0       ??_C@_0EF@CFMCBGOA@Getting?5ForegroundColorFromAttr@ 100189f0     AccessBridgeJavaEntryPoints.obj
 0002:00009a38       ??_C@_0ED@CGONGGIL@Getting?5ForegroundColorFromAttr@ 10018a38     AccessBridgeJavaEntryPoints.obj
 0002:00009a80       ??_C@_0EE@PHBDPPPO@Getting?5ForegroundColorFromAttr@ 10018a80     AccessBridgeJavaEntryPoints.obj
 0002:00009ac8       ??_C@_0EH@PCLFBD@Getting?5ForegroundColorFromAttr@ 10018ac8     AccessBridgeJavaEntryPoints.obj
 0002:00009b10       ??_C@_0ED@FLMDNEKH@Getting?5ForegroundColorFromAttr@ 10018b10     AccessBridgeJavaEntryPoints.obj
 0002:00009b58       ??_C@_1GA@DDCOJJLA@?$AA?$FL?$AAI?$AAN?$AAF?$AAO?$AA?$FN?$AA?3?$AA?5?$AA?5?$AA?5?$AAA?$AAt?$AAt?$AAr?$AAi@ 10018b58     AccessBridgeJavaEntryPoints.obj
 0002:00009bb8       ??_C@_0ED@OIBIKEBF@Getting?5ForegroundColorFromAttr@ 10018bb8     AccessBridgeJavaEntryPoints.obj
 0002:00009bfc       ??_C@_0DD@EGLIFJNP@?$FLWARN?$FN?3?5?5?5AttributeSet?8s?5foregr@ 10018bfc     AccessBridgeJavaEntryPoints.obj
 0002:00009c30       ??_C@_0EK@JAILLABF@?$FLERROR?$FN?3?5either?5env?5?$DN?$DN?50?5or?5get@ 10018c30     AccessBridgeJavaEntryPoints.obj
 0002:00009c7c       ??_C@_0DB@NPCHLNMB@?$FLINFO?$FN?3?5?5Getting?5fontFamily?5fro@ 10018c7c     AccessBridgeJavaEntryPoints.obj
 0002:00009cb0       ??_C@_0EA@OFLFMJOA@Getting?5FontFamilyFromAttribute@ 10018cb0     AccessBridgeJavaEntryPoints.obj
 0002:00009cf0       ??_C@_0DO@ECEGIKHO@Getting?5FontFamilyFromAttribute@ 10018cf0     AccessBridgeJavaEntryPoints.obj
 0002:00009d30       ??_C@_0DP@DKKAFCIB@Getting?5FontFamilyFromAttribute@ 10018d30     AccessBridgeJavaEntryPoints.obj
 0002:00009d70       ??_C@_0EC@BGJOLKCB@Getting?5FontFamilyFromAttribute@ 10018d70     AccessBridgeJavaEntryPoints.obj
 0002:00009db4       ??_C@_0DO@DPGIDIFC@Getting?5FontFamilyFromAttribute@ 10018db4     AccessBridgeJavaEntryPoints.obj
 0002:00009df8       ??_C@_1FE@LCMANMIC@?$AA?$FL?$AAI?$AAN?$AAF?$AAO?$AA?$FN?$AA?3?$AA?5?$AA?5?$AA?5?$AAA?$AAt?$AAt?$AAr?$AAi@ 10018df8     AccessBridgeJavaEntryPoints.obj
 0002:00009e4c       ??_C@_0DO@IMLDEIOA@Getting?5FontFamilyFromAttribute@ 10018e4c     AccessBridgeJavaEntryPoints.obj
 0002:00009e8c       ??_C@_0CN@DFPIBNDO@?$FLWARN?$FN?3?5?5?5AttributeSet?8s?5fontFa@ 10018e8c     AccessBridgeJavaEntryPoints.obj
 0002:00009ec0       ??_C@_0EF@MEIJBCDI@?$FLERROR?$FN?3?5either?5env?5?$DN?$DN?50?5or?5get@ 10018ec0     AccessBridgeJavaEntryPoints.obj
 0002:00009f08       ??_C@_0DA@NKBCCHCB@?$FLINFO?$FN?3?5?5Getting?5font?5size?5from@ 10018f08     AccessBridgeJavaEntryPoints.obj
 0002:00009f38       ??_C@_0DL@OGKGFGCH@Getting?5FontSizeFromAttributeSe@ 10018f38     AccessBridgeJavaEntryPoints.obj
 0002:00009f74       ??_C@_0CI@MMDBDPDB@?$FLINFO?$FN?3?5?5?5AttributeSet?8s?5font?5s@ 10018f74     AccessBridgeJavaEntryPoints.obj
 0002:00009fa0       ??_C@_0EE@EGBGOKJP@?$FLERROR?$FN?3?5either?5env?5?$DN?$DN?50?5or?5get@ 10018fa0     AccessBridgeJavaEntryPoints.obj
 0002:00009fe4       ??_C@_0DM@KMMBHJCP@Getting?5FontSizeFromAttributeSe@ 10018fe4     AccessBridgeJavaEntryPoints.obj
 0002:0000a020       ??_C@_0DM@BPBKAJJN@Getting?5FontSizeFromAttributeSe@ 10019020     AccessBridgeJavaEntryPoints.obj
 0002:0000a05c       ??_C@_0CI@DPJLKBCH@?5Getting?5alignment?5from?5Attribu@ 1001905c     AccessBridgeJavaEntryPoints.obj
 0002:0000a084       ??_C@_0DM@IEKBPPGN@Getting?5AlignmentFromAttributeS@ 10019084     AccessBridgeJavaEntryPoints.obj
 0002:0000a0c0       ??_C@_0DN@DKKKNGAI@Getting?5AlignmentFromAttributeS@ 100190c0     AccessBridgeJavaEntryPoints.obj
 0002:0000a100       ??_C@_0DN@IJHBKGLK@Getting?5AlignmentFromAttributeS@ 10019100     AccessBridgeJavaEntryPoints.obj
 0002:0000a140       ??_C@_0DA@IEHDNKCA@?$FLINFO?$FN?3?5?5Getting?5bidiLevel?5from@ 10019140     AccessBridgeJavaEntryPoints.obj
 0002:0000a170       ??_C@_0DM@HHHEIBLO@Getting?5BidiLevelFromAttributeS@ 10019170     AccessBridgeJavaEntryPoints.obj
 0002:0000a1b0       ??_C@_0EE@FHPLAGJN@?$FLERROR?$FN?3?5either?5env?5?$DN?$DN?50?5or?5get@ 100191b0     AccessBridgeJavaEntryPoints.obj
 0002:0000a1f4       ??_C@_0DN@CFIDIABI@Getting?5BidiLevelFromAttributeS@ 100191f4     AccessBridgeJavaEntryPoints.obj
 0002:0000a234       ??_C@_0DN@JGFIPAKK@Getting?5BidiLevelFromAttributeS@ 10019234     AccessBridgeJavaEntryPoints.obj
 0002:0000a274       ??_C@_0DH@CAJPMJAH@?$FLERROR?$FN?3?5?5Getting?5firstLineInde@ 10019274     AccessBridgeJavaEntryPoints.obj
 0002:0000a2b0       ??_C@_0EC@GDNCLBBP@Getting?5FirstLineIndentFromAttr@ 100192b0     AccessBridgeJavaEntryPoints.obj
 0002:0000a2f8       ??_C@_0EK@JNGBIMLH@?$FLERROR?$FN?3?5either?5env?5?$DN?$DN?50?5or?5get@ 100192f8     AccessBridgeJavaEntryPoints.obj
 0002:0000a348       ??_C@_0ED@IEEGLFFG@Getting?5FirstLineIndentFromAttr@ 10019348     AccessBridgeJavaEntryPoints.obj
 0002:0000a390       ??_C@_0ED@DHJNMFOE@Getting?5FirstLineIndentFromAttr@ 10019390     AccessBridgeJavaEntryPoints.obj
 0002:0000a3d4       ??_C@_0DB@GIKOBABF@?$FLINFO?$FN?3?5?5Getting?5leftIndent?5fro@ 100193d4     AccessBridgeJavaEntryPoints.obj
 0002:0000a408       ??_C@_0DN@GGPJCLGF@Getting?5LeftIndentFromAttribute@ 10019408     AccessBridgeJavaEntryPoints.obj
 0002:0000a448       ??_C@_0EF@JFNBAGAC@?$FLERROR?$FN?3?5either?5env?5?$DN?$DN?50?5or?5get@ 10019448     AccessBridgeJavaEntryPoints.obj
 0002:0000a490       ??_C@_0DO@DEJDAGOO@Getting?5LeftIndentFromAttribute@ 10019490     AccessBridgeJavaEntryPoints.obj
 0002:0000a4d0       ??_C@_0DO@IHEIHGFM@Getting?5LeftIndentFromAttribute@ 100194d0     AccessBridgeJavaEntryPoints.obj
 0002:0000a510       ??_C@_0DC@OHJHAPPB@?$FLINFO?$FN?3?5?5Getting?5rightIndent?5fr@ 10019510     AccessBridgeJavaEntryPoints.obj
 0002:0000a544       ??_C@_0DO@GPANPNCO@Getting?5RightIndentFromAttribut@ 10019544     AccessBridgeJavaEntryPoints.obj
 0002:0000a588       ??_C@_0EG@FKGIOCMJ@?$FLERROR?$FN?3?5either?5env?5?$DN?$DN?50?5or?5get@ 10019588     AccessBridgeJavaEntryPoints.obj
 0002:0000a5d0       ??_C@_0DP@NFJEGKCA@Getting?5RightIndentFromAttribut@ 100195d0     AccessBridgeJavaEntryPoints.obj
 0002:0000a610       ??_C@_0DP@GGEPBKJC@Getting?5RightIndentFromAttribut@ 10019610     AccessBridgeJavaEntryPoints.obj
 0002:0000a650       ??_C@_0DC@FBCMPKE@?$FLINFO?$FN?3?5?5Getting?5lineSpacing?5fr@ 10019650     AccessBridgeJavaEntryPoints.obj
 0002:0000a684       ??_C@_0DO@OLMNNFJE@Getting?5LineSpacingFromAttribut@ 10019684     AccessBridgeJavaEntryPoints.obj
 0002:0000a6c8       ??_C@_0EH@DJGGHDHL@?$FLERROR?$FN?3?5?5either?5env?5?$DN?$DN?50?5or?5ge@ 100196c8     AccessBridgeJavaEntryPoints.obj
 0002:0000a710       ??_C@_0DP@POKEPAJK@Getting?5LineSpacingFromAttribut@ 10019710     AccessBridgeJavaEntryPoints.obj
 0002:0000a750       ??_C@_0DP@ENHPIACI@Getting?5LineSpacingFromAttribut@ 10019750     AccessBridgeJavaEntryPoints.obj
 0002:0000a790       ??_C@_0DB@BBFBINOC@?$FLINFO?$FN?3?5?5Getting?5spaceAbove?5fro@ 10019790     AccessBridgeJavaEntryPoints.obj
 0002:0000a7c4       ??_C@_0DN@LICNMEPC@Getting?5SpaceAboveFromAttribute@ 100197c4     AccessBridgeJavaEntryPoints.obj
 0002:0000a808       ??_C@_0EG@DEAABEIJ@?$FLERROR?$FN?3?5?5either?5env?5?$DN?$DN?50?5or?5ge@ 10019808     AccessBridgeJavaEntryPoints.obj
 0002:0000a850       ??_C@_0DO@FKCGNEOG@Getting?5SpaceAboveFromAttribute@ 10019850     AccessBridgeJavaEntryPoints.obj
 0002:0000a890       ??_C@_0DO@OJPNKEFE@Getting?5SpaceAboveFromAttribute@ 10019890     AccessBridgeJavaEntryPoints.obj
 0002:0000a8d0       ??_C@_0DB@IPEMBOFF@?$FLINFO?$FN?3?5?5Getting?5spaceBelow?5fro@ 100198d0     AccessBridgeJavaEntryPoints.obj
 0002:0000a904       ??_C@_0DN@KGEHENNL@Getting?5SpaceBelowFromAttribute@ 10019904     AccessBridgeJavaEntryPoints.obj
 0002:0000a948       ??_C@_0EG@PAJHHADM@?$FLERROR?$FN?3?5?5either?5env?5?$DN?$DN?50?5or?5ge@ 10019948     AccessBridgeJavaEntryPoints.obj
 0002:0000a990       ??_C@_0DO@BIIKCGAD@Getting?5SpaceBelowFromAttribute@ 10019990     AccessBridgeJavaEntryPoints.obj
 0002:0000a9d0       ??_C@_0DO@KLFBFGLB@Getting?5SpaceBelowFromAttribute@ 100199d0     AccessBridgeJavaEntryPoints.obj
 0002:0000aa10       ??_C@_0DD@NEPODHGJ@?$FLINFO?$FN?3?5?5Decrementing?5reference@ 10019a10     AccessBridgeJavaEntryPoints.obj
 0002:0000aa44       ??_C@_0DJ@KDCCLHCF@Releasing?5AttributeSet?5object?5?9@ 10019a44     AccessBridgeJavaEntryPoints.obj
 0002:0000aa80       ??_C@_0DF@KOJHMOGM@?$FLERROR?$FN?3?5?5either?5env?5?$DN?$DN?50?5or?5ac@ 10019a80     AccessBridgeJavaEntryPoints.obj
 0002:0000aab8       ??_C@_0DJ@BAPJMHJH@Releasing?5AttributeSet?5object?5?9@ 10019ab8     AccessBridgeJavaEntryPoints.obj
 0002:0000aaf4       ??_C@_0DI@FAAGAOKI@?$FLINFO?$FN?3?5?5Getting?5full?5attribute@ 10019af4     AccessBridgeJavaEntryPoints.obj
 0002:0000ab2c       ??_C@_0DD@BPFGOEDD@?$FLINFO?$FN?3?5?5returned?5from?5CallObje@ 10019b2c     AccessBridgeJavaEntryPoints.obj
 0002:0000ab60       ??_C@_1FG@IBEGPOLG@?$AA?$FL?$AAI?$AAN?$AAF?$AAO?$AA?$FN?$AA?3?$AA?5?$AA?5?$AA?5?$AAA?$AAc?$AAc?$AAe?$AAs@ 10019b60     AccessBridgeJavaEntryPoints.obj
 0002:0000abb8       ??_C@_0FC@NKKMDLMK@?$FLERROR?$FN?3?5?5either?5env?5?$DN?$DN?50?5or?5ge@ 10019bb8     AccessBridgeJavaEntryPoints.obj
 0002:0000ac10       ??_C@_0EB@FOBGJMBG@Getting?5AccessibleAttributeSetA@ 10019c10     AccessBridgeJavaEntryPoints.obj
 0002:0000ac58       ??_C@_0FD@ONBHOKNL@?$FLINFO?$FN?3?5Calling?5AccessBridgeJav@ 10019c58     AccessBridgeJavaEntryPoints.obj
 0002:0000acac       ??_C@_0DL@PJLLEMMJ@Getting?5AccessibleXcoordTextRec@ 10019cac     AccessBridgeJavaEntryPoints.obj
 0002:0000ace8       ??_C@_0BG@CDBEIJEJ@?$FLINFO?$FN?3?5?5X?5coord?5?$DN?5?$CFd@ 10019ce8     AccessBridgeJavaEntryPoints.obj
 0002:0000ad00       ??_C@_0FF@CICHONC@?$FLERROR?$FN?3?5either?5env?5?$DN?$DN?50?5or?5get@ 10019d00     AccessBridgeJavaEntryPoints.obj
 0002:0000ad58       ??_C@_0DL@BBKMNMGI@Getting?5AccessibleYcoordTextRec@ 10019d58     AccessBridgeJavaEntryPoints.obj
 0002:0000ad98       ??_C@_0FF@LPGHAKKN@?$FLINFO?$FN?3?5?5either?5env?5?$DN?$DN?50?5or?5get@ 10019d98     AccessBridgeJavaEntryPoints.obj
 0002:0000adf0       ??_C@_0DK@GOMAAIJJ@Getting?5AccessibleWidthTextRect@ 10019df0     AccessBridgeJavaEntryPoints.obj
 0002:0000ae2c       ??_C@_0BD@PFFPBFHC@?$FLINFO?$FN?3?5Width?5?$DN?5?$CFd@ 10019e2c     AccessBridgeJavaEntryPoints.obj
 0002:0000ae40       ??_C@_0FD@LFKJAPPJ@?$FLINFO?$FN?3?5either?5env?5?$DN?$DN?50?5or?5getA@ 10019e40     AccessBridgeJavaEntryPoints.obj
 0002:0000ae94       ??_C@_0DL@LIFPGLAA@Getting?5AccessibleHeightTextRec@ 10019e94     AccessBridgeJavaEntryPoints.obj
 0002:0000aed0       ??_C@_0BE@BNGOGMPP@?$FLINFO?$FN?3?5Height?5?$DN?5?$CFd@ 10019ed0     AccessBridgeJavaEntryPoints.obj
 0002:0000aee8       ??_C@_0FG@JCNMAPKJ@?$FLERROR?$FN?3?5?5either?5env?5?$DN?$DN?50?5or?5ge@ 10019ee8     AccessBridgeJavaEntryPoints.obj
 0002:0000af40       ??_C@_0EO@GAEGCFMP@?$FLINFO?$FN?3?5Calling?5AccessBridgeJav@ 10019f40     AccessBridgeJavaEntryPoints.obj
 0002:0000af90       ??_C@_0DF@JPKJOLBB@Getting?5caret?5X?5coordinate?5?9?5ca@ 10019f90     AccessBridgeJavaEntryPoints.obj
 0002:0000afc8       ??_C@_0DK@INHGMNIG@?$FLERROR?$FN?3?5?5either?5env?5?$DN?$DN?50?5or?5ge@ 10019fc8     AccessBridgeJavaEntryPoints.obj
 0002:0000b004       ??_C@_0DF@NBCAOALI@Getting?5caret?5Y?5coordinate?5?9?5ca@ 1001a004     AccessBridgeJavaEntryPoints.obj
 0002:0000b03c       ??_C@_0DK@FAOABEAD@?$FLERROR?$FN?3?5?5either?5env?5?$DN?$DN?50?5or?5ge@ 1001a03c     AccessBridgeJavaEntryPoints.obj
 0002:0000b078       ??_C@_0CO@LPKJFNHN@Getting?5caret?5width?5?9?5call?5to?5C@ 1001a078     AccessBridgeJavaEntryPoints.obj
 0002:0000b0a8       ??_C@_0DO@KCIKCBGA@?$FLERROR?$FN?3?5?5either?5env?5?$DN?$DN?50?5or?5ge@ 1001a0a8     AccessBridgeJavaEntryPoints.obj
 0002:0000b0e8       ??_C@_0CP@DKBLCBME@Getting?5caret?5height?5?9?5call?5to?5@ 1001a0e8     AccessBridgeJavaEntryPoints.obj
 0002:0000b118       ??_C@_0DP@MHKONHOK@?$FLERROR?$FN?3?5?5either?5env?5?$DN?$DN?50?5or?5ge@ 1001a118     AccessBridgeJavaEntryPoints.obj
 0002:0000b158       ??_C@_0EO@OPGMODFN@?$FLINFO?$FN?3?5Calling?5AccessBridgeJav@ 1001a158     AccessBridgeJavaEntryPoints.obj
 0002:0000b1a8       ??_C@_0DP@HIDGMFDD@Getting?5AccessibleTextLineLeftB@ 1001a1a8     AccessBridgeJavaEntryPoints.obj
 0002:0000b1e8       ??_C@_0BK@INECDNLO@?$FLINFO?$FN?3?5?5?5startIndex?5?$DN?5?$CFd@ 1001a1e8     AccessBridgeJavaEntryPoints.obj
 0002:0000b208       ??_C@_0FD@BGKHJCDH@?$FLERROR?$FN?3?5?5either?5env?5?$DN?$DN?50?5or?5ge@ 1001a208     AccessBridgeJavaEntryPoints.obj
 0002:0000b260       ??_C@_0EA@OJGAJNKG@Getting?5AccessibleTextLineRight@ 1001a260     AccessBridgeJavaEntryPoints.obj
 0002:0000b2a0       ??_C@_0BI@NAKKCMDP@?$FLINFO?$FN?3?5?5?5endIndex?5?$DN?5?$CFd@ 1001a2a0     AccessBridgeJavaEntryPoints.obj
 0002:0000b2b8       ??_C@_0FE@HOJFBBNL@?$FLERROR?$FN?3?5?5either?5env?5?$DN?$DN?50?5or?5ge@ 1001a2b8     AccessBridgeJavaEntryPoints.obj
 0002:0000b310       ??_C@_0FM@PBOJPFBI@?$FLINFO?$FN?3?5Calling?5AccessBridgeJav@ 1001a310     AccessBridgeJavaEntryPoints.obj
 0002:0000b36c       ??_C@_0BH@GCPBFEO@?$FLERROR?$FN?3?5?5end?5?$DM?5start?$CB@ 1001a36c     AccessBridgeJavaEntryPoints.obj
 0002:0000b384       ??_C@_0DJ@OHJBLKEE@Getting?5AccessibleTextRange?5?9?5c@ 1001a384     AccessBridgeJavaEntryPoints.obj
 0002:0000b3c0       ??_C@_0DH@MLKPAEJI@Getting?5AccessibleTextRange?5?9?5c@ 1001a3c0     AccessBridgeJavaEntryPoints.obj
 0002:0000b3f8       ??_C@_1HO@MOIAIALP@?$AA?$FL?$AAI?$AAN?$AAF?$AAO?$AA?$FN?$AA?3?$AA?5?$AA?5?$AA?5?$AAA?$AAc?$AAc?$AAe?$AAs@ 1001a3f8     AccessBridgeJavaEntryPoints.obj
 0002:0000b478       ??_C@_0DB@GEMONLMO@?$FLINFO?$FN?3?5?5Accessible?5Text?5string@ 1001a478     AccessBridgeJavaEntryPoints.obj
 0002:0000b4b0       ??_C@_1HM@KJDBDPH@?$AA?$FL?$AAI?$AAN?$AAF?$AAO?$AA?$FN?$AA?3?$AA?5?$AA?5?$AA?5?$AAA?$AAc?$AAc?$AAe?$AAs@ 1001a4b0     AccessBridgeJavaEntryPoints.obj
 0002:0000b52c       ??_C@_0DI@HDEAPMEC@Getting?5AccessibleTextRange?5?9?5c@ 1001a52c     AccessBridgeJavaEntryPoints.obj
 0002:0000b564       ??_C@_0DL@BFPJOBGO@Getting?5AccessibleTextRange?5?9?5c@ 1001a564     AccessBridgeJavaEntryPoints.obj
 0002:0000b5a0       ??_C@_0DH@LGIBLGLE@Getting?5AccessibleTextRange?5?9?5c@ 1001a5a0     AccessBridgeJavaEntryPoints.obj
 0002:0000b5d8       ??_C@_1EM@MAOOPBBK@?$AA?$FL?$AAI?$AAN?$AAF?$AAO?$AA?$FN?$AA?3?$AA?5?$AA?5?$AA?5?$AAA?$AAc?$AAc?$AAe?$AAs@ 1001a5d8     AccessBridgeJavaEntryPoints.obj
 0002:0000b624       ??_C@_0DH@FFKMGAG@Getting?5AccessibleTextRange?5?9?5c@ 1001a624     AccessBridgeJavaEntryPoints.obj
 0002:0000b65c       ??_C@_0DB@ENPGLEMN@?$FLWARN?$FN?3?5?5?5current?5Accessible?5Te@ 1001a65c     AccessBridgeJavaEntryPoints.obj
 0002:0000b690       ??_C@_0EJ@IGDKNKCL@?$FLERROR?$FN?3?5either?5env?5?$DN?$DN?50?5or?5get@ 1001a690     AccessBridgeJavaEntryPoints.obj
 0002:0000b6e0       ??_C@_0FH@DFGPJEBI@?$FLINFO?$FN?3?5Calling?5AccessBridgeJav@ 1001a6e0     AccessBridgeJavaEntryPoints.obj
 0002:0000b738       ??_C@_0DM@FMEJNEAF@Getting?5CurrentAccessibleValue?5@ 1001a738     AccessBridgeJavaEntryPoints.obj
 0002:0000b774       ??_C@_0DK@DEBJEKPP@Getting?5CurrentAccessibleValue?5@ 1001a774     AccessBridgeJavaEntryPoints.obj
 0002:0000b7b0       ??_C@_0DL@KAGJLOPH@Getting?5CurrentAccessibleValue?5@ 1001a7b0     AccessBridgeJavaEntryPoints.obj
 0002:0000b7ec       ??_C@_0DO@FGJBGIKN@Getting?5CurrentAccessibleValue?5@ 1001a7ec     AccessBridgeJavaEntryPoints.obj
 0002:0000b82c       ??_C@_0DK@EJDHPIND@Getting?5CurrentAccessibleValue?5@ 1001a82c     AccessBridgeJavaEntryPoints.obj
 0002:0000b868       ??_C@_0CI@LHBKPIPL@?$FLINFO?$FN?3?5?5?5current?5Accessible?5Va@ 1001a868     AccessBridgeJavaEntryPoints.obj
 0002:0000b890       ??_C@_0DK@PKOMIIGB@Getting?5CurrentAccessibleValue?5@ 1001a890     AccessBridgeJavaEntryPoints.obj
 0002:0000b8cc       ??_C@_0CM@JBCHBMHL@?$FLWARN?$FN?3?5?5?5current?5Accessible?5Va@ 1001a8cc     AccessBridgeJavaEntryPoints.obj
 0002:0000b8f8       ??_C@_0EN@CEFCJCHP@?$FLERROR?$FN?3?5?5either?5env?5?$DN?$DN?50?5or?5ge@ 1001a8f8     AccessBridgeJavaEntryPoints.obj
 0002:0000b948       ??_C@_0FH@LDANAJBK@?$FLINFO?$FN?3?5Calling?5AccessBridgeJav@ 1001a948     AccessBridgeJavaEntryPoints.obj
 0002:0000b9a0       ??_C@_0DM@CNMGLEAD@Getting?5MaximumAccessibleValue?5@ 1001a9a0     AccessBridgeJavaEntryPoints.obj
 0002:0000b9dc       ??_C@_0DK@LPOBNFBI@Getting?5MaximumAccessibleValue?5@ 1001a9dc     AccessBridgeJavaEntryPoints.obj
 0002:0000ba18       ??_C@_0DL@JOIMDBLD@Getting?5MaximumAccessibleValue?5@ 1001aa18     AccessBridgeJavaEntryPoints.obj
 0002:0000ba54       ??_C@_0DO@ENHJNPPM@Getting?5MaximumAccessibleValue?5@ 1001aa54     AccessBridgeJavaEntryPoints.obj
 0002:0000ba94       ??_C@_0DK@MCMPGHDE@Getting?5MaximumAccessibleValue?5@ 1001aa94     AccessBridgeJavaEntryPoints.obj
 0002:0000bad0       ??_C@_0CI@MOLFAIEC@?$FLINFO?$FN?3?5?5?5maximum?5Accessible?5Va@ 1001aad0     AccessBridgeJavaEntryPoints.obj
 0002:0000baf8       ??_C@_0DK@HBBEBHIG@Getting?5MaximumAccessibleValue?5@ 1001aaf8     AccessBridgeJavaEntryPoints.obj
 0002:0000bb34       ??_C@_0CM@EENPAHAF@?$FLWARN?$FN?3?5?5?5maximum?5Accessible?5Va@ 1001ab34     AccessBridgeJavaEntryPoints.obj
 0002:0000bb60       ??_C@_0EM@DECMFMLP@?$FLERROR?$FN?3?5either?5env?5?$DN?$DN?50?5or?5get@ 1001ab60     AccessBridgeJavaEntryPoints.obj
 0002:0000bbb0       ??_C@_0FH@NCJCNBPB@?$FLINFO?$FN?3?5Calling?5AccessBridgeJav@ 1001abb0     AccessBridgeJavaEntryPoints.obj
 0002:0000bc08       ??_C@_0DM@EKOMNNCH@Getting?5MinimumAccessibleValue?5@ 1001ac08     AccessBridgeJavaEntryPoints.obj
 0002:0000bc44       ??_C@_0DK@POFOBDIM@Getting?5MinimumAccessibleValue?5@ 1001ac44     AccessBridgeJavaEntryPoints.obj
 0002:0000bc80       ??_C@_0DL@GJKPNJCI@Getting?5MinimumAccessibleValue?5@ 1001ac80     AccessBridgeJavaEntryPoints.obj
 0002:0000bcbc       ??_C@_0DO@IIPPIAIM@Getting?5MinimumAccessibleValue?5@ 1001acbc     AccessBridgeJavaEntryPoints.obj
 0002:0000bcfc       ??_C@_0DK@IDHAKBKA@Getting?5MinimumAccessibleValue?5@ 1001acfc     AccessBridgeJavaEntryPoints.obj
 0002:0000bd38       ??_C@_0CI@HMFEBFFJ@?$FLINFO?$FN?3?5?5?5mimimum?5Accessible?5Va@ 1001ad38     AccessBridgeJavaEntryPoints.obj
 0002:0000bd60       ??_C@_0DK@DAKLNBBC@Getting?5MinimumAccessibleValue?5@ 1001ad60     AccessBridgeJavaEntryPoints.obj
 0002:0000bd9c       ??_C@_0CM@LFDDPHLF@?$FLWARN?$FN?3?5?5?5mimimum?5Accessible?5Va@ 1001ad9c     AccessBridgeJavaEntryPoints.obj
 0002:0000bdc8       ??_C@_0EM@FNBMNDID@?$FLERROR?$FN?3?5either?5env?5?$DN?$DN?50?5or?5get@ 1001adc8     AccessBridgeJavaEntryPoints.obj
 0002:0000be18       ??_C@_0FE@GLAEHJLA@?$FLINFO?$FN?3?5Calling?5AccessBridgeJav@ 1001ae18     AccessBridgeJavaEntryPoints.obj
 0002:0000be6c       ??_C@_0DI@HFNIIMHH@Doing?5addAccessibleSelection?5?9?5@ 1001ae6c     AccessBridgeJavaEntryPoints.obj
 0002:0000bea4       ??_C@_0CP@EBNEHGHB@?$FLERROR?$FN?3?5?$CK?$CK?$CK?5Exception?5occured?5@ 1001aea4     AccessBridgeJavaEntryPoints.obj
 0002:0000bed4       ??_C@_0CL@OKIJNCBD@?$FLINFO?$FN?3?5?5?5returned?5from?5CallObj@ 1001aed4     AccessBridgeJavaEntryPoints.obj
 0002:0000bf00       ??_C@_0EK@CMGGDKGL@?$FLERROR?$FN?3?5?5either?5env?5?$DN?$DN?50?5or?5ad@ 1001af00     AccessBridgeJavaEntryPoints.obj
 0002:0000bf50       ??_C@_0FG@JICCBONC@?$FLINFO?$FN?3?5Calling?5AccessBridgeJav@ 1001af50     AccessBridgeJavaEntryPoints.obj
 0002:0000bfa8       ??_C@_0DK@GPKPKKON@Doing?5clearAccessibleSelection?5@ 1001afa8     AccessBridgeJavaEntryPoints.obj
 0002:0000bfe8       ??_C@_0EM@NKPDGGGN@?$FLERROR?$FN?3?5?5either?5env?5?$DN?$DN?50?5or?5cl@ 1001afe8     AccessBridgeJavaEntryPoints.obj
 0002:0000c038       ??_C@_0FE@PIPHOHFI@?$FLINFO?$FN?3?5Calling?5AccessBridgeJav@ 1001b038     AccessBridgeJavaEntryPoints.obj
 0002:0000c090       ??_C@_0EA@EDHDCMHP@Getting?5AccessibleSelectionCont@ 1001b090     AccessBridgeJavaEntryPoints.obj
 0002:0000c0d0       ??_C@_0DM@IFLFNJN@Getting?5AccessibleSelectionCont@ 1001b0d0     AccessBridgeJavaEntryPoints.obj
 0002:0000c10c       ??_C@_0DO@FEBBEFGL@Getting?5AccessibleSelectionCont@ 1001b10c     AccessBridgeJavaEntryPoints.obj
 0002:0000c150       ??_C@_0FA@KGJFECGD@?$FLERROR?$FN?3?5either?5env?5?$DN?$DN?50?5or?5get@ 1001b150     AccessBridgeJavaEntryPoints.obj
 0002:0000c1a0       ??_C@_0FJ@KDCCHMFP@?$FLINFO?$FN?3?5Calling?5AccessBridgeJav@ 1001b1a0     AccessBridgeJavaEntryPoints.obj
 0002:0000c1fc       ??_C@_0DL@JPLKCOEB@Getting?5AccessibleSelectionCoun@ 1001b1fc     AccessBridgeJavaEntryPoints.obj
 0002:0000c238       ??_C@_0EO@LLPLNNDE@?$FLERROR?$FN?3?5either?5env?5?$DN?$DN?50?5or?5get@ 1001b238     AccessBridgeJavaEntryPoints.obj
 0002:0000c288       ??_C@_0FH@BEGAHKNM@?$FLINFO?$FN?3?5Calling?5AccessBridgeJav@ 1001b288     AccessBridgeJavaEntryPoints.obj
 0002:0000c2e0       ??_C@_0DO@DGOGEINB@Doing?5isAccessibleChildSelected@ 1001b2e0     AccessBridgeJavaEntryPoints.obj
 0002:0000c320       ??_C@_0EM@FIJEFPDC@?$FLERROR?$FN?3?5either?5env?5?$DN?$DN?50?5or?5isA@ 1001b320     AccessBridgeJavaEntryPoints.obj
 0002:0000c370       ??_C@_0FH@DBFJFKMJ@?$FLINFO?$FN?3?5Calling?5AccessBridgeJav@ 1001b370     AccessBridgeJavaEntryPoints.obj
 0002:0000c3c8       ??_C@_0DL@BHDCMLKI@Doing?5removeAccessibleSelection@ 1001b3c8     AccessBridgeJavaEntryPoints.obj
 0002:0000c408       ??_C@_0EN@HJFMAEOO@?$FLERROR?$FN?3?5?5either?5env?5?$DN?$DN?50?5or?5re@ 1001b408     AccessBridgeJavaEntryPoints.obj
 0002:0000c458       ??_C@_0FK@MANGNIPE@?$FLINFO?$FN?3?5Calling?5AccessBridgeJav@ 1001b458     AccessBridgeJavaEntryPoints.obj
 0002:0000c4b4       ??_C@_0DO@JHGLNKHC@Doing?5selectAllAccessibleSelect@ 1001b4b4     AccessBridgeJavaEntryPoints.obj
 0002:0000c4f8       ??_C@_0EP@JCKDPHMN@?$FLERROR?$FN?3?5either?5env?5?$DN?$DN?50?5or?5sel@ 1001b4f8     AccessBridgeJavaEntryPoints.obj
 0002:0000c548       ??_C@_0EO@IEPNANKM@?$FLINFO?$FN?3?5?5?5in?5AccessBridgeJavaEn@ 1001b548     AccessBridgeJavaEntryPoints.obj
 0002:0000c598       ??_C@_0DK@GPMPKEMH@Doing?5addJavaEventNotification?5@ 1001b598     AccessBridgeJavaEntryPoints.obj
 0002:0000c5d8       ??_C@_0EA@IOOHIHIM@?$FLERROR?$FN?3?5either?5env?5?$DN?$DN?50?5or?5add@ 1001b5d8     AccessBridgeJavaEntryPoints.obj
 0002:0000c618       ??_C@_0FA@BBNLJKAK@?$FLINFO?$FN?3?5?5in?5AccessBridgeJavaEnt@ 1001b618     AccessBridgeJavaEntryPoints.obj
 0002:0000c668       ??_C@_0DN@IBNHMLMO@Doing?5removeJavaEventNotificati@ 1001b668     AccessBridgeJavaEntryPoints.obj
 0002:0000c6a8       ??_C@_0ED@LKLPMFCD@?$FLERROR?$FN?3?5either?5env?5?$DN?$DN?50?5or?5rem@ 1001b6a8     AccessBridgeJavaEntryPoints.obj
 0002:0000c6f0       ??_C@_0FH@ICFBIMPG@?$FLINFO?$FN?3?5?5?5in?5AccessBridgeJavaEn@ 1001b6f0     AccessBridgeJavaEntryPoints.obj
 0002:0000c748       ??_C@_0FL@OCFIPKDP@?$FLINFO?$FN?3?5?5?5?5addAccessibilityEven@ 1001b748     AccessBridgeJavaEntryPoints.obj
 0002:0000c7a4       ??_C@_0DH@DNDEHAJF@Doing?5addAccessibilityEvent?5?9?5c@ 1001b7a4     AccessBridgeJavaEntryPoints.obj
 0002:0000c7e0       ??_C@_0EJ@BAMHEIMC@?$FLERROR?$FN?3?5either?5env?5?$DN?$DN?50?5or?5add@ 1001b7e0     AccessBridgeJavaEntryPoints.obj
 0002:0000c830       ??_C@_0ED@BCNEMPCF@?$FLINFO?$FN?3?5?5?5?5?5addAccessibilityEve@ 1001b830     AccessBridgeJavaEntryPoints.obj
 0002:0000c878       ??_C@_0FJ@JPJKPKP@?$FLINFO?$FN?3?5?5in?5AccessBridgeJavaEnt@ 1001b878     AccessBridgeJavaEntryPoints.obj
 0002:0000c8d4       ??_C@_0DK@KGOHAMJ@Doing?5removeAccessibilityEvent?5@ 1001b8d4     AccessBridgeJavaEntryPoints.obj
 0002:0000c910       ??_C@_0EM@MPLDCCAE@?$FLERROR?$FN?3?5either?5env?5?$DN?$DN?50?5or?5rem@ 1001b910     AccessBridgeJavaEntryPoints.obj
 0002:0000c95c       ??_C@_0BM@BIAOFPJG@AccessBridge?9FromJava?9Hello@ 1001b95c     AccessBridgeMessages.obj
 0002:0000c978       ??_C@_0BP@OELHMMDF@AccessBridge?9FromWindows?9Hello@ 1001b978     AccessBridgeMessages.obj
 0002:0000c998       ??_C@_0CN@HNEPECB@?$FLINFO?$FN?3?5JavaAccessBridge?4DLL?5ru@ 1001b998     JavaAccessBridge.obj
 0002:0000c9c8       ??_C@_0CN@OBDABACD@?$FLINFO?$FN?3?5In?5AccessBridgeDialog?5?9@ 1001b9c8     JavaAccessBridge.obj
 0002:0000c9f8       ??_C@_0DM@LEGKGBDC@?$FLINFO?$FN?3?5In?5AccessBridgeDialog?5?9@ 1001b9f8     JavaAccessBridge.obj
 0002:0000ca34       ??_C@_0DP@KFGJNONL@?$FLINFO?$FN?3?5In?5AccessBridgeDialog?5?9@ 1001ba34     JavaAccessBridge.obj
 0002:0000ca74       ??_C@_0DN@BOPHDCMF@?$FLINFO?$FN?3?5In?5AccessBridgeDialog?5?9@ 1001ba74     JavaAccessBridge.obj
 0002:0000cab8       ??_C@_0EG@LODLDNEL@?$FLINFO?$FN?3?5In?5AccessBridgeDialog?5?9@ 1001bab8     JavaAccessBridge.obj
 0002:0000cb00       ??_C@_0EE@OLIPFHDH@?$FLINFO?$FN?3?5In?5AccessBridgeDialog?5?9@ 1001bb00     JavaAccessBridge.obj
 0002:0000cb44       ??_C@_0DO@KFBCLDPM@?$FLINFO?$FN?3?5In?5AccessBridgeDialog?5?9@ 1001bb44     JavaAccessBridge.obj
 0002:0000cb88       ??_C@_0EF@PPOLOLIM@?$FLINFO?$FN?3?5In?5AccessBridgeDialog?5?9@ 1001bb88     JavaAccessBridge.obj
 0002:0000cbd0       ??_C@_0BD@BOAKDBCO@java_access_bridge@ 1001bbd0     JavaAccessBridge.obj
 0002:0000cbe4       ??_C@_0DB@JHKNDMME@?$FLINFO?$FN?3?5in?5JavaAccessBridge?3?3?$HOJ@ 1001bbe4     JavaAccessBridge.obj
 0002:0000cc18       ??_C@_0CF@DJNKIAAH@?$FLINFO?$FN?3?5?5telling?5?$CFp?5we?8re?5going@ 1001bc18     JavaAccessBridge.obj
 0002:0000cc40       ??_C@_0CP@BKDEGDJC@?$FLINFO?$FN?3?5?5finished?5telling?5ATs?5a@ 1001bc40     JavaAccessBridge.obj
 0002:0000cc70       ??_C@_0CA@EIEOEDOI@?$FLINFO?$FN?3?5?5?5finished?5deleting?5ATs@ 1001bc70     JavaAccessBridge.obj
 0002:0000cc90       ??_C@_0BP@EBFMIPOK@?$FLINFO?$FN?3?5GOODBYE?5CRUEL?5WORLD?4?4?4@ 1001bc90     JavaAccessBridge.obj
 0002:0000ccb0       ??_C@_0DB@BKKBMMIL@?$FLINFO?$FN?3?5JavaAccessBridge?3?3javaR@ 1001bcb0     JavaAccessBridge.obj
 0002:0000cce4       ??_C@_0BJ@CDAHIMFI@?$FLINFO?$FN?3?5?5?5?9?$DO?5javaVM?5?$DN?5?$CFp@ 1001bce4     JavaAccessBridge.obj
 0002:0000cd00       ??_C@_0CF@HBJLLMBP@?$FLINFO?$FN?3?5?5?9?$DO?5windowsThreadJNIEnv@ 1001bd00     JavaAccessBridge.obj
 0002:0000cd28       ??_C@_0DL@EDCIECNK@?$FLINFO?$FN?3?5?5?5all?5Java?5thread?5entry@ 1001bd28     JavaAccessBridge.obj
 0002:0000cd64       ??_C@_0DO@DHHHOLPH@?$FLINFO?$FN?3?5?5?5all?5Windows?5thread?5en@ 1001bd64     JavaAccessBridge.obj
 0002:0000cda4       ??_C@_0CF@FINMKFHO@?$FLINFO?$FN?3?5?5?5Window?5created?4?5?5HWND@ 1001bda4     JavaAccessBridge.obj
 0002:0000cdcc       ??_C@_0CG@KCHIBPOJ@?$FLERROR?$FN?3?5?5?5FAILED?5TO?5CREATE?5WIN@ 1001bdcc     JavaAccessBridge.obj
 0002:0000cdf4       ??_C@_0BJ@LMONFDOG@ACCESSBRIDGESTATUSWINDOW@ 1001bdf4     JavaAccessBridge.obj
 0002:0000ce10       ??_C@_0DG@HAJICJFK@?$FLINFO?$FN?3?5In?5JavaAccessBridge?3?3po@ 1001be10     JavaAccessBridge.obj
 0002:0000ce48       ??_C@_0CO@FLLNHCIG@?$FLINFO?$FN?3?5?5?5calling?5PostMessage?$CI?$CF@ 1001be48     JavaAccessBridge.obj
 0002:0000ce78       ??_C@_0CM@DCNJAPPO@?$FLERROR?$FN?3?5ATs?5?$DN?$DN?50?$CB?5?$CIshouldn?8t?5h@ 1001be78     JavaAccessBridge.obj
 0002:0000cea4       ??_C@_0DH@JMPJBGDF@?$FLINFO?$FN?3?5JavaAccessBridge?3?3recei@ 1001bea4     JavaAccessBridge.obj
 0002:0000cee0       ??_C@_0EB@GECAJJE@?$FLERROR?$FN?3?5?9?5ATs?5?$DN?$DN?50?5?$CIshouldn?8t?5@ 1001bee0     JavaAccessBridge.obj
 0002:0000cf24       ??_C@_0DL@FAPEODKG@?$FLERROR?$FN?3?5receiving?5memory?5packa@ 1001bf24     JavaAccessBridge.obj
 0002:0000cf60       ??_C@_0DM@MJCPMIJG@?$FLINFO?$FN?3?5Processing?5package?5sent@ 1001bf60     JavaAccessBridge.obj
 0002:0000cf9c       ??_C@_0BL@EFABEHOK@?$FLINFO?$FN?3?5?5PackageType?5?$DN?5?$CFX?3@ 1001bf9c     JavaAccessBridge.obj
 0002:0000cfb8       ??_C@_0DC@HOEDKHHL@?$FLINFO?$FN?3?5?5?5type?5?$DN?$DN?5cMemoryMapped@ 1001bfb8     JavaAccessBridge.obj
 0002:0000cff0       ??_C@_0EC@JELBKKLB@?$FLERROR?$FN?3?5?5?5?5processing?5FAILED?$CB?$CB@ 1001bff0     JavaAccessBridge.obj
 0002:0000d034       ??_C@_0CM@EGHIFACB@?$FLINFO?$FN?3?5?5?5type?5?$DN?$DN?5cReleaseJavaO@ 1001c034     JavaAccessBridge.obj
 0002:0000d060       ??_C@_0EB@PCOLNIOI@?$FLERROR?$FN?3?5?5?5processing?5FAILED?$CB?$CB?5@ 1001c060     JavaAccessBridge.obj
 0002:0000d0a4       ??_C@_0DB@HJBBLNK@?$FLINFO?$FN?3?5?5?5type?5?$DN?$DN?5cGetAccessBri@ 1001c0a4     JavaAccessBridge.obj
 0002:0000d0d8       ??_C@_0CH@OGPNINNH@?$FLINFO?$FN?3?5?5?5type?5?$DN?$DN?5cIsJavaWindow@ 1001c0d8     JavaAccessBridge.obj
 0002:0000d100       ??_C@_0CF@KCGBFLNL@?$FLINFO?$FN?3?5?5?5?5?5?9?$DO?5returning?5result@ 1001c100     JavaAccessBridge.obj
 0002:0000d128       ??_C@_0CH@FFMGBMGP@?$FLINFO?$FN?3?5?5?5type?5?$DN?$DN?5cIsSameObject@ 1001c128     JavaAccessBridge.obj
 0002:0000d150       ??_C@_0DI@FGDPIMOI@?$FLINFO?$FN?3?5?5?5?5type?5?$DN?$DN?5cGetAccessib@ 1001c150     JavaAccessBridge.obj
 0002:0000d188       ??_C@_0CN@KFALDIEC@?$FLINFO?$FN?3?5?5?5?5?5?5?9?$DO?5returning?5AC?5?$DN?5@ 1001c188     JavaAccessBridge.obj
 0002:0000d1b8       ??_C@_0DI@ICOCNDDM@?$FLINFO?$FN?3?5?5?5?5type?5?$DN?$DN?5cGetHWNDFrom@ 1001c1b8     JavaAccessBridge.obj
 0002:0000d1f0       ??_C@_0CD@DNCFKFDK@?$FLINFO?$FN?3?5?5?5?5?5?9?$DO?5returning?5HWND?5?$DN@ 1001c1f0     JavaAccessBridge.obj
 0002:0000d214       ??_C@_0CK@DBBKGOKJ@?$FLINFO?$FN?3?5?5?5type?5?$DN?$DN?5cSetTextConte@ 1001c214     JavaAccessBridge.obj
 0002:0000d240       ??_C@_0JK@BDICEONN@?$FLINFO?$FN?3?5?5?5type?5?$DN?$DN?5cGetParentWit@ 1001c240     JavaAccessBridge.obj
 0002:0000d2dc       ??_C@_0CM@FMGIHPCP@?$FLINFO?$FN?3?5?5?5type?5?$DN?$DN?5cGetTopLevelO@ 1001c2dc     JavaAccessBridge.obj
 0002:0000d308       ??_C@_0DC@EMOAFCHE@?$FLINFO?$FN?3?5?5?5?5?5?5?9?$DO?5returning?5rAcce@ 1001c308     JavaAccessBridge.obj
 0002:0000d33c       ??_C@_0DE@EHPIAHAD@?$FLINFO?$FN?3?5?5?5type?5?$DN?$DN?5cGetParentWit@ 1001c33c     JavaAccessBridge.obj
 0002:0000d370       ??_C@_0CJ@CIIOKEJA@?$FLINFO?$FN?3?5?5?5type?5?$DN?$DN?5cGetObjectDep@ 1001c370     JavaAccessBridge.obj
 0002:0000d39c       ??_C@_0CG@CCMHCDED@?$FLINFO?$FN?3?5?5?5?5?5?9?$DO?5returning?5rResul@ 1001c39c     JavaAccessBridge.obj
 0002:0000d3c4       ??_C@_0CO@HPDBNII@?$FLINFO?$FN?3?5?5?5type?5?$DN?$DN?5cGetActiveDes@ 1001c3c4     JavaAccessBridge.obj
 0002:0000d3f4       ??_C@_0CO@EEGIDCBJ@?$FLINFO?$FN?3?5?5?9?$DO?5returning?5rAccessib@ 1001c3f4     JavaAccessBridge.obj
 0002:0000d424       ??_C@_0DB@BLNOEMHA@?$FLINFO?$FN?3?5?5?5type?5?$DN?$DN?5cGetAccessibl@ 1001c424     JavaAccessBridge.obj
 0002:0000d458       ??_C@_0DI@BBJPLAPN@?$FLINFO?$FN?3?5?5?5type?5?$DN?$DN?5cGetAccessibl@ 1001c458     JavaAccessBridge.obj
 0002:0000d490       ??_C@_0DD@EKFFDOAF@?$FLINFO?$FN?3?5?5?5type?5?$DN?$DN?5cGetAccessibl@ 1001c490     JavaAccessBridge.obj
 0002:0000d4c4       ??_C@_0DI@HCCMIAAH@?$FLINFO?$FN?3?5?5?5type?5?$DN?$DN?5cGetAccessibl@ 1001c4c4     JavaAccessBridge.obj
 0002:0000d4fc       ??_C@_0DK@EHNJMPFO@?$FLINFO?$FN?3?5?5?5?5type?5?$DN?$DN?5cGetAccessib@ 1001c4fc     JavaAccessBridge.obj
 0002:0000d538       ??_C@_0DI@DNENMOMG@?$FLINFO?$FN?3?5?5?5?5?$CD?$CD?$CD?$CD?$CD?5type?5?$DN?$DN?5cGetAc@ 1001c538     JavaAccessBridge.obj
 0002:0000d570       ??_C@_0CG@KFAMLONA@?$FLINFO?$FN?3?5?5?5?5?$CD?$CD?$CD?$CD?$CD?5processing?5suc@ 1001c570     JavaAccessBridge.obj
 0002:0000d598       ??_C@_0EI@KKCFGLCL@?$FLERROR?$FN?3?5?5?5?5?$CD?$CD?$CD?$CD?$CD?5processing?5FA@ 1001c598     JavaAccessBridge.obj
 0002:0000d5e0       ??_C@_0DM@ONBKHFBE@?$FLINFO?$FN?3?5?5?5?5?$CD?$CD?$CD?$CD?$CD?5type?5?$DN?$DN?5cGetAc@ 1001c5e0     JavaAccessBridge.obj
 0002:0000d61c       ??_C@_0DN@MOEKMKGM@?$FLINFO?$FN?3?5?5?5?5?$CD?$CD?$CD?$CD?$CD?5type?5?$DN?$DN?5cGetAc@ 1001c61c     JavaAccessBridge.obj
 0002:0000d660       ??_C@_0EA@CAKJDHMA@?$FLINFO?$FN?3?5?5?5?5?$CD?$CD?$CD?$CD?$CD?5type?5?$DN?$DN?5cGetAc@ 1001c660     JavaAccessBridge.obj
 0002:0000d6a0       ??_C@_0EC@JLIHGBEM@?$FLINFO?$FN?3?5?5?5?5?$CD?$CD?$CD?$CD?$CD?5type?5?$DN?$DN?5cGetAc@ 1001c6a0     JavaAccessBridge.obj
 0002:0000d6e8       ??_C@_0EF@DBAFGNDK@?$FLINFO?$FN?3?5?5?5?5?$CD?$CD?$CD?$CD?$CD?5type?5?$DN?$DN?5cGetAc@ 1001c6e8     JavaAccessBridge.obj
 0002:0000d730       ??_C@_0EI@BCPJNOBP@?$FLINFO?$FN?3?5?5?5?5?$CD?$CD?$CD?$CD?$CD?5type?5?$DN?$DN?5cGetAc@ 1001c730     JavaAccessBridge.obj
 0002:0000d778       ??_C@_0EF@ONIGGHFH@?$FLINFO?$FN?3?5?5?5?5?$CD?$CD?$CD?$CD?$CD?5type?5?$DN?$DN?5cGetAc@ 1001c778     JavaAccessBridge.obj
 0002:0000d7c0       ??_C@_0DO@ENBHEGBB@?$FLINFO?$FN?3?5?5?5?5?$CD?$CD?$CD?$CD?$CD?5type?5?$DN?$DN?5cIsAcc@ 1001c7c0     JavaAccessBridge.obj
 0002:0000d800       ??_C@_0EB@PMALJKOF@?$FLINFO?$FN?3?5?5?5?5?$CD?$CD?$CD?$CD?$CD?5type?5?$DN?$DN?5cIsAcc@ 1001c800     JavaAccessBridge.obj
 0002:0000d848       ??_C@_0EE@NFLEEFCE@?$FLINFO?$FN?3?5?5?5?5?$CD?$CD?$CD?$CD?$CD?5type?5?$DN?$DN?5cGetAc@ 1001c848     JavaAccessBridge.obj
 0002:0000d890       ??_C@_0EH@DNDNECPC@?$FLINFO?$FN?3?5?5?5?5?5?5?$CD?$CD?$CD?$CD?$CD?5cGetAccessib@ 1001c890     JavaAccessBridge.obj
 0002:0000d8d8       ??_C@_0EF@PFDKDHMH@?$FLINFO?$FN?3?5?5?5?5?5?5?$CD?$CD?$CD?$CD?$CD?5cGetAccessib@ 1001c8d8     JavaAccessBridge.obj
 0002:0000d920       ??_C@_0EB@FNPEGMEK@?$FLINFO?$FN?3?5?5?5?5?$CD?$CD?$CD?$CD?$CD?5type?5?$DN?$DN?5cGetAc@ 1001c920     JavaAccessBridge.obj
 0002:0000d964       ??_C@_0DH@HGKABJI@?$FLINFO?$FN?3?5?5?5?5?$CD?$CD?$CD?$CD?$CD?5type?5?$DN?$DN?5cGetAc@ 1001c964     JavaAccessBridge.obj
 0002:0000d99c       ??_C@_0DK@PHHNIBJB@?$FLINFO?$FN?3?5?5?5?5?$CD?$CD?$CD?$CD?$CD?5type?5?$DN?$DN?5cGetAc@ 1001c99c     JavaAccessBridge.obj
 0002:0000d9d8       ??_C@_0DJ@ECCDOPKO@?$FLINFO?$FN?3?5?5?5?5?$CD?$CD?$CD?$CD?$CD?5type?5?$DN?$DN?5cGetAc@ 1001c9d8     JavaAccessBridge.obj
 0002:0000da14       ??_C@_0DK@GDIGFCLP@?$FLINFO?$FN?3?5?5?5?5?$CD?$CD?$CD?$CD?$CD?5type?5?$DN?$DN?5cGetAc@ 1001ca14     JavaAccessBridge.obj
 0002:0000da50       ??_C@_0DI@BPKDDCHO@?$FLINFO?$FN?3?5?5?5?5?$CD?$CD?$CD?$CD?$CD?5type?5?$DN?$DN?5cGetAc@ 1001ca50     JavaAccessBridge.obj
 0002:0000da88       ??_C@_0DN@OAAMPEIM@?$FLINFO?$FN?3?5?5?5?5?$CD?$CD?$CD?$CD?$CD?5type?5?$DN?$DN?5cActiv@ 1001ca88     JavaAccessBridge.obj
 0002:0000dac8       ??_C@_0DN@GBPFAJCJ@?$FLINFO?$FN?3?5?5?5?5?$CD?$CD?$CD?$CD?$CD?5type?5?$DN?$DN?5cGetAc@ 1001cac8     JavaAccessBridge.obj
 0002:0000db08       ??_C@_0DM@HFKCAKHD@?$FLINFO?$FN?3?5?5?5?5?$CD?$CD?$CD?$CD?$CD?5processing?5suc@ 1001cb08     JavaAccessBridge.obj
 0002:0000db44       ??_C@_0DL@BKPFGPAI@?$FLINFO?$FN?3?5?5?5?5?$CD?$CD?$CD?$CD?$CD?5type?5?$DN?$DN?5cGetAc@ 1001cb44     JavaAccessBridge.obj
 0002:0000db80       ??_C@_0EB@HBBMKHLL@?$FLINFO?$FN?3?5?5?5?5?$CD?$CD?$CD?$CD?$CD?5type?5?$DN?$DN?5cGetAc@ 1001cb80     JavaAccessBridge.obj
 0002:0000dbc4       ??_C@_0DI@EGGEEHLE@?$FLINFO?$FN?3?5?5?5?5?$CD?$CD?$CD?$CD?$CD?5type?5?$DN?$DN?5cGetAc@ 1001cbc4     JavaAccessBridge.obj
 0002:0000dbfc       ??_C@_0DK@LOBFOEFG@?$FLINFO?$FN?3?5?5?5?5?$CD?$CD?$CD?$CD?$CD?5type?5?$DN?$DN?5cGetAc@ 1001cbfc     JavaAccessBridge.obj
 0002:0000dc38       ??_C@_0DE@NCPKKLJG@?$FLINFO?$FN?3?5?5?5?5?$CD?$CD?$CD?$CD?$CD?5type?5?$DN?$DN?5cGetAc@ 1001cc38     JavaAccessBridge.obj
 0002:0000dc70       ??_C@_0EH@OKFMNJOP@?$FLERROR?$FN?3?5?5?5?$CD?$CD?$CD?$CD?$CD?5processing?5FAI@ 1001cc70     JavaAccessBridge.obj
 0002:0000dcb8       ??_C@_0DG@CDFKKFMN@?$FLINFO?$FN?3?5?5?5?5?$CD?$CD?$CD?$CD?$CD?5type?5?$DN?$DN?5cGetAc@ 1001ccb8     JavaAccessBridge.obj
 0002:0000dcf0       ??_C@_0DF@GOCDLFHO@?$FLINFO?$FN?3?5?5?5?5?$CD?$CD?$CD?$CD?$CD?5type?5?$DN?$DN?5cDoAcc@ 1001ccf0     JavaAccessBridge.obj
 0002:0000dd28       ??_C@_0DJ@FOPNGHK@?$FLINFO?$FN?3?5?5?5?5?$CD?$CD?$CD?$CD?$CD?5type?5?$DN?$DN?5GetVir@ 1001cd28     JavaAccessBridge.obj
 0002:0000dd64       ??_C@_0CN@KKAHFJLP@?$FLINFO?$FN?3?5?5?5?5?$CD?$CD?$CD?$CD?$CD?5type?5?$DN?$DN?5Reques@ 1001cd64     JavaAccessBridge.obj
 0002:0000dd94       ??_C@_0DA@BDJNNLOI@?$FLINFO?$FN?3?5?5?5?5?$CD?$CD?$CD?$CD?$CD?5type?5?$DN?$DN?5Select@ 1001cd94     JavaAccessBridge.obj
 0002:0000ddc4       ??_C@_0DJ@JNPDLANK@?$FLINFO?$FN?3?5?5?5?5?$CD?$CD?$CD?$CD?$CD?5type?5?$DN?$DN?5GetTex@ 1001cdc4     JavaAccessBridge.obj
 0002:0000de00       ??_C@_0DI@KCHGBBIN@?$FLINFO?$FN?3?5?5?5?5?$CD?$CD?$CD?$CD?$CD?5type?5?$DN?$DN?5GetVis@ 1001ce00     JavaAccessBridge.obj
 0002:0000de38       ??_C@_0DD@HFEKHIPA@?$FLINFO?$FN?3?5?5?5?5?$CD?$CD?$CD?$CD?$CD?5type?5?$DN?$DN?5GetVis@ 1001ce38     JavaAccessBridge.obj
 0002:0000de6c       ??_C@_0DB@HDPFDIKC@?$FLINFO?$FN?3?5?5?5?5?$CD?$CD?$CD?$CD?$CD?5type?5?$DN?$DN?5SetCar@ 1001ce6c     JavaAccessBridge.obj
 0002:0000dea0       ??_C@_0DB@MBKJOFKA@?$FLINFO?$FN?3?5?5?5?5type?5?$DN?$DN?5cGetAccessib@ 1001cea0     JavaAccessBridge.obj
 0002:0000ded4       ??_C@_0DC@FACNMLJM@?$FLINFO?$FN?3?5?5?5?5type?5?$DN?$DN?5cGetAccessib@ 1001ced4     JavaAccessBridge.obj
 0002:0000df08       ??_C@_0DK@BMAJHBGM@?$FLINFO?$FN?3?5?5?5?5type?5?$DN?$DN?5cGetAccessib@ 1001cf08     JavaAccessBridge.obj
 0002:0000df44       ??_C@_0DK@KLKIIEMH@?$FLINFO?$FN?3?5?5?5?5type?5?$DN?$DN?5cGetAccessib@ 1001cf44     JavaAccessBridge.obj
 0002:0000df80       ??_C@_0DF@LJIJJCFL@?$FLINFO?$FN?3?5?5?5?5type?5?$DN?$DN?5cGetAccessib@ 1001cf80     JavaAccessBridge.obj
 0002:0000dfb8       ??_C@_0CM@DKHFKJOD@?$FLINFO?$FN?3?5?5?5?5type?5?$DN?$DN?5cGetCaretLoc@ 1001cfb8     JavaAccessBridge.obj
 0002:0000dfe4       ??_C@_0DH@CHPJDHJL@?$FLINFO?$FN?3?5?5?5?5type?5?$DN?$DN?5cGetAccessib@ 1001cfe4     JavaAccessBridge.obj
 0002:0000e01c       ??_C@_0DC@HMIBGEHP@?$FLINFO?$FN?3?5?5?5?5type?5?$DN?$DN?5cGetAccessib@ 1001d01c     JavaAccessBridge.obj
 0002:0000e050       ??_C@_0EA@OJBBPFCG@?$FLINFO?$FN?3?5?5?5?5type?5?$DN?$DN?5cGetCurrentA@ 1001d050     JavaAccessBridge.obj
 0002:0000e090       ??_C@_0EA@FFJJPODP@?$FLINFO?$FN?3?5?5?5?5type?5?$DN?$DN?5cGetMaximumA@ 1001d090     JavaAccessBridge.obj
 0002:0000e0d0       ??_C@_0EA@GABLOPGB@?$FLINFO?$FN?3?5?5?5?5type?5?$DN?$DN?5cGetMinimumA@ 1001d0d0     JavaAccessBridge.obj
 0002:0000e110       ??_C@_0DN@NHMKNOBO@?$FLINFO?$FN?3?5?5?5?5type?5?$DN?$DN?5cAddAccessib@ 1001d110     JavaAccessBridge.obj
 0002:0000e150       ??_C@_0DP@CDAIIOJL@?$FLINFO?$FN?3?5?5?5?5type?5?$DN?$DN?5cClearAccess@ 1001d150     JavaAccessBridge.obj
 0002:0000e190       ??_C@_0DN@FGNKIKEK@?$FLINFO?$FN?3?5?5?5?5type?5?$DN?$DN?5cGetAccessib@ 1001d190     JavaAccessBridge.obj
 0002:0000e1d0       ??_C@_0EC@JGIFJEAP@?$FLINFO?$FN?3?5?5?5?5type?5?$DN?$DN?5cGetAccessib@ 1001d1d0     JavaAccessBridge.obj
 0002:0000e218       ??_C@_0EA@BDFAJBM@?$FLINFO?$FN?3?5?5?5?5type?5?$DN?$DN?5cIsAccessibl@ 1001d218     JavaAccessBridge.obj
 0002:0000e258       ??_C@_0EA@NOOOKPJ@?$FLINFO?$FN?3?5?5?5?5type?5?$DN?$DN?5cRemoveAcces@ 1001d258     JavaAccessBridge.obj
 0002:0000e298       ??_C@_0ED@CNEBOKEO@?$FLINFO?$FN?3?5?5?5?5type?5?$DN?$DN?5cSelectAllAc@ 1001d298     JavaAccessBridge.obj
 0002:0000e2dc       ??_C@_0DD@FDABBAIG@?$FLINFO?$FN?3?5?5?5?5type?5?$DN?5cAddJavaEvent@ 1001d2dc     JavaAccessBridge.obj
 0002:0000e310       ??_C@_0DG@CJJGFHBD@?$FLINFO?$FN?3?5?5?5?5type?5?$DN?5cRemoveJavaEv@ 1001d310     JavaAccessBridge.obj
 0002:0000e348       ??_C@_0DM@IHHPMOM@?$FLINFO?$FN?3?5?5?5?5type?5?$DN?5cAddAccessibi@ 1001d348     JavaAccessBridge.obj
 0002:0000e384       ??_C@_0DP@CLPLFGHM@?$FLINFO?$FN?3?5?5?5?5type?5?$DN?5cRemoveAccess@ 1001d384     JavaAccessBridge.obj
 0002:0000e3c8       ??_C@_0EG@DADDGPDA@?$FLERROR?$FN?3?5?5?5?5processing?5FAILED?$CB?$CB@ 1001d3c8     JavaAccessBridge.obj
 0002:0000e410       ??_C@_0CI@PMGDCMNI@?$FLINFO?$FN?3?5?5?5?5package?5processing?5c@ 1001d410     JavaAccessBridge.obj
 0002:0000e438       ??_C@_0CO@NOIJCKLH@?$FLINFO?$FN?3?5?5?5in?5MemoryMappedFileCr@ 1001d438     JavaAccessBridge.obj
 0002:0000e468       ??_C@_0DJ@MGBOAEHL@?$FLINFO?$FN?3?5?5?5?5?5just?5created?5a?5new?5@ 1001d468     JavaAccessBridge.obj
 0002:0000e4a4       ??_C@_0DA@PCLBAGKL@?$FLINFO?$FN?3?5?5?5Successfully?5initiate@ 1001d4a4     JavaAccessBridge.obj
 0002:0000e4d4       ??_C@_0CL@IAFANAPB@?$FLERROR?$FN?3?5Failed?5to?5initiate?5IPC@ 1001d4d4     JavaAccessBridge.obj
 0002:0000e500       ??_C@_0DE@FDNKAIDO@?$FLINFO?$FN?3?5in?5JavaAccessBridge?3?3Wi@ 1001d500     JavaAccessBridge.obj
 0002:0000e534       ??_C@_0CO@DDCCLLBJ@?$FLERROR?$FN?3?5?9?$DO?5ATs?5?$DN?$DN?50?$CB?5?$CIshouldn?8@ 1001d534     JavaAccessBridge.obj
 0002:0000e564       ??_C@_0CP@IIHJFGGB@?$FLINFO?$FN?3?5?5?5data?5structures?5succe@ 1001d564     JavaAccessBridge.obj
 0002:0000e594       ??_C@_0DB@JABMCGEJ@?$FLERROR?$FN?3?5couldn?8t?5find?5matching@ 1001d594     JavaAccessBridge.obj
 0002:0000e5c8       ??_C@_0CP@LEPCODGO@?$FLINFO?$FN?3?5In?5JavaAccessBridge?3?3re@ 1001d5c8     JavaAccessBridge.obj
 0002:0000e5f8       ??_C@_0BH@GNOIGMFE@?$FLINFO?$FN?3?5?5?5object?5X?3?5?$CFp@ 1001d5f8     JavaAccessBridge.obj
 0002:0000e610       ??_C@_0CE@NAEKPPND@?$FLINFO?$FN?3?5?5?5global?5reference?5dele@ 1001d610     JavaAccessBridge.obj
 0002:0000e634       ??_C@_0CC@DPMNCGAA@?$FLERROR?$FN?3?5windowsThreadJNIEnv?5?$DN?$DN@ 1001d634     JavaAccessBridge.obj
 0002:0000e658       ??_C@_0DF@HMNKBJGB@?$FLINFO?$FN?3?5?5?5adding?5Java?5event?5typ@ 1001d658     JavaAccessBridge.obj
 0002:0000e690       ??_C@_0CO@OPGCCICC@?$FLINFO?$FN?3?5?5?5found?5HWND?0?5javaEvent@ 1001d690     JavaAccessBridge.obj
 0002:0000e6c0       ??_C@_0CP@MJMPLPDN@?$FLINFO?$FN?3?5?5?5union?5of?5all?5Java?5AT?5@ 1001d6c0     JavaAccessBridge.obj
 0002:0000e6f0       ??_C@_0FO@PMMLAHPF@?$FLINFO?$FN?3?5?5?5no?5other?5AT?5wanted?5th@ 1001d6f0     JavaAccessBridge.obj
 0002:0000e750       ??_C@_0DJ@DFJLLFAC@?$FLINFO?$FN?3?5?5?5removing?5Java?5event?5t@ 1001d750     JavaAccessBridge.obj
 0002:0000e790       ??_C@_0FO@LBFBGKHJ@?$FLINFO?$FN?3?5?5?5no?5other?5AT?5wanted?5th@ 1001d790     JavaAccessBridge.obj
 0002:0000e7f0       ??_C@_0DN@PDHOAFNL@?$FLINFO?$FN?3?5?5?5adding?5Accesibility?5e@ 1001d7f0     JavaAccessBridge.obj
 0002:0000e830       ??_C@_0DH@EPKDBDGJ@?$FLINFO?$FN?3?5?5?5found?5HWND?0?5accessibi@ 1001d830     JavaAccessBridge.obj
 0002:0000e868       ??_C@_0DI@IJKEHAJM@?$FLINFO?$FN?3?5?5?5union?5of?5all?5Accessib@ 1001d868     JavaAccessBridge.obj
 0002:0000e8a0       ??_C@_0GG@CGBBDJFJ@?$FLINFO?$FN?3?5?5?5no?5other?5AT?5wanted?5th@ 1001d8a0     JavaAccessBridge.obj
 0002:0000e908       ??_C@_0EB@PJLIMJAJ@?$FLINFO?$FN?3?5?5?5removing?5Accesibility@ 1001d908     JavaAccessBridge.obj
 0002:0000e950       ??_C@_0GH@FGGMCIOE@?$FLINFO?$FN?3?5?5?5no?5other?5AT?5wanted?5th@ 1001d950     JavaAccessBridge.obj
 0002:0000e9b8       ??_C@_0GL@DLLNHKDB@?$FLINFO?$FN?3?5Java_com_sun_java_acces@ 1001d9b8     JavaAccessBridge.obj
 0002:0000ea24       ??_C@_0BI@GOJFHMPI@?$FLINFO?$FN?3?5?5?5sending?5to?5AT@ 1001da24     JavaAccessBridge.obj
 0002:0000ea40       ??_C@_0EA@HDPEOOCD@?$FLINFO?$FN?3?5?5?5GlobalRef?8d?5Event?3?5?$CFp@ 1001da40     JavaAccessBridge.obj
 0002:0000ea80       ??_C@_0CN@HLLEMELD@?$FLINFO?$FN?3?5?5done?5with?5propertyCare@ 1001da80     JavaAccessBridge.obj
 0002:0000eab0       ??_C@_0HB@FIEPPBDD@?$FLINFO?$FN?3?5Java_com_sun_java_acces@ 1001dab0     JavaAccessBridge.obj
 0002:0000eb24       ??_C@_0BL@ENCPOIKC@java?1lang?1OutOfMemoryError@ 1001db24     JavaAccessBridge.obj
 0002:0000eb40       ??_C@_1O@CEDCILHN@?$AA?$CI?$AAn?$AAu?$AAl?$AAl?$AA?$CJ@ 1001db40     JavaAccessBridge.obj
 0002:0000eb50       ??_C@_0DE@IIPLELBE@?$FLINFO?$FN?3?5?5?5done?5with?5propertyDes@ 1001db50     JavaAccessBridge.obj
 0002:0000eb88       ??_C@_0GK@FGEOELMA@?$FLINFO?$FN?3?5Java_com_sun_java_acces@ 1001db88     JavaAccessBridge.obj
 0002:0000ebf4       ??_C@_0CM@LHIINGJI@?$FLINFO?$FN?3?5?5done?5with?5propertyName@ 1001dbf4     JavaAccessBridge.obj
 0002:0000ec20       ??_C@_0GH@NDFIEILD@?$FLINFO?$FN?3?5Java_com_sun_java_acces@ 1001dc20     JavaAccessBridge.obj
 0002:0000ec88       ??_C@_0DC@IDEPNPKP@?$FLINFO?$FN?3?5?5?5done?5with?5propertySel@ 1001dc88     JavaAccessBridge.obj
 0002:0000ecc0       ??_C@_0GL@LHHKNKCF@?$FLINFO?$FN?3?5Java_com_sun_java_acces@ 1001dcc0     JavaAccessBridge.obj
 0002:0000ed2c       ??_C@_0DI@HBGABKPB@?$FLINFO?$FN?3?5?5?5GlobalRef?8d?5Event?3?5?$CFp@ 1001dd2c     JavaAccessBridge.obj
 0002:0000ed64       ??_C@_0CN@HPCDPOIL@?$FLINFO?$FN?3?5?5done?5with?5propertyStat@ 1001dd64     JavaAccessBridge.obj
 0002:0000ed98       ??_C@_0GC@GKPNHBKM@?$FLINFO?$FN?3?5Java_com_sun_java_acces@ 1001dd98     JavaAccessBridge.obj
 0002:0000edfc       ??_C@_0CM@MKJMCAOF@?$FLINFO?$FN?3?5?5done?5with?5propertyText@ 1001ddfc     JavaAccessBridge.obj
 0002:0000ee28       ??_C@_0GL@LMHLMBIC@?$FLINFO?$FN?3?5Java_com_sun_java_acces@ 1001de28     JavaAccessBridge.obj
 0002:0000ee94       ??_C@_0CO@LJOPOKFE@?$FLINFO?$FN?3?5?5?5done?5with?5propertyVal@ 1001de94     JavaAccessBridge.obj
 0002:0000eec8       ??_C@_0GJ@PEJPEKID@?$FLINFO?$FN?3?5Java_com_sun_java_acces@ 1001dec8     JavaAccessBridge.obj
 0002:0000ef34       ??_C@_0DD@LNFBPAKO@?$FLINFO?$FN?3?5?5done?5with?5propertyVisi@ 1001df34     JavaAccessBridge.obj
 0002:0000ef68       ??_C@_0HD@JKCIIIAC@?$FLINFO?$FN?3?5Java_com_sun_java_acces@ 1001df68     JavaAccessBridge.obj
 0002:0000efdc       ??_C@_0BH@HMENLEAO@?$FLINFO?$FN?3?5?5sending?5to?5AT@ 1001dfdc     JavaAccessBridge.obj
 0002:0000eff8       ??_C@_0GP@GEKEHDBB@?$FLINFO?$FN?3?5?5GlobalRef?8d?5Event?3?5?$CFp?5@ 1001dff8     JavaAccessBridge.obj
 0002:0000f068       ??_C@_0CN@LGDOHOEO@?$FLINFO?$FN?3?5?5done?5with?5propertyChil@ 1001e068     JavaAccessBridge.obj
 0002:0000f098       ??_C@_0HO@MNNKGDDP@?$FLINFO?$FN?3?5Java_com_sun_java_acces@ 1001e098     JavaAccessBridge.obj
 0002:0000f118       ??_C@_0IG@DNLGNOND@?$FLINFO?$FN?3?5?5?5GlobalRef?8d?5Event?3?5?$CFp@ 1001e118     JavaAccessBridge.obj
 0002:0000f1a0       ??_C@_0CO@GOOPPCJH@?$FLINFO?$FN?3?5?5done?5with?5propertyActi@ 1001e1a0     JavaAccessBridge.obj
 0002:0000f1d0       ??_C@_0GP@NILNKGMP@?$FLINFO?$FN?3?5Java_com_sun_java_acces@ 1001e1d0     JavaAccessBridge.obj
 0002:0000f240       ??_C@_0BA@KOMOFG@?5?5sending?5to?5AT@ 1001e240     JavaAccessBridge.obj
 0002:0000f250       ??_C@_0DC@FMNGEBKI@?$FLINFO?$FN?3?5?5done?5with?5propertyTabl@ 1001e250     JavaAccessBridge.obj
 0002:0000f284       ??_C@_0DA@ODJJOIDA@?$FLINFO?$FN?3?5Firing?5event?5id?5?$DN?5?$CFd?$CI?$CFp@ 1001e284     JavaAccessBridge.obj
 0002:0000f2b4       ??_C@_0CF@EPNHEIBO@?$FLINFO?$FN?3?5?5?5done?5with?5firing?5AWT?5@ 1001e2b4     JavaAccessBridge.obj
 0002:0000f2dc       ??_C@_0DI@NNGMMOBO@?$FLINFO?$FN?3?5Firing?5event?5id?5?$DN?5?$CFd?$CI?$CFp@ 1001e2dc     JavaAccessBridge.obj
 0002:0000f314       ??_C@_0DJ@GLLLDFPO@?$FLINFO?$FN?3?5javaEventMask?5?$DN?5?$CFX?5even@ 1001e314     JavaAccessBridge.obj
 0002:0000f350       ??_C@_1CO@CCIONPKC@?$AAA?$AAc?$AAc?$AAe?$AAs?$AAs?$AAB?$AAr?$AAi?$AAd?$AAg?$AAe?$AA?4?$AAj?$AAa@ 1001e350     JavaAccessBridge.obj
 0002:0000f380       __pDefaultRawDllMain       1001e380     MSVCRT:dll_dllmain.obj
 0002:0000f380       __pRawDllMain              1001e380     MSVCRT:dll_dllmain.obj
 0002:0000f388       ??_7exception@std@@6B@     1001e388     MSVCRT:throw_bad_alloc.obj
 0002:0000f390       ??_C@_0BC@EOODALEL@Unknown?5exception@ 1001e390     MSVCRT:throw_bad_alloc.obj
 0002:0000f3a8       ??_7bad_alloc@std@@6B@     1001e3a8     MSVCRT:throw_bad_alloc.obj
 0002:0000f3b0       ??_C@_0P@GHFPNOJB@bad?5allocation@ 1001e3b0     MSVCRT:throw_bad_alloc.obj
 0002:0000f3c4       ??_7bad_array_new_length@std@@6B@ 1001e3c4     MSVCRT:throw_bad_alloc.obj
 0002:0000f3cc       ??_C@_0BF@KINCDENJ@bad?5array?5new?5length@ 1001e3cc     MSVCRT:throw_bad_alloc.obj
 0002:0000f3f0       ??_7type_info@@6B@         1001e3f0     MSVCRT:std_type_info_static.obj
 0002:0000f470       __load_config_used         1001e470     MSVCRT:loadcfg.obj
 0002:0000f510       ??_R4exception@std@@6B@    1001e510     MSVCRT:throw_bad_alloc.obj
 0002:0000f524       ??_R3exception@std@@8      1001e524     MSVCRT:throw_bad_alloc.obj
 0002:0000f534       ??_R2exception@std@@8      1001e534     MSVCRT:throw_bad_alloc.obj
 0002:0000f53c       ??_R1A@?0A@EA@exception@std@@8 1001e53c     MSVCRT:throw_bad_alloc.obj
 0002:0000f558       ??_R4bad_alloc@std@@6B@    1001e558     MSVCRT:throw_bad_alloc.obj
 0002:0000f56c       ??_R3bad_alloc@std@@8      1001e56c     MSVCRT:throw_bad_alloc.obj
 0002:0000f57c       ??_R2bad_alloc@std@@8      1001e57c     MSVCRT:throw_bad_alloc.obj
 0002:0000f588       ??_R1A@?0A@EA@bad_alloc@std@@8 1001e588     MSVCRT:throw_bad_alloc.obj
 0002:0000f5a4       ??_R4bad_array_new_length@std@@6B@ 1001e5a4     MSVCRT:throw_bad_alloc.obj
 0002:0000f5b8       ??_R3bad_array_new_length@std@@8 1001e5b8     MSVCRT:throw_bad_alloc.obj
 0002:0000f5c8       ??_R2bad_array_new_length@std@@8 1001e5c8     MSVCRT:throw_bad_alloc.obj
 0002:0000f5d8       ??_R1A@?0A@EA@bad_array_new_length@std@@8 1001e5d8     MSVCRT:throw_bad_alloc.obj
 0002:0000f5f4       ??_R4type_info@@6B@        1001e5f4     MSVCRT:std_type_info_static.obj
 0002:0000f608       ??_R3type_info@@8          1001e608     MSVCRT:std_type_info_static.obj
 0002:0000f618       ??_R2type_info@@8          1001e618     MSVCRT:std_type_info_static.obj
 0002:0000f620       ??_R1A@?0A@EA@type_info@@8 1001e620     MSVCRT:std_type_info_static.obj
 0002:0000f640       ___safe_se_handler_table   1001e640     <linker-defined>
 0002:0000f8f8       ___rtc_iaa                 1001e8f8     MSVCRT:initsect.obj
 0002:0000f8fc       ___rtc_izz                 1001e8fc     MSVCRT:initsect.obj
 0002:0000f900       ___rtc_taa                 1001e900     MSVCRT:initsect.obj
 0002:0000f904       ___rtc_tzz                 1001e904     MSVCRT:initsect.obj
 0002:0000f964       __TI2?AVbad_alloc@std@@    1001e964     MSVCRT:throw_bad_alloc.obj
 0002:0000f974       __CTA2?AVbad_alloc@std@@   1001e974     MSVCRT:throw_bad_alloc.obj
 0002:0000f980       __CT??_R0?AVbad_alloc@std@@@8??0bad_alloc@std@@QAE@ABV01@@Z12 1001e980     MSVCRT:throw_bad_alloc.obj
 0002:0000f99c       __CT??_R0?AVexception@std@@@8??0exception@std@@QAE@ABV01@@Z12 1001e99c     MSVCRT:throw_bad_alloc.obj
 0002:0000f9b8       __TI3?AVbad_array_new_length@std@@ 1001e9b8     MSVCRT:throw_bad_alloc.obj
 0002:0000f9c8       __CTA3?AVbad_array_new_length@std@@ 1001e9c8     MSVCRT:throw_bad_alloc.obj
 0002:0000f9d8       __CT??_R0?AVbad_array_new_length@std@@@8??0bad_array_new_length@std@@QAE@ABV01@@Z12 1001e9d8     MSVCRT:throw_bad_alloc.obj
 0002:00010498       __IMPORT_DESCRIPTOR_KERNEL32 1001f498     kernel32:KERNEL32.dll
 0002:000104ac       __IMPORT_DESCRIPTOR_USER32 1001f4ac     user32:USER32.dll
 0002:000104c0       __IMPORT_DESCRIPTOR_jawt   1001f4c0     jawt:jawt.dll
 0002:000104d4       __IMPORT_DESCRIPTOR_VCRUNTIME140 1001f4d4     vcruntime:VCRUNTIME140.dll
 0002:000104e8       __IMPORT_DESCRIPTOR_api-ms-win-crt-string-l1-1-0 1001f4e8     ucrt:api-ms-win-crt-string-l1-1-0.dll
 0002:000104fc       __IMPORT_DESCRIPTOR_api-ms-win-crt-runtime-l1-1-0 1001f4fc     ucrt:api-ms-win-crt-runtime-l1-1-0.dll
 0002:00010510       __IMPORT_DESCRIPTOR_api-ms-win-crt-stdio-l1-1-0 1001f510     ucrt:api-ms-win-crt-stdio-l1-1-0.dll
 0002:00010524       __IMPORT_DESCRIPTOR_api-ms-win-crt-environment-l1-1-0 1001f524     ucrt:api-ms-win-crt-environment-l1-1-0.dll
 0002:00010538       __IMPORT_DESCRIPTOR_api-ms-win-crt-heap-l1-1-0 1001f538     ucrt:api-ms-win-crt-heap-l1-1-0.dll
 0002:0001054c       __NULL_IMPORT_DESCRIPTOR   1001f54c     kernel32:KERNEL32.dll
 0003:00000000       ___security_cookie_complement 10020000     MSVCRT:gs_cookie.obj
 0003:00000004       ___security_cookie         10020004     MSVCRT:gs_cookie.obj
 0003:00000008       __fltused                  10020008     MSVCRT:fltused.obj
 0003:0000000c       ___scrt_native_dllmain_reason 1002000c     MSVCRT:utility.obj
 0003:00000010       ___isa_enabled             10020010     MSVCRT:cpu_disp.obj
 0003:00000014       ___scrt_ucrt_dll_is_in_use 10020014     MSVCRT:ucrt_stubs.obj
 0003:00000018       ??_R0?AVbad_alloc@std@@@8  10020018     MSVCRT:throw_bad_alloc.obj
 0003:00000034       ??_R0?AVexception@std@@@8  10020034     MSVCRT:throw_bad_alloc.obj
 0003:00000050       ??_R0?AVbad_array_new_length@std@@@8 10020050     MSVCRT:throw_bad_alloc.obj
 0003:00000078       ??_R0?AVtype_info@@@8      10020078     MSVCRT:std_type_info_static.obj
 0003:00000090       ?JavaBridgeThreadId@@3KA   10020090     AccessBridgeATInstance.obj
 0003:00000098       ?_OptionsStorage@?1??__local_stdio_printf_options@@9@4_KA 10020098     AccessBridgeDebug.obj
 0003:000000a4       ?theFromJavaHelloMsgID@@3IA 100200a4     AccessBridgeMessages.obj
 0003:000000a8       ?theFromWindowsHelloMsgID@@3IA 100200a8     AccessBridgeMessages.obj
 0003:000000ac       ?theJavaAccessBridge@@3PAVJavaAccessBridge@@A 100200ac     JavaAccessBridge.obj
 0003:000000b0       ?theDialogWindow@@3PAUHWND__@@A 100200b0     JavaAccessBridge.obj
 0003:000000b4       ?receiveMemoryIPCLock@@3U_RTL_CRITICAL_SECTION@@A 100200b4     JavaAccessBridge.obj
 0003:000003f0       ?__type_info_root_node@@3U__type_info_node@@A 100203f0     MSVCRT:tncleanup.obj
 0003:000003f8       ?_OptionsStorage@?1??__local_stdio_scanf_options@@9@4_KA 100203f8     MSVCRT:default_local_stdio_options.obj
 0003:00000400       ___scrt_current_native_startup_state 10020400     MSVCRT:utility.obj
 0003:00000404       ___scrt_native_startup_lock 10020404     MSVCRT:utility.obj
 0003:00000424       ___scrt_debugger_hook_flag 10020424     MSVCRT:utility_desktop.obj
 0003:00000428       ___isa_available           10020428     MSVCRT:cpu_disp.obj
 0003:0000042c       ___favor                   1002042c     MSVCRT:cpu_disp.obj
 0003:00000430       ___dyn_tls_init_callback   10020430     <common>

 entry point at        0001:0000c6b9

 Static symbols

 0000:fffdd000       .debug$S                   10000000     ucrt:api-ms-win-crt-string-l1-1-0.dll
 0000:fffdd000       .debug$S                   10000000     kernel32:KERNEL32.dll
 0000:fffdd000       .debug$S                   10000000     kernel32:KERNEL32.dll
 0000:fffdd000       .debug$S                   10000000     kernel32:KERNEL32.dll
 0000:fffdd000       .debug$S                   10000000     kernel32:KERNEL32.dll
 0000:fffdd000       .debug$S                   10000000     kernel32:KERNEL32.dll
 0000:fffdd000       .debug$S                   10000000     kernel32:KERNEL32.dll
 0000:fffdd000       .debug$S                   10000000     kernel32:KERNEL32.dll
 0000:fffdd000       .debug$S                   10000000     kernel32:KERNEL32.dll
 0000:fffdd000       .debug$S                   10000000     kernel32:KERNEL32.dll
 0000:fffdd000       .debug$S                   10000000     kernel32:KERNEL32.dll
 0000:fffdd000       .debug$S                   10000000     kernel32:KERNEL32.dll
 0000:fffdd000       .debug$S                   10000000     kernel32:KERNEL32.dll
 0000:fffdd000       .debug$S                   10000000     user32:USER32.dll
 0000:fffdd000       .debug$S                   10000000     user32:USER32.dll
 0000:fffdd000       .debug$S                   10000000     user32:USER32.dll
 0000:fffdd000       .debug$S                   10000000     user32:USER32.dll
 0000:fffdd000       .debug$S                   10000000     user32:USER32.dll
 0000:fffdd000       .debug$S                   10000000     user32:USER32.dll
 0000:fffdd000       .debug$S                   10000000     user32:USER32.dll
 0000:fffdd000       .debug$S                   10000000     user32:USER32.dll
 0000:fffdd000       .debug$S                   10000000     user32:USER32.dll
 0000:fffdd000       .debug$S                   10000000     jawt:jawt.dll
 0000:fffdd000       .debug$S                   10000000     vcruntime:VCRUNTIME140.dll
 0000:fffdd000       .debug$S                   10000000     vcruntime:VCRUNTIME140.dll
 0000:fffdd000       .debug$S                   10000000     vcruntime:VCRUNTIME140.dll
 0000:fffdd000       .debug$S                   10000000     vcruntime:VCRUNTIME140.dll
 0000:fffdd000       .debug$S                   10000000     vcruntime:VCRUNTIME140.dll
 0000:fffdd000       .debug$S                   10000000     vcruntime:VCRUNTIME140.dll
 0000:fffdd000       .debug$S                   10000000     vcruntime:VCRUNTIME140.dll
 0000:fffdd000       .debug$S                   10000000     ucrt:api-ms-win-crt-string-l1-1-0.dll
 0000:fffdd000       .debug$S                   10000000     ucrt:api-ms-win-crt-string-l1-1-0.dll
 0000:fffdd000       .debug$S                   10000000     ucrt:api-ms-win-crt-string-l1-1-0.dll
 0000:fffdd000       .debug$S                   10000000     ucrt:api-ms-win-crt-runtime-l1-1-0.dll
 0000:fffdd000       .debug$S                   10000000     ucrt:api-ms-win-crt-string-l1-1-0.dll
 0000:fffdd000       .debug$S                   10000000     ucrt:api-ms-win-crt-string-l1-1-0.dll
 0000:fffdd000       .debug$S                   10000000     ucrt:api-ms-win-crt-stdio-l1-1-0.dll
 0000:fffdd000       .debug$S                   10000000     javaaccessbridge.exp
 0000:fffdd000       .debug$S                   10000000     ucrt:api-ms-win-crt-stdio-l1-1-0.dll
 0000:fffdd000       .debug$S                   10000000     kernel32:KERNEL32.dll
 0000:fffdd000       .debug$S                   10000000     kernel32:KERNEL32.dll
 0000:fffdd000       .debug$S                   10000000     kernel32:KERNEL32.dll
 0000:fffdd000       .debug$S                   10000000     kernel32:KERNEL32.dll
 0000:fffdd000       .debug$S                   10000000     kernel32:KERNEL32.dll
 0000:fffdd000       .debug$S                   10000000     kernel32:KERNEL32.dll
 0000:fffdd000       .debug$S                   10000000     kernel32:KERNEL32.dll
 0000:fffdd000       .debug$S                   10000000     kernel32:KERNEL32.dll
 0000:fffdd000       .debug$S                   10000000     kernel32:KERNEL32.dll
 0000:fffdd000       .debug$S                   10000000     kernel32:KERNEL32.dll
 0000:fffdd000       .debug$S                   10000000     kernel32:KERNEL32.dll
 0000:fffdd000       .debug$S                   10000000     kernel32:KERNEL32.dll
 0000:fffdd000       .debug$S                   10000000     ucrt:api-ms-win-crt-stdio-l1-1-0.dll
 0000:fffdd000       .debug$S                   10000000     ucrt:api-ms-win-crt-stdio-l1-1-0.dll
 0000:fffdd000       .debug$S                   10000000     ucrt:api-ms-win-crt-stdio-l1-1-0.dll
 0000:fffdd000       .debug$S                   10000000     ucrt:api-ms-win-crt-environment-l1-1-0.dll
 0000:fffdd000       .debug$S                   10000000     ucrt:api-ms-win-crt-string-l1-1-0.dll
 0000:fffdd000       .debug$S                   10000000     ucrt:api-ms-win-crt-runtime-l1-1-0.dll
 0000:fffdd000       .debug$S                   10000000     ucrt:api-ms-win-crt-runtime-l1-1-0.dll
 0000:fffdd000       .debug$S                   10000000     ucrt:api-ms-win-crt-runtime-l1-1-0.dll
 0000:fffdd000       .debug$S                   10000000     ucrt:api-ms-win-crt-runtime-l1-1-0.dll
 0000:fffdd000       .debug$S                   10000000     ucrt:api-ms-win-crt-runtime-l1-1-0.dll
 0000:fffdd000       .debug$S                   10000000     ucrt:api-ms-win-crt-runtime-l1-1-0.dll
 0000:fffdd000       .debug$S                   10000000     ucrt:api-ms-win-crt-runtime-l1-1-0.dll
 0000:fffdd000       .debug$S                   10000000     ucrt:api-ms-win-crt-runtime-l1-1-0.dll
 0000:fffdd000       .debug$S                   10000000     ucrt:api-ms-win-crt-runtime-l1-1-0.dll
 0000:fffdd000       .debug$S                   10000000     ucrt:api-ms-win-crt-runtime-l1-1-0.dll
 0000:fffdd000       .debug$S                   10000000     ucrt:api-ms-win-crt-heap-l1-1-0.dll
 0000:fffdd000       .debug$S                   10000000     ucrt:api-ms-win-crt-runtime-l1-1-0.dll
 0000:fffdd000       .debug$S                   10000000     ucrt:api-ms-win-crt-runtime-l1-1-0.dll
 0000:fffdd000       .debug$S                   10000000     ucrt:api-ms-win-crt-heap-l1-1-0.dll
 0000:fffdd000       .debug$S                   10000000     ucrt:api-ms-win-crt-heap-l1-1-0.dll
 0000:fffdd000       .debug$S                   10000000     ucrt:api-ms-win-crt-string-l1-1-0.dll
 0001:0000008f       ?JavaBridgeThread@@YGIPAX@Z 1000108f f   AccessBridgeATInstance.obj
 0001:0000011b       ?do_event@@YAXPADHPAUHWND__@@1@Z 1000111b f   AccessBridgeATInstance.obj
 0001:0000bd18       $LN261                     1000cd18     JavaAccessBridge.obj
 0001:0000c320       $$000000                   1000d320     MSVCRT:ulldiv.obj
 0001:0000c399       ?dllmain_crt_dispatch@@YGHQAUHINSTANCE__@@KQAX@Z 1000d399 f   MSVCRT:dll_dllmain.obj
 0001:0000c3ec       ?dllmain_crt_process_attach@@YAHQAUHINSTANCE__@@QAX@Z 1000d3ec f   MSVCRT:dll_dllmain.obj
 0001:0000c4f6       ?dllmain_crt_process_detach@@YAH_N@Z 1000d4f6 f   MSVCRT:dll_dllmain.obj
 0001:0000c588       ?dllmain_dispatch@@YAHQAUHINSTANCE__@@KQAX@Z 1000d588 f   MSVCRT:dll_dllmain.obj
 0001:0000c68e       ?dllmain_raw@@YGHQAUHINSTANCE__@@KQAX@Z 1000d68e f   MSVCRT:dll_dllmain.obj
 0001:0000c919       ___get_entropy             1000d919 f   MSVCRT:gs_support.obj
 0001:0000c9ec       ?find_pe_section@@YAPAU_IMAGE_SECTION_HEADER@@QAEI@Z 1000d9ec f   MSVCRT:utility.obj
 0001:0000ce70       $$000000                   1000de70     MSVCRT:sehprolg4.obj
 0002:0000f3e4       _GS_ExceptionPointers      1001e3e4     MSVCRT:gs_report.obj
 0002:0000f908       __sehtable$?dllmain_crt_process_attach@@YAHQAUHINSTANCE__@@QAX@Z 1001e908     MSVCRT:dll_dllmain.obj
 0002:0000f928       __sehtable$?dllmain_crt_process_detach@@YAH_N@Z 1001e928     MSVCRT:dll_dllmain.obj
 0002:0000f948       __sehtable$?dllmain_dispatch@@YAHQAUHINSTANCE__@@KQAX@Z 1001e948     MSVCRT:dll_dllmain.obj
 0002:0000f9f8       __sehtable$___scrt_is_nonwritable_in_current_image 1001e9f8     MSVCRT:utility.obj
 0002:0000fa20       .edata                     1001ea20     javaaccessbridge.exp
 0002:0000fa48       rgpv                       1001ea48     javaaccessbridge.exp
 0002:0000fac0       rgszName                   1001eac0     javaaccessbridge.exp
 0002:0000fb38       rgwOrd                     1001eb38     javaaccessbridge.exp
 0002:0000fb74       szName                     1001eb74     javaaccessbridge.exp
 0002:0000fb89       $N00001                    1001eb89     javaaccessbridge.exp
 0002:0000fbcf       $N00002                    1001ebcf     javaaccessbridge.exp
 0002:0000fc15       $N00003                    1001ec15     javaaccessbridge.exp
 0002:0000fc59       $N00004                    1001ec59     javaaccessbridge.exp
 0002:0000fc9f       $N00005                    1001ec9f     javaaccessbridge.exp
 0002:0000fd00       $N00006                    1001ed00     javaaccessbridge.exp
 0002:0000fd61       $N00007                    1001ed61     javaaccessbridge.exp
 0002:0000fda8       $N00008                    1001eda8     javaaccessbridge.exp
 0002:0000fdf1       $N00009                    1001edf1     javaaccessbridge.exp
 0002:0000fe38       $N00010                    1001ee38     javaaccessbridge.exp
 0002:0000fe7f       $N00011                    1001ee7f     javaaccessbridge.exp
 0002:0000fec6       $N00012                    1001eec6     javaaccessbridge.exp
 0002:0000ff0c       $N00013                    1001ef0c     javaaccessbridge.exp
 0002:0000ff53       $N00014                    1001ef53     javaaccessbridge.exp
 0002:0000ff9b       $N00015                    1001ef9b     javaaccessbridge.exp
 0002:0000ffe7       $N00016                    1001efe7     javaaccessbridge.exp
 0002:0001003e       $N00017                    1001f03e     javaaccessbridge.exp
 0002:00010093       $N00018                    1001f093     javaaccessbridge.exp
 0002:000100ec       $N00019                    1001f0ec     javaaccessbridge.exp
 0002:0001013a       $N00020                    1001f13a     javaaccessbridge.exp
 0002:00010188       $N00021                    1001f188     javaaccessbridge.exp
 0002:000101dc       $N00022                    1001f1dc     javaaccessbridge.exp
 0002:00010229       $N00023                    1001f229     javaaccessbridge.exp
 0002:0001027b       $N00024                    1001f27b     javaaccessbridge.exp
 0002:000102c9       $N00025                    1001f2c9     javaaccessbridge.exp
 0002:0001031c       $N00026                    1001f31c     javaaccessbridge.exp
 0002:00010369       $N00027                    1001f369     javaaccessbridge.exp
 0002:000103b7       $N00028                    1001f3b7     javaaccessbridge.exp
 0002:0001040b       $N00029                    1001f40b     javaaccessbridge.exp
 0002:0001044b       $N00030                    1001f44b     javaaccessbridge.exp
 0002:0001075a       .idata$6                   1001f75a     kernel32:KERNEL32.dll
 0002:00010816       .idata$6                   1001f816     user32:USER32.dll
 0002:00010834       .idata$6                   1001f834     jawt:jawt.dll
 0002:000108d4       .idata$6                   1001f8d4     vcruntime:VCRUNTIME140.dll
 0002:00010a66       .idata$6                   1001fa66     ucrt:api-ms-win-crt-string-l1-1-0.dll
 0002:00010a88       .idata$6                   1001fa88     ucrt:api-ms-win-crt-runtime-l1-1-0.dll
 0002:00010aaa       .idata$6                   1001faaa     ucrt:api-ms-win-crt-stdio-l1-1-0.dll
 0002:00010aca       .idata$6                   1001faca     ucrt:api-ms-win-crt-environment-l1-1-0.dll
 0002:00010af0       .idata$6                   1001faf0     ucrt:api-ms-win-crt-heap-l1-1-0.dll
 0003:000000a0       _logFP                     100200a0     AccessBridgeDebug.obj
 0003:000000cc       ?__proc_attached@@3HA      100200cc     MSVCRT:dll_dllmain.obj
 0003:000000d0       _GS_ExceptionRecord        100200d0     MSVCRT:gs_report.obj
 0003:00000120       _GS_ContextRecord          10020120     MSVCRT:gs_report.obj
 0003:00000408       ?is_initialized_as_dll@@3_NA 10020408     MSVCRT:utility.obj
 0003:00000409       ?module_local_atexit_table_initialized@@3_NA 10020409     MSVCRT:utility.obj
 0003:0000040c       ?module_local_atexit_table@@3U_onexit_table_t@@A 1002040c     MSVCRT:utility.obj
 0003:00000418       ?module_local_at_quick_exit_table@@3U_onexit_table_t@@A 10020418     MSVCRT:utility.obj
 0004:00000120       $R000000                   10021120     javaaccessbridge.dll.res
 0004:00000338       $R000218                   10021338     javaaccessbridge.dll.res
 0004:000003c8       $R0002A8                   100213c8     javaaccessbridge.dll.res
